:020000040000FA
:100000000212FC022003FFFFFFFFFF02200BFFFF95
:10001000FFFFFF020E5DFFFFFFFFFF02201BFFFF40
:10002000FFFFFF022023FFFFFFFFFF02202BFFFF48
:10003000FFFFFF022033FFFFFFFFFF020EA0FFFFC5
:10004000FFFFFF022043FFFFFFFFFF02204BFFFFE8
:10005000FFFFFF022053FFFFFFFFFF02205BFFFFB8
:10006000FFFFFF022063FFFFFFFFFF02206BFFFF88
:10007000FFFFFF022073FFFFFFFFFF02207BFFFF58
:10008000FFFFFF022083FFFFFFFFFF02208BFFFF28
:10009000FFFF70DFFFFF040000000002000000C847
:1000A0000300030369A5020269A501000000000026
:1000B00004003273000074F8121043900393E06060
:1000C0001590030274FEF0900304744DF0A37405C0
:1000D000F07A011206747F0102116074F712104366
:1000E00074FF1212687E00801F851882851983E0D4
:1000F00064FE70069003877401F085188285198369
:10010000E0F8900384E068F07C017D00AA18AB1948
:10011000120E188B09EA450970030201E98518825D
:10012000851983E064EF70027E07E0C0E0900387EA
:10013000E0F8900385E0FAE82AF8E434001206C7F4
:10014000D0E0F0900387E060A014600E14602A14E1
:10015000603A14605014606680A0900384E4F085D7
:100160001882851983E0900386F0C39480900387FA
:100170004003E4808474028080851882851983E0BE
:10018000900382F090038774030200F9851882853A
:100190001983E0900383F0900386E0601990038751
:1001A00074040200F9900385E004F0F8900386E0FF
:1001B0006860030200FA90038774050200F9900357
:1001C00085E4F0900387F0900384E0F88518828539
:1001D0001983E06860030200FA900382E0644D60D6
:1001E000030200FA12031E8002EEF97401121234A7
:1001F0007F0202116074F712104374FB121268EA56
:10020000FEEBFF75080475090078081212CC740221
:100210001212E57A907B007904120EC17402121258
:1002200034120666121336E0687003A3E069701298
:10023000851882851983E0F47003A3E0F46003025B
:1002400002FE74041212DD1206D38A088B09A80874
:10025000A9097402121336E8F0A3E9F0740412132A
:1002600036E0600879011200B6020317851882850E
:100270001983E0687003A3E0697076851882851998
:1002800083E0F47003A3E0F470197402121336745F
:1002900010F0A37420F08518828519837410F0A3E0
:1002A0007420F075080175090078081212CC7402E8
:1002B0001212E57A247B08120F467402121234756A
:1002C000080478081212CC74021212E57A907B00AE
:1002D0007904120EC1740212123412066612133619
:1002E000E0687003A3E069700479028006790480F5
:1002F0000279031200B68E828F83741E80058E826F
:100300008F83E4F0120666121336E0687003A3E0F0
:1003100069700479018002790074050201ED74EDC1
:1003200012104374F8121268900307E0FA90030663
:10033000E0FB8B08EAF8E4C8F9EB28FEE93408FF93
:10034000751001880C750D068F0974027808121259
:1003500093C39508F8E49509F9740228F50E74031F
:1003600039F50F8E088F09740978081212EDE50827
:10037000F511EE2410F508E43FF509EEF50AEF5407
:1003800001F50B900383E0146054147003020453CE
:100390001470030204CE14601024FE700302058959
:1003A000147003020639020649750D03794E120CCA
:1003B0005890030712065C7402F0A3744012065AA8
:1003C000740812065AF0A3F0751012AA10A90C12A4
:1003D0000674A90D74081212347F0C021160750D99
:1003E00004794E120C58EE450B7005A911120FAC92
:1003F000C3EE9425EF9408503CC3E5089424E50926
:1004000094084031E50E2496F8E50F3420F98882EF
:100410008983E0701BA3AA82AB83E07013900388EA
:100420007401F08882898374A5F08A828B838004AA
:10043000900388E4F075081075090078081212CC52
:100440007C087D03EEFAEFFB120F467402121234A1
:100450000203CB750D05E511C394794006750C01B7
:100460000203CB75124075130078121212CC7C096E
:100470007D037402780A121293AA0AAB0BA9111217
:100480000EC17402121234900307E0A3F090030629
:10049000E0A3F0751043C3EE9425EF9408400302E7
:1004A00003CBC3E5089424E509940850030203CB69
:1004B000900388E070030203CBE50E2497F8E50F64
:1004C0003420F988828983E4F0A3F00203CB750815
:1004D0000475090078081212CC74021212E57A90A1
:1004E0007B007904120EC1740212123474021213CA
:1004F00036E0F8A3E0F9851882851983E068700377
:10050000A3E069851882851983700BE0F47003A35A
:10051000E0F470578009E0F47003A3E0F4700D85F7
:1005200018828519837410F0A37420F012066612E5
:100530001336E8F0A3E9F075080178081212CC74BC
:10054000021212E57A247B08120F4674021212344A
:1005500075080478081212CC74021212E57A907BA6
:10056000007904120EC174021212341206661213BC
:1005700036E0687003A3E0697006750D010203CBD5
:10058000750D02750C070203CB900391E0600764C0
:100590000260030203CBEAFF7A017900120674E0DD
:1005A000600302062D8003120D19120D23E970F766
:1005B000740412133612064E74041213367808129D
:1005C000131A85080C85090D850A0E850B0F9005F9
:1005D000A2780C1212B97404121336780C12130B91
:1005E000E5084509450A450B70CE8EC2E5C554E0C5
:1005F0004FF5C5740412133612064E7404121336E6
:10060000780812131A85080C85090D850A0E850BCA
:100610000F9005A2780C1212B97404121336780CDC
:1006200012130BE5084509450A450B70CE7A01798E
:100630000012067479080203D4EB900393F0700360
:100640000203CB750D090203CB79060203D4E4F053
:10065000A37426F0A3E4F0A3F022F0A3E4F0A3F047
:10066000A3F0A3F0A322851882851983E0F8A3E004
:10067000F974022274F6121043EAFE900305E0D2E8
:10068000E7F0E9A3F0EE900303F08E0A74042AFE6B
:100690007A028004E0620A0AEAF83395E01206C79B
:1006A0008E08C3E89508E99400A2D265D03340E4EF
:1006B000E50AF0740128FC3395E0FD7A027B031211
:1006C0000E487F03021160F9740228F58274033921
:1006D000F5832274E91210437582007583FE1211AE
:1006E000FB8A168B177514007515008A828B83E4BC
:1006F000F0900391E07006D2AAD2AF800464027039
:100700000579001200B6750C00750D20750E007588
:100710000F00900391E0600464027015120D19122D
:1007200000DBE9F87409686003020803790012002D
:10073000B675080075090278081212CC74021212FC
:10074000E5850C08850D09AA08E5095407FB850E07
:100750000A850F0B740B780812124FA908120EC1EC
:1007600074021212347E007F009005AAC0828E109F
:10077000EFF5113395E0F512F513850C08850D0999
:10078000850E0A850F0B780879101212A69005A61F
:1007900078081212B9758305D08278081211DC50DE
:1007A0001D851882851983E5822EF582E5833FF544
:1007B00083E0F9AA14AB151208328A148B150EEED9
:1007C00070010FC3EF940240A09005AE780C121296
:1007D000B99005B2780C1211DC40030207127900BF
:1007E000AA14AB1512083279001208328B15900347
:1007F00091E07004C2AFC2AAEA451570277AA57BC2
:10080000A58021E8700302073174066870030207AF
:100810003174076870030207318516828517837467
:1008200001F080BA7582007583021211FB7F1002FD
:100830001160C008C0097C088A088B09740F780809
:100840001212EDEA25E0FAEB33FBE9A2E75004745B
:10085000014AFAE508A2E0500874216AFA74106BA4
:10086000FBE9C333F91CEC70CFD009D0082274F730
:1008700012104378007900802374942508F582E4EF
:100880003403F583E08A828B83F09004141209F319
:100890004005900414E4F008E87001099004141273
:1008A000095D6007C3E89CE99D40CEE8FAE9FB7F5B
:1008B0000202116074F5121043900498E0FEA3E068
:1008C000FF8F08EEC39508F895E0F9EFC39EE85056
:1008D0000B120ADA701178007900801B247F500116
:1008E00009C39CE99D50EF7A007B008041E004F051
:1008F000D2E908E8700109C3E89CE99D502C8A827E
:100900008B83E0C0E0900499E0FE74182EF582E439
:100910003404F583D0E0120ACA90049AE4F09004FB
:1009200099E0C3947F40C6E480C5E8FAE9FB7F0400
:1009300002116074F7121043C2E990049812095D25
:10094000601874182508F582E43404F583E0F5C1D5
:10095000900498120AF14002E4F00208AFE0F508B2
:10096000A3E065082274F71210437800790090051F
:100970001DE07063A3E0705F75F900C28FC284A2AE
:100980008340FCA28F4004A28350F8E5F9C28FA2F5
:10099000835004D2848040C0E0E0FE749D2EF58236
:1009A000E43404F583D0E0F090051E120AF140D340
:1009B000E4F080CF749D2508F582E43404F583E0EB
:1009C0008A828B83F090051D1209F3400590051D66
:1009D000E4F008E870010990051D12095D6007C385
:1009E000E89CE99D40CEE8497006E4F090051DF0D2
:1009F0000208ABE004120ACEC394802274F81210ED
:100A0000439005A0E0FF8F82A88290059FE0FEEF53
:100A1000C39EE0500DC398F895E0F9120AD97018FA
:100A20008012C398F895E0F9E8247F500109C39C2F
:100A3000E99D4004EC4D70077A007B00020AC58AEC
:100A4000828B83E0F5F9A3AA82AB837801790080D9
:100A500008E004F008E8700109C3E89CE99D50270C
:100A60008A828B83E0C0E09005A0E0FE741F2EF523
:100A700082E43405F583D0E0120ACA9005A0E0C3F1
:100A8000947F40CDE480CCC28FA28340FCC284A27C
:100A90008F4004A28350F890059F120AE4E0F5F914
:100AA000C28F90059FE0FAA3E06A90059F7005123F
:100AB0000AE48005120AF14002E4F0A28350D0D289
:100AC00084E8FAE9FB7F01021160120ACE22F08A63
:100AD000828B83A3AA82AB8322E824FF18E934FF28
:100AE000F9E84922E0FA741F2AF582E43405F58317
:100AF00022E004F0C394802274FB1212687E0090FE
:100B000005CA780812131A9005CA7401F0A3F0A35D
:100B10007469F0A374A5F09005B6780812127E707F
:100B2000030E80159005BA780812127E6008E59DC4
:100B3000541864107003022000120C7EEEA2E050E4
:100B400003020BFBAA18AB191201F5E97003020BA3
:100B5000FB851882851983E0C3943C500CE0F8743F
:100B60003CC398FA95E0FB80047A007B00120D3CB0
:100B7000E97003020BFB900391E06401700C75F8BF
:100B800000C2AB539AF7D2EA805E79071200B680B2
:100B900003120D19120D23E970F77401121336E4D4
:100BA000F0A37426F0A3E4F0A3F0740112133678D6
:100BB0000812131A85080C85090D850A0E850B0F7E
:100BC0009005A2780C1212B97401121336780C1227
:100BD000130BE5084509450A450B70CE758600C222
:100BE000AAC28B539AFBC2E990000174CDF0022097
:100BF00000C2AF75C9AB75C95B80FE750800750989
:100C000000750A00750B00900391E0701BD2AAD208
:100C1000AF79051200B6E07003120D191200DBE97E
:100C2000F8740968700980E9794E120C5880ED74E7
:100C3000016870E2E07017120D199005BE78081275
:100C400012B99005C278081211DC50EBC2AAC2AFEB
:100C500075C9AB75C95B80FEC082C08378109005F2
:100C6000A1E0C399501575B60FE5B4A2E750FAE5B7
:100C7000BBC39940F118E870EDE9F0020D37C0826E
:100C8000C08353BEFBE59DA2E650FA0078F87901D7
:100C900000120AD970FA75C6807480659E70FA4396
:100CA000BE049062707408F0794A120C58900001EA
:100CB00074F5F07403F5D575D489A2A0E4339003DC
:100CC00091F0A2E05029D28453F3F753F3EF53FD90
:100CD000F743FD10538FF753F7DF43FC2043F10236
:100CE00053F5DF75F82043F4F0D2FED2AB802853E1
:100CF000FF3F85FFFF53F1FE43F30C53F2F375867C
:100D00008075C48090049BE4F0A3F075C2D875C5CB
:100D10000B75C402438640801E8003120933A2E98A
:100D200040F922C082C083900498E0F8A3E0686094
:100D300004790180027900D083D0822274F11210EC
:100D40004374FF1212687E00900391E06401706B9F
:100D5000C2849003927401F07508388E098E0A8E51
:100D60000B7C017D00AA18AB19120E188B0DEA45F9
:100D70000D6018851882851983E06410602CE0648A
:100D8000EF70088E088E098E0A8E0B85080C850977
:100D90000D850A0E850B0F9005A278081212B9E591
:100DA0000C450D450E450F70330E900391E0640124
:100DB0007056D284900392E4F08051D2AAD2AF8AC6
:100DC000088B09E4F50AF50B9005C6780C12131A86
:100DD0007808790C120FC379061200B6900391E0DF
:100DE0006003020D61120D191200DBE9F874096845
:100DF000700779061200B680927407686085E86013
:100E00008A74066870A48083C2AFC2AAEEF9740126
:100E10001212347F08021160C082C083900391E0F7
:100E2000700512086E801E900392E06015A28F502C
:100E30000BE5F98A828B83F07A0180027A007B00CD
:100E40008003120965020D37C082C083900391E0D0
:100E500070051208B480031209FC020D37C0E0745B
:100E6000F21210A9900001E064CD700512201380E9
:100E70002AE064F57024E5C1C28BC0E0900415E05F
:100E8000F8749428F582E43403F583D0E0F09004FC
:100E900015120AF14005E4F08001007F01021108FB
:100EA000C0E074F21210A9900001E064CD70051248
:100EB000203B800BE064F57005120933800100804F
:100EC000DA74F51210438908740F5508F50A750B8A
:100ED00000740B780A121293EA2400F8EB3480F9BC
:100EE000E82400E9350BF9E5C7F509A2AFE433F5CD
:100EF0000AC2AFE508C4540FFAE5C754F84AF5C76B
:100F0000740B121336E0FAA3E0FB801C88828983FD
:100F1000E08C828D83F088828983A3A882A9838C48
:100F2000828D83A3AC82AD83EAFEEBFFEE24FF1A31
:100F3000EF34FFFBEE4F70D48509C7E50AA2E092BB
:100F4000AF7F0402116074F7121043ED900389F033
:100F5000ECA3F0A37462F0A37473F0A3E0541FF049
:100F60007409121336E0F508A3E0F509E5083333F8
:100F700054FC90038EF0740678081212EDE5089088
:100F8000038DF090038F7412F0A37442F075D1FEBC
:100F900075D601EA906271F0EBA3F0906270E0D236
:100FA000E1F0E0A2E740FB7F02021160C082C08353
:100FB000E9C333906272F0906270E0D2E0F0D083C7
:100FC000D08222080808EAC0E0EBC0E086F0E7A47F
:100FD000FA180986F0E7A42AFA180986F0E7A42A85
:100FE000FA180986F0E7A42AFA1986F0E7A4FBE5C7
:100FF000F02AFA190886F0E7A42BFBE5F03AFA1973
:101000000886F0E7A42BFBE5F03AFA18180986F0F9
:10101000E7A4C5F02BFBE43AFA1908E7C5F0C6A42B
:1010200026F6E5F03BFBE43AFA1886F0E7A4F6E58D
:10103000F00826F6E43B08F6E43A08F6D0E0FBD0E8
:10104000E0FA222518C582C0E0E51934FFC583C047
:10105000E0E518C3958224F910AF088583198582CD
:10106000188008858319858218D2AFCEF0A3E520B9
:10107000F0A37808E608F0A3DEFAEFF0A3E58124F8
:10108000FBF8E608F0A3E608F0A30808E608F0A3DA
:10109000E608F0A315811581D0E0FED0E0F81581B7
:1010A0001581E8C0E0EEC0E022C0D02518C582C09E
:1010B000E0E51934FFC583C0E0E518C3958224F349
:1010C00010AF088583198582188008858319858269
:1010D00018D2AFC8F0A3E9F0A3EAF0A3EBF0A3792C
:1010E00008E709F0A3D8FAECF0A3EDF0A3EEF0A323
:1010F000EFF0A3D0E0F0A3D0E0F0A3D0E0F0A3E5C0
:1011000020F0A3E5F0F0A322851983851882E0C0C2
:10111000E0A3E0F9A3E0FAA3E0FBA37808E0F60877
:10112000A3DFFAE0FCA3E0FDA3E0FEA3E0FFA3E061
:10113000C0E0A3E0C0E0A3E0F5D0A3E0F520A3E089
:10114000A3F5F010AF088583198582188008858380
:1011500019858218D2AFD082D083D0E0F8D0E032A7
:10116000851983851882E0A3FEE0A3F5207808E0C6
:10117000A3F608DFFAE0A3FFE0A3C0E0E0A3C0E02D
:10118000E0A3C0E0E0A3C0E010AF0885821885832B
:10119000198008858218858319D2AFD083D0822226
:1011A000E490030278A179038002F0A3D8FCD9FA75
:1011B0007AA27B0590008E782979018015E493A3AB
:1011C000AD82AE838A828B83F0A3AA82AB838D82A9
:1011D0008E83D8E9D9E7120AF8121340C008C3E099
:1011E00096F50808A3E096420808A3E0964208088E
:1011F000A3E09645087001D3D00822C5822518C502
:1012000082C583351910AF07F5198582188007F557
:1012100019858218D2AFC583222518F58210AF0830
:10122000F518400C15198008F51840021519D2AFB1
:101230008519832200C0D0251810AF08F518500C6E
:1012400005198008F51850020519D2AFD0D02260D8
:1012500016080808C6C313C618C613C618C613C690
:1012600018C613C6D5E0EA22251810AF08F51840B5
:101270000C15198008F51840021519D2AF22E06646
:10128000701008A3E066700A08A3E066700408A363
:10129000E06622700422600D18C6C333C608C63348
:1012A000C6D5E0F41822E627F60809E637F608095D
:1012B000E637F60809E637F622E026F608A3E03618
:1012C000F608A3E036F608A3E036F62274028000A2
:1012D000C0E0F404121219D0E0121329222518FAE2
:1012E000E43519FB222518FCE43519FD22600C08B1
:1012F000C6C313C618C613C6D5E0F42275D0007550
:10130000813F7518027519030211A0E6F008A3E6E3
:10131000F008A3E6F008A3E6F022E0F608A3E0F662
:1013200008A3E0F608A3E0F622CAC0E0E6F0A308AE
:10133000DAFAD0E0FA222518F582E43519F583228D
:1013400000000080FBFFFFFFFFFFFFFFFFFFFFFF2D
:10135000FFFFFFFFFFFFFFFFFFFFFFFFFFFFFFFF9D
:10136000FFFFFFFFFFFFFFFFFFFFFFFFFFFFFFFF8D
:10137000FFFFFFFFFFFFFFFFFFFFFFFFFFFFFFFF7D
:10138000FFFFFFFFFFFFFFFFFFFFFFFFFFFFFFFF6D
:0A1FF600CA05094338860000000008
:020000040003F7
:01FFF000F020
:020000040000FA
:10200000022C420221EAFFFFFFFFFFFFFFFFFFFF5D
:10201000FFFFFFFFFFFFFFFFFFFFFFFFFFFFFFFFD0
:10202000FFFFFFFFFFFFFFFFFFFFFF02291CFFFF76
:10203000FFFFFFFFFFFFFFFFFFFFFFFFFFFFFFFFB0
:10204000FFFFFF022749FFFFFFFFFFFFFFFFFFFF2B
:10205000FFFFFF022126FFFFFFFFFFFFFFFFFFFF44
:10206000FFFFFFFFFFFFFFFFFFFFFF0228F4FFFF5F
:10207000FFFFFFFFFFFFFFFFFFFFFFFFFFFFFFFF70
:10208000FFFFFF02218601FFFFFFFFFFFFFFFFFFB2
:102090001020102001FF01010503010F10FEFF10A9
:1020A0004D00000000A84C00000000FF000000FFF1
:1020B00000010000C139000000001339FF3A5B390C
:1020C000753A0000493900000000000000000000DF
:1020D0000000000000000000000000000000FF0100
:1020E0000100A907000000E803FFFF2408E80364DB
:1020F000006400B8010202000800000502070101A7
:10210000051E02051E020A0A0103B80B02803E01E9
:1021100002FEFFE8030A050001FFFF0A01E09651F5
:1021200018000206FFFFC0E074F2122567A2AFE4B8
:1021300033FED2AFE5A7FFE5A1F5085F54106006B6
:1021400012446575A1EFE5085F5408600812446BFE
:1021500075A1F78024E508A2E092F0EFA2E082F0FA
:102160005017906198E0F8900D5BE0C398A2D2659B
:10217000D0335002E8F075A1FE751A00EEA2E0928D
:10218000AF7F010225C6C0E074F2122567A2AFE45A
:1021900033FED2AF9061A4E0F8759B00E5915854EE
:1021A0000860087591F71244B38023E591585410E4
:1021B00060087591EF1244B98014E591A2E092F0A5
:1021C000E8A2E082F05007E0C2E0F012460F906112
:1021D000A3E0F8E5E9585404600E1245E575E9FB03
:1021E000906193E0A2E640F2808FC0E074F2122585
:1021F00067A2AFE433FED2AF9061A5E0F8E5BF5827
:102200005404600675BFFB124627022179C3E49887
:10221000F8E499F912224E8026C3E49AFAE49BFB73
:10222000E920E7E912224EE498F8E499F922C3E4A0
:1022300098F8E499F912224EE498F8E499F9C3E485
:102240009AFAE49BFB22EB20E7CFE920E7E0B90014
:1022500010BB0008E88AF084F8AAF022E4FBC8FA70
:1022600022EB70227B10C833C8C933C9335007C36F
:102270009AC3DBF280069A50012ADBEAC833F4C81D
:10228000C933F4C9FA2275F008E4C833C8C933C9A0
:1022900033C99AC99B5004C92AC93BD5F0ECFBC885
:1022A00033F4C8E4C9FA2274F512250174FA122A2B
:1022B000C87508047509007808122A217404122AC6
:1022C000AA7AF87B07790312433F7402122A3490EA
:1022D00080B07808122C707402122CC77808122A69
:1022E000DE70497508027509007808122A21740207
:1022F000122AAA7AF67B07790312433F7402122A44
:1023000034851882851983E0F47003A3E0F4601C1F
:10231000851882851983E0F8A3E0F988828983749F
:1023200002F0A3F0A37469F0A374A5F0C2AF75D650
:102330009F0200007406122A347F0402278C0808CA
:1023400008EAC0E0EBC0E086F0E7A4FA180986F0DE
:10235000E7A42AFA180986F0E7A42AFA180986F0F1
:10236000E7A42AFA1986F0E7A4FBE5F02AFA19088F
:1023700086F0E7A42BFBE5F03AFA190886F0E7A40B
:102380002BFBE5F03AFA18180986F0E7A4C5F02B04
:10239000FBE43AFA1908E7C5F0C6A426F6E5F03BD7
:1023A000FBE43AFA1886F0E7A4F6E5F00826F6E42E
:1023B0003B08F6E43A08F6D0E0FBD0E0FA22E4CF9E
:1023C000C0E0E4CEC0E0E4CDC0E0E4CCC0E075F015
:1023D00020E626F608E633F608E633F608E633F696
:1023E000181818EC33FCED33FDEE33FEEF33FFC36A
:1023F000EC9709ED9709EE9709EF97191919400F16
:10240000FFEC97FC09ED97FD09EE97FE191906D52B
:10241000F0BFECF709EDF709EEF709EFF719191915
:10242000D0E0FCD0E0FDD0E0FED0E0FF222518C5D2
:1024300082C0E0E51934FFC583C0E0E518C395828A
:1024400024F810AF088583198582188008858319C0
:10245000858218D2AFCEF0A3E520F0A37808E60875
:10246000F0A3DEFAEFF0A3E58124FAF8E608F0A382
:10247000E608F0A3E608F0A30808E608F0A3E608DB
:10248000F0A315811581D0E0FED0E0F8158115810B
:102490001581E8C0E0EEC0E022122CBCB9000302B6
:1024A00024EBE49004D1781379118002F0A3D8FCD6
:1024B000D9FA781A9020867A01BA00028007E4934C
:1024C000A3F608DAF97AE37B1490209478937901E3
:1024D0008015E493A3AD82AE838A828B83F0A3AA96
:1024E00082AB838D828E83D8E9D9E7758228758384
:1024F0008F74061229E075823B75834A7400122995
:10250000E02518C582C0E0E51934FFC583C0E0E5C9
:1025100018C3958224F910AF088583198582188025
:1025200008858319858218D2AFCEF0A3E520F0A3E9
:102530007808E608F0A3DEFAEFF0A3E58124FBF8C3
:10254000E608F0A3E608F0A30808E608F0A3E6080A
:10255000F0A315811581D0E0FED0E0F8158115813A
:10256000E8C0E0EEC0E022C0D02518C582C0E0E59A
:102570001934FFC583C0E0E518C3958224F310AF7A
:10258000088583198582188008858319858218D269
:10259000AFC8F0A3E9F0A3EAF0A3EBF0A37908E752
:1025A00009F0A3D8FAECF0A3EDF0A3EEF0A3EFF05E
:1025B000A3D0E0F0A3D0E0F0A3D0E0F0A3E520F0BA
:1025C000A3E5F0F0A322851983851882E0C0E0A37B
:1025D000E0F9A3E0FAA3E0FBA37808E0F608A3DFA4
:1025E000FAE0FCA3E0FDA3E0FEA3E0FFA3E0C0E06F
:1025F000A3E0C0E0A3E0F5D0A3E0F520A3E0A3F5BD
:10260000F010AF08858319858218800885831985A5
:102610008218D2AFD082D083D0E0F8D0E032E47319
:1026200075F0108E218F228582268583258518825C
:10263000851983E0CEA3E0CF852682852583EBC96B
:10264000EAC8EDCBECCAC3E833C8E933C9EA33CAF8
:10265000EB33CBC3EA9EF524EB9FF523B35004ABD9
:1026600023AA24EC33CCED33CDD5F0DAAE21AF2262
:1026700022D083D082ECC0E0EDC0E0E493A3FCE480
:1026800093A3FDED4C600D1227CCEC24FFFCED3440
:10269000FFFD80EFE493A3FCE493A3FDED4C600DFC
:1026A00012289FEC24FFFCED34FFFD80EFD0E0FD0D
:1026B000D0E0FCE493A3C0E0E493C0E0228519835A
:1026C000851882E0A3FEE0A3F5207808E0A3F608D1
:1026D000DFFAE0A3FFE0A3C0E0E0A3C0E0E0A3C016
:1026E000E0E0A3C0E0E0A3C0E010AF088582188559
:1026F00083198008858218858319D2AFD083D08250
:102700000229E6D083D082E9C0E0E493A3C386F037
:10271000C5F095F0F908E493A386F0C5F095F07044
:102720000BE493A3C3994005E9048002A3E475F088
:1027300002A42582F582E5F03583F583D0E0F9E443
:1027400093A3C0E0E493C0E022C0E074F2122567D6
:10275000A2AFE433FED2AFC2C09013DBE0700BE552
:10276000D1A2E4501D1243C38018E5D1A2E3500664
:1027700075D1F7124399E5D1A2E4500675D1EF1255
:10278000439FEEA2E092AF7F010225C685198385A3
:102790001882E0A3FEE0A3F5207808E0A3F608DFA6
:1027A000FAE0A3FFE0A3C0E0E0A3C0E0E0A3C0E044
:1027B000E0A3C0E010AF08858218858319800885E2
:1027C0008218858319D2AFD083D08222C0E0C3E4BF
:1027D0009396087401939618400FE4936670080866
:1027E000740193661870007019A3A3C3E49396084C
:1027F0007401939618A3A3400DD0E0D0E0D0E0027E
:1028000026ADA3A3A3A3A3A3D0E022D083D082C5E7
:10281000F0E493A3C5F0C395F0F5F0E493A3C3955A
:10282000F04005E5F0048001E475F002A42582F58E
:1028300082E5F03583F583E493A3C0E0E493C0E040
:10284000227404800474028000CCC0E0EDC0E0E596
:1028500018C39CCCAD1950011D10AF068C188D19F2
:1028600080068C188D19D2AF122962D0E0FDD0E01D
:10287000FC2274028000CCC0E0EDC0E0E518C39CEF
:10288000CCAD1950011D10AF068C188D1980068C27
:10289000188D19D2AF122940D0E0FDD0E0FC22C043
:1028A000E0C0F088F0E4936670080874019366183D
:1028B0007000A8F0A3A3700BD0F0D0E0D0E0D0E07F
:1028C0000226ADA3A3D0F0D0E022D083D082CCC02A
:1028D000E0E493A360061229A21470FAE493A360C3
:1028E00006122AB21470FAD0E0FCE493A3C0E0E42C
:1028F00093C0E022C0E074F2122567758900C2C55A
:102900009013DBE0700E7A007B1090071DE0F91247
:102910003C9180031248A37F010225C6C0E0C0D0CD
:10292000E8C0E0E9C0E0E5A8D2AFC2C7751A00A2CE
:10293000E7A2E792AFD0E0F9D0E0F8D0D0D0E03213
:10294000CAC0E0E493A3C582CCC582C583CDC5834C
:10295000F0A3C582CCC582C583CDC583DAE5D0E0BE
:10296000CA22CAC0E0E0A3C582CCC582C583CDC55A
:1029700083F0A3C582CCC582C583CDC583DAE6D0FA
:10298000E0CA22C008C3E096F50808A3E096420812
:1029900008A3E096420808A3E09645087001D3D04A
:1029A0000822C0E0E493A3D39C5010E493A3C39CFB
:1029B000400AD0E0D0E0D0E00228E7A3A3A3D0E013
:1029C000227009080808226016181818C6C333C6F2
:1029D00008C633C608C633C608C633C6D5E0EA22E1
:1029E000C09FF59FE473D09F22D083D082C09FE424
:1029F00093C0E0740193C0E0740293F59F22251800
:102A0000F58210AF08F518400C15198008F518402C
:102A1000021519D2AF851983227404800A740380C9
:102A200006740280027401C0E0F4041229FED0E0B2
:102A3000122C7F2200C0D0251810AF08F518500CBA
:102A400005198008F51850020519D2AFD0D022BB65
:102A50000102E722C082C08389828A83BB0003E02F
:102A60008002E493D083D082226016080808C6C38F
:102A700013C618C613C618C613C618C613C6D5E0A3
:102A8000EA22C3E0C696F608A3E0C696F608A3E0DD
:102A9000C696F608A3E0C696F6222518F8E435197E
:102AA000F9222518FAE43519FB222518FCE435191A
:102AB000FD22C0E0E493A36C7009D0E0D0E0D0E048
:102AC0000228E7A3A3D0E022251810AF08F518408C
:102AD0000C15198008F51840021519D2AF22E066CE
:102AE000701008A3E066700A08A3E066700408A3EB
:102AF000E06622C3E09608A3E09608A3E09608A348
:102B0000E096A2D265D03322E76670100809E76626
:102B1000700A0809E76670040809E76622C3E096B0
:102B2000F008A3E096F008A3E096F008A3E096F082
:102B300022C3E697F60809E697F60809E697F6082D
:102B400009E697F622C3E4939608740193960874F5
:102B5000029396087403939622E647F60809E6471F
:102B6000F60809E647F60809E647F622E056F008B7
:102B7000A3E056F008A3E056F008A3E056F022E0E8
:102B800026F008A3E036F008A3E036F008A3E0360C
:102B9000F022E627F60809E637F60809E637F608D0
:102BA00009E637F622E657F60809E657F60809E679
:102BB00057F60809E657F622E056F608A3E056F65F
:102BC00008A3E056F608A3E056F622E026F608A38E
:102BD000E036F608A3E036F608A3E036F6227004E5
:102BE00022600D18C6C333C608C633C6D5E0F41834
:102BF00022E4C396F608E496F608E496F608E4960E
:102C0000F622C6F4C608C6F4C608C6F4C608C6F45A
:102C1000C622600D08C6A2E713C618C613C6D5E0C3
:102C2000F322C3E7960809E7960809E7960809E73B
:102C30009622C3E09608A3E09608A3E09608A3E0D6
:102C4000962275D00075813F7518D1751904000260
:102C50002499600C08C6C313C618C613C6D5E0F481
:102C600022E6F008A3E6F008A3E6F008A3E6F022C7
:102C7000E0F608A3E0F608A3E0F608A3E0F622CA0F
:102C8000C0E0E6F0A308DAFAD0E0FA22EAF0A3EB1B
:102C9000F0A3ECF0A3EDF022E0FAA3E0FBA3E0FC4C
:102CA000A3E0FD22E0F8A3E0F9A3E0FAA3E0FB2211
:102CB000E8F0A3E9F0A3EAF0A3EBF022E5C754F8AB
:102CC0004401F5C77901222518F582E43519F58309
:102CD000221229E9DDA8031229E907A9031229E92B
:102CE00080A9031229E9D9A9031229E93AAA0312F2
:102CF00029E979AC031229E94DAE031229E92CAF79
:102D0000031229E965B0031229E918B3031229E96E
:102D10002BB6031229E93AB6031229E9C6B6031203
:102D200029E97CB7031229E9C3B7031229E90CB8D2
:102D3000031229E948B8031229E9BEB8031229E9A8
:102D40002AB9031229E946B9031229E977B903120E
:102D500029E9B6B9031229E9B7BA031229E966BB12
:102D6000031229E9F7BD031229E950BF031229E92B
:102D7000E3BF031229E96DC0031229E9D3C003128E
:102D800029E912C1031229E988C1031229E9DDC228
:102D9000031229E980C3031229E998C3031229E920
:102DA0003BC4031229E9C5C6031229E966C8031208
:102DB00029E984C8031229E90080021229E95A800E
:102DC000021229E9C480021229E94D81021229E97F
:102DD0000982021229E95182021229E98C82021227
:102DE00029E9E282021229E94A83021229E9CE8303
:102DF000021229E9E783021229E90C84021229E967
:102E00004A84021229E99984021229E9C284021231
:102E100029E91185021229E9BD85021229E9858671
:102E2000021229E9EA86021229E9B787021229E982
:102E3000FD87021229E91988021229E94B8802123A
:102E400029E9F389021229E9CA8A021229E9F68AD4
:102E5000021229E92C8B021229E94D8B021229E971
:102E60005C8B021229E9678B021229E91B8C021282
:102E700029E98E8C021229E9008D021229E9088DB8
:102E8000021229E9838D021229E9DC8D021229E957
:102E90001F8E021229E9B190021229E9F79102125C
:102EA00029E98794021229E96F95021229E9A2956E
:102EB000021229E96496021229E91397021229E9FC
:102EC0005B97021229E9BD97021229E9E2970212E3
:102ED00029E9F397021229E96B98021229E9F3987C
:102EE000021229E95799021229E93C9A021229E9AA
:102EF000619A021229E9829B021229E9A09B02121F
:102F000029E9B39B021229E9269C021229E9359C82
:102F1000021229E9BD9C021229E9059D021229E944
:102F2000129D021229E91B9D021229E91B9F021220
:102F300029E96FA0021229E97FA0021229E99BA1C9
:102F4000021229E914A2021229E94AA3021229E96C
:102F50008CA3021229E9C8A3021229E99CA5021236
:102F600029E901A8021229E915A8021229E91FA8D6
:102F7000021229E929A8021229E933A8021229E933
:102F80003DA8021229E956A8021229E960A80212F6
:102F900029E96AA8021229E974A8021229E9A3A85A
:102FA000021229E9CBA8021229E9D6A8021229E9BE
:102FB00020A9021229E92AA9021229E935A9021237
:102FC00029E959A9021229E97DA9021229E9DEA9F4
:102FD000021229E929AA021229E945AA021229E9BD
:102FE000AFAA021229E9FBAA021229E943AB021295
:102FF00029E9BEAB021229E958AC021229E91CAE3C
:10300000021229E98AAE021229E9BCAF021229E9AB
:10301000E2AF021229E952B1021229E906B5021201
:1030200029E906B7021229E9DEB8021229E977B9BF
:10303000021229E989BB021229E94BBC021229E9D3
:1030400097BC021229E9FDBC021229E90FBD021248
:1030500029E95FBF021229E94EC0021229E98DC198
:10306000021229E9DFC1021229E984C2021229E908
:103070003FC4021229E970C5021229E98EC5021265
:1030800029E9E3C5021229E9E1C6021229E909C7C3
:10309000021229E96CC7021229E96DC8021229E956
:1030A000E0C8021229E90ECA021229E979CA0212FD
:1030B00029E969CB021229E9CFCD021229E9FDCD18
:1030C000021229E9F8CE021229E996D0021229E962
:1030D000E6D0021229E99ED1021229E953D2021246
:1030E00029E9B7D2021229E970D3021229E910D4D2
:1030F000021229E974D4021229E9BED4021229E984
:10310000FBD4021229E963D6021229E915810112C2
:1031100029E95781011229E95284011229E9A5847C
:10312000011229E9EB84011229E92C86011229E90F
:103130009186011229E9D186011229E91488011228
:1031400029E9568B011229E97F8C011229E9C097E0
:10315000011229E96098011229E9539B011229E91A
:103160008A9C011229E9009D011229E92A9E011277
:1031700029E97A9F011229E961A0011229E9CAA26D
:10318000011229E9D8A4011229E969A5011229E946
:103190003DA6011229E9C9A6011229E9D3A6011207
:1031A00029E9FBA6011229E9A8A7011229E993A898
:1031B000011229E966A9011229E9F3A9011229E9F5
:1031C00009AA011229E96DAA011229E996AA011298
:1031D00029E9C3AA011229E908AD011229E9E3ADE1
:1031E000011229E927AE011229E998AE011229E955
:1031F00051AF011229E983AF011229E9CAAF0112C7
:1032000029E9FDAF011229E962B0011229E9B1B043
:10321000011229E9B6B0011229E90AB1011229E91E
:1032200054B1011229E950B2011229E9B5B20112D3
:1032300029E913B3011229E95DB6011229E931B771
:10324000011229E9BEB8011229E998BB011229E946
:103250004BBC011229E972BE011229E917BF011204
:1032600029E955BF011229E925C1011229E938C10F
:10327000011229E941C1011229E94AC1011229E9D2
:103280005FC1011229E97EC1011229E9B3C301120C
:1032900029E906C4011229E910C4011229E91AC456
:1032A000011229E975C4011229E9D1C4011229E9E1
:1032B000E9C5011229E94AC6011229E999C7011293
:1032C00029E9E2C7011229E9BAC8011229E9E5C9C9
:1032D000011229E99BCA011229E99DCB011229E9B2
:1032E0009FCC011229E984CD011229E99BCD01125D
:1032F00029E9D8CD011229E9E2CD011229E9ECCD65
:10330000011229E9F7CD011229E915CE011229E9A7
:1033100057CE011229E9B5CE011229E9DACE011200
:1033200029E9F4CE011229E981CF011229E9BACFA6
:10333000011229E90AD1011229E961D1011229E911
:103340007BD2011229E9B1D2011229E94DD3011230
:1033500029E9C9D3011229E939D5011229E954D63D
:10336000011229E91AD7011229E9C4D7011229E962
:1033700049D8011229E9B1D8011229E966D9011207
:1033800029E9B8D9011229E92DDA011229E9F6DA79
:10339000011229E919DB011229E9DDDB011229E912
:1033A00001DC011229E923DC011229E984DC011284
:1033B00029E9CFDE011229E9AADF011229E954E047
:1033C000011229E995E2011229E9E3E2011229E952
:1033D00026E3011229E97EE3011229E9DCE3011267
:1033E00029E906E4011229E92AE4011229E95BE44A
:1033F000011229E985E4011229E9CCE4011229E945
:103400002AE5011229E986E5011229E987E6011278
:1034100029E9F1E7011229E92FE8011229E958E821
:10342000011229E9E9E8011229E933E9011229E940
:1034300057E9011229E9ADE9011229E9C8E90112A8
:1034400029E983EA011229E9ADEA011229E9F0EA42
:10345000011229E946EB011229E94BEE011229E993
:103460007EEE011229E93BEF011229E916F0011263
:1034700029E9A6F0011229E9E7F0011229E964A778
:10348000051229E99CA7051229E9BDA7051229E91A
:10349000FFA7051229E963A8051229E96DA80512FD
:1034A00029E97DA8051229E9B4A8051229E95DAC2E
:1034B000051229E925AE051229E919B0051229E9F5
:1034C000B7B0051229E93EB1051229E94D80041271
:1034D00029E9F680041229E9D581041229E9F0824C
:1034E000041229E91083041229E93284041229E91B
:1034F000CF85041229E93C86041229E912870412B7
:1035000029E91888041229E97D88041229E9B98873
:10351000041229E91289041229E94B89041229E9C4
:103520009489041229E9268A041229E9C38A04121B
:1035300029E9988B041229E9658C041229E9F28C97
:10354000041229E9188D041229E9458D041229E98C
:10355000768D041229E94B8E041229E95B8E041240
:1035600029E9AE8E041229E9BB8E041229E9C88E1E
:10357000041229E9D18E041229E9358F041229E9B0
:10358000938F041229E9DE8F041229E9F98F0412BE
:1035900029E92090041229E93D90041229E9499073
:1035A000041229E9ED91041229E90692041229E98D
:1035B0008292041229E99592041229E9A592041233
:1035C00029E94B93041229E9BB94041229E9CE9509
:1035D000041229E96E96041229E97896041229E961
:1035E000E696041229E9F796041229E9369704129F
:1035F00029E96497041229E93198041229E9889885
:10360000041229E9CD98041229E92399041229E921
:103610004199041229E98F99041229E95D9A04124B
:1036200029E9AB9A041229E9ED9A041229E9709B61
:10363000041229E99A9B041229E9D09B041229E972
:10364000DF9B041229E93D9C041229E9B59C041270
:1036500029E9F69C041229E9459D041229E9709D87
:10366000041229E98A9D041229E9A49D041229E97A
:10367000799E041229E9839E041229E9BE9E041250
:1036800029E9CE9E041229E9D79E041229E9289F30
:10369000041229E93C9F041229E95AA0041229E9DD
:1036A0006DA0041229E984A0041229E999A004124A
:1036B00029E933A1041229E9B2A1041229E955A28A
:1036C000041229E960A2041229E9ADA3041229E930
:1036D000C9A3041229E921A4041229E98FA4041220
:1036E00029E9DBA4041229E9F5A4041229E955A566
:1036F000041229E9F3A5041229E93EA6041229E9D6
:10370000A1A8041229E939A9041229E9B0A90412CF
:1037100029E9F6AB041229E90EAC041229E911AC2F
:10372000041229E91DAC041229E931AC041229E97B
:1037300039AC041229E970AC041229E964AD041211
:1037400029E9EEAD041229E970AE041229E9E5AECB
:10375000041229E9BDAF041229E9DFAF041229E9F7
:1037600076B0041229E982B0041229E9DFB004120C
:1037700029E9E2B0041229E90FB1041229E924B1C0
:10378000041229E993B1041229E9DFB2041229E9EC
:10379000F2B3041229E97DB4041229E990B50412A8
:1037A00029E95AB6041229E98BB6041229E9B1B6FF
:1037B000041229E9BAB6041229E9E9B6041229E982
:1037C00099B7041229E949B8041229E9BCB80412CE
:1037D00029E96EB9041229E9E1B9041229E920BAEC
:1037E000041229E969BA041229E99EBA041229E9E6
:1037F000559A051229E9C09A051229E9079B051275
:1038000029E97D9B051229E9CD9B051229E9519CE7
:10381000051229E9959E051229E9C0A0051229E99A
:103820009DA4051229E91AA5051229E955A5051235
:1038300029E973A5051229E9D3A5051229E9FBA5F4
:10384000051229E92BA6051229E95CA6051229E92A
:1038500089A6051229E9E2A6051229E92DA7051274
:1038600029E90080051229E97C80051229E9A28056
:10387000051229E9D980051229E93282051229E9C0
:103880004E82051229E99382051229E92383051244
:1038900029E97B83051229E95084051229E92E853F
:1038A000051229E97885051229E9D985051229E942
:1038B0005D86051229E98686051229E9C786051263
:1038C00029E97588051229E94589051229E90C8A33
:1038D000051229E9DF8A051229E9198B051229E960
:1038E000718B051229E9938B051229E9278C0512A2
:1038F00029E9DA8C051229E91CEE051229E981EE85
:10390000051229E928EF051229E960EF051229E9D6
:10391000A8F1011229E953F2011229E9F0F3011289
:1039200029E96CF4011229E9A4F4011229E98FF7BD
:10393000011229E921F9011229E98BF9011229E97A
:10394000C3FC011229E964FE011229E90C94061254
:1039500029E93494061229E92095061229E97AC644
:10396000051229E9FDC6051229E914C7051229E93E
:1039700087C7051229E9EDC7051229E916C80512FE
:1039800029E99BC8051229E93DC9051229E9A0C901
:10399000051229E905CA051229E925CA051229E9EE
:1039A00055CA051229E971CA051229E9A0CA0512EA
:1039B00029E9D0CA051229E906CB051229E966CB07
:1039C000051229E92E8D051229E9FE8D051229E936
:1039D000238E051229E9438E051229E9578E051217
:1039E00029E9BF8E051229E9E38E051229E96190C4
:1039F000051229E98791051229E96892051229E93A
:103A0000CC92051229E9F892051229E97C93051256
:103A100029E9CD93051229E9EE93051229E9669467
:103A2000051229E90A96051229E96D96051229E978
:103A3000FD97051229E9CA98051229E90599051289
:103A400029E92A99051229E94A99051229E9709963
:103A5000051229E98499051229E9ED99051229E948
:103A6000419A051229E99488061229E99E880612CE
:103A700029E9BF88061229E938E9041229E946EC48
:103A8000041229E973ED041229E94EEF041229E921
:103A9000D8EF041229E991F0041229E9BAF00412CE
:103AA00029E904F1041229E9BFF1041229E932F2EB
:103AB000041229E935F2041229E938F2041229E93D
:103AC00081A4031229E95BF2041229E95EF20412CF
:103AD00029E977F2041229E9DBF2041229E9CDF38E
:103AE000041229E902F5041229E94FF5041229E923
:103AF00056F6041229E928F7041229E9D6D602124B
:103B000029E90ED7021229E9CCDB021229E99EDC51
:103B1000021229E925DD021229E956DD021229E9FE
:103B200084DD021229E99FA8031229E906DE0212A8
:103B300029E927DF021229E955DF021229E983DF8B
:103B4000021229E9B9DF021229E966E0021229E925
:103B50008CE0021229E9EBE0021229E961E202128B
:103B600029E9FBE2021229E9ECE3021229E9C9E49E
:103B7000021229E913E5021229E962E5021229E994
:103B8000CEE5021229E936E6021229E983E602129D
:103B900029E9F3E6021229E904E8021229E9F8E822
:103BA000021229E9A9E9021229E9DEE9021229E94A
:103BB00033EA021229E9D5EA021229E903EB0212DB
:103BC00029E988EC021229E90DED021229E94DEDEF
:103BD000021229E98CED021229E9A5ED021229E968
:103BE00054EE021229E91EEF021229E9C5EF021272
:103BF00029E959F0021229E9FFF0021229E969F1D5
:103C0000021229E9F4F1021229E987F2021229E9E4
:103C1000A5F2021229E978F3021229E936F4021218
:103C200029E9ECF4021229E98AF5021229E967BAB6
:103C3000051229E9A8BA051229E911BB051229E9DB
:103C400032BB051229E94BBB051229E905BC051257
:103C500029E90EBC051229E95FBC051229E988BCD7
:103C6000051229E99FBC051229E903BD051229E9BE
:103C700095BD051229E9C6BD051229E922BE051226
:103C800029E988BE051229E9BCBE051229E92FBF22
:103C9000051229E971BF051229E9B1BF051229E909
:103CA000E9BF051229E9FBBF051229E90DC005127C
:103CB00029E93EC0051229E97EC0051229E9A7C0FD
:103CC000051229E9C8D6051229E90BD8051229E9F8
:103CD00031D8051229E942D8051229E95ADA051224
:103CE00029E979DA051229E9E18A061229E9178B0F
:103CF000061229E9628B061229E9AE8C061229E91F
:103D00000CD5041229E94AD6041229E986D60412F0
:103D100029E94BD8041229E975D8041229E9FBDAFC
:103D2000041229E93BDB041229E9D0DC041229E959
:103D300065DD041229E9C3DD041229E954DE041209
:103D400029E98CDE041229E9CEDE041229E948E0D3
:103D5000041229E9D1E1041229E907E4041229E94E
:103D600035E4041229E961E4041229E96AE4041241
:103D700029E9C0E4041229E950E5041229E957E8C9
:103D8000041229E9DBE8041229E9499E061229E90F
:103D90005F9E061229E9699E061229E9B99E06125C
:103DA00029E9A0E5051229E9B9E5051229E95EE648
:103DB000051229E99EE6051229E9B7E6051229E967
:103DC000EBE6051229E938E7051229E96CE7051247
:103DD00029E9AEE7051229E984E9051229E9EFE9A5
:103DE000051229E98996061229E9DE96061229E9C3
:103DF0003797061229E9FA9C061229E94D9D061209
:103E000029E98F9D061229E99F9D061229E9BDC85F
:103E1000031229E915C9031229E9B5C9031229E9D1
:103E2000CDCA031229E9B9CB031229E986CC0312C2
:103E300029E99BCC031229E9E5CC031229E93CCD01
:103E4000031229E9A8CD031229E9BBCD031229E900
:103E500013CE031229E982CE031229E91DD10312E0
:103E600029E919D2031229E974D2031229E9BAD235
:103E7000031229E9D8D4031229E928D5031229E924
:103E8000A9D5031229E97BD6031229E9B4D6031276
:103E900029E9D3D6031229E91ED7031229E934D719
:103EA000031229E941D7031229E97AD7031229E934
:103EB0008CD7031229E962D8031229E96DD80312BD
:103EC00029E9F2D8031229E94AD9031229E996D936
:103ED000031229E9CDDA031229E9F5DA031229E9F7
:103EE00071DD031229E999DD031229E9ABDE031222
:103EF00029E9DADE031229E952DF031229E914E085
:103F0000031229E948E0031229E9B8E0031229E97C
:103F100095E1031229E9CEE1031229E9D8E1031260
:103F200029E9DBE1031229E9E5E1031229E901E2CC
:103F3000031229E97DE2031229E9B6E2031229E915
:103F4000D2E2031229E9FEE2031229E939E303125E
:103F500029E954E3031229E95EE3031229E98DE319
:103F6000031229E9A3E3031229E9BFE3031229E9B4
:103F7000EEE3031229E90EE4031229E957E40312E0
:103F800029E9A0E4031229E9AAE5031229E9C29963
:103F9000061229E9D399061229E95C9A061229E941
:103FA0009178001229E9E078001229E99E7A00123E
:103FB00029E9717C001229E9AF7C001229E9857D8D
:103FC000001229E98A7E001229E9AC7E001229E953
:103FD000087F001229E9897F001229E9F64F0012B3
:103FE00029E91850001229E96A51001229E9B35150
:103FF000001229E92C52001229E9A752001229E9DE
:104000001053001229E95753001229E9C553001231
:1040100029E96A54001229E9F054001229E92C55C3
:10402000001229E98059001229E98E5B001229E962
:10403000C15B001229E9005C001229E90D5D001244
:1040400029E9F65F001229E9A060001229E94B6214
:10405000001229E97E63001229E99464001229E91B
:104060000965001229E9D565001229E96C6600127C
:1040700029E97C66001229E93367001229E9696899
:10408000001229E9AD6A001229E9506D001229E9F0
:104090002E6E001229E96B6F001229E9B07200122E
:1040A00029E9C072001229E9F773001229E9AA74FC
:1040B000001229E9DB75001229E94976001229E985
:1040C0008077001229E9D577001229E906BB04128E
:1040D00029E9ADBB041229E91FBC041229E92FBC50
:1040E000041229E9B1BC041229E908BD041229E926
:1040F000FDBD041229E924BE041229E9C9BE041237
:1041000029E918BF041229E976BF041229E9D1BFB1
:10411000041229E9ACC2041229E965C3041229E991
:10412000CAC3041229E95DC5041229E9FDC50412B8
:1041300029E996C6041229E9F3C6041229E969C7D8
:10414000041229E965C8041229E958C9041229E9A9
:10415000B1C9041229E9C7C9041229E9E8C904123E
:1041600029E927CA041229E9B7CA041229E9FACBB6
:10417000041229E9B7CD041229E901CF041229E973
:104180003BD0041229E946D1041229E9E6D10412F0
:1041900029E955D2041229E972D3041229E9F5E676
:1041A000031229E960E7031229E9A8E7031229E9C4
:1041B0000FE8031229E96BE8031229E9A6E80312C4
:1041C00029E942E9031229E99CE9031229E908EBEC
:1041D000031229E981EB031229E9B8EC031229E95A
:1041E000E0EC031229E9BEED031229E9CFED031239
:1041F00029E9E5ED031229E9D7EE031229E9FAEEE0
:10420000031229E9C2EF031229E9EAEF031229E9AF
:1042100001F0031229E91BF0031229E947F0031208
:1042200029E967F0031229E98DF0031229E9A4F0C6
:10423000031229E979F1031229E9D3F1031229E9DB
:10424000ABF2031229E927F3031229E93EF3031223
:1042500029E9B8F3031229E900F4031229E926F445
:10426000031229E983F5031229E988F5031229E9E4
:10427000C5F5031229E93CF6031229E9A8F6031251
:1042800029E9A3F7031229E97DF8031229E9C9F8FE
:10429000031229E9E1F9031229E9DBFA031229E9FA
:1042A0007DFB031229E9C6FB031229E9DBFB03129C
:1042B00029E9EDFC031229E98EFD031229E9ECFD41
:1042C000031229E9A2D1051229E9DFD1051229E952
:1042D00078D2051229E983D3051229E9CBD5051235
:1042E00029E947D6051229E97AF9051229E9A8FA38
:1042F000051229E970FB051229E9C5FB051229E918
:1043000048FC051229E99A8F061229E9B59A061286
:1043100029E9C69A061229E9669B061229E9D2FF05
:10432000021229E9E57F001229E9809B061229E99A
:10433000909B061229E9A59B061229E9369C0612D4
:1043400029E9BE98061229E94399061229E9A99993
:10435000061229E9F9FF011229E9E0FF011229E912
:10436000F0FF011229E9F3FF011229E9F6FF01121A
:1043700029E9F87F001229E9118D061229E9338D08
:10438000061229E9A18E061229E9258F061229E9CC
:10439000B7FF011229E9C0FF011229E9C9FF011283
:1043A00029E9D7FF011229E9D1C0051229E93DC148
:1043B000051229E905C2051229E9FEC2051229E9FB
:1043C000EBC4051229E945C5051229E998C505126E
:1043D00029E9A9C5051229E9BBC5051229E927C69E
:1043E000051229E93BC6051229E946C6051229E945
:1043F00054C6051229E966C6051229E91ACC051228
:1044000029E946CC051229E9EDCE051229E942CF6A
:10441000051229E97ECF051229E992CF051229E973
:10442000ABCF051229E99ED0051229E97AD10512F0
:1044300029E98ED1051229E99792061229E9BB9242
:10444000061229E9D492061229E91393061229E9E2
:104450004693061229E97693061229E980930612FB
:1044600029E9E893061229E9EB93061229E9F59365
:10447000061229E90294061229E9E685061229E9BD
:104480000E86061229E94F86061229E96D86061264
:1044900029E98886061229E9F086061229E9FC86B0
:1044A000061229E95B87061229E97F87061229E9A6
:1044B0004088061229E94D88061229E95E8806120D
:1044C00029E9E79E061229E9FF9E061229E9259FA0
:1044D000061229E911DC051229E95ADD051229E93C
:1044E00060DD051229E977DD051229E998DD05125D
:1044F00029E9AEDD051229E9C2DD051229E941DE0F
:10450000051229E9A6DE051229E92EDF051229E99F
:10451000A7DF051229E980E0051229E990E00512DC
:1045200029E99FE0051229E9B09D061229E9D49DE9
:10453000061229E9FC9D061229E9249E061229E9A2
:104540002783061229E99383061229E9B28306120A
:1045500029E91884061229E9DAFC051229E9F3FC95
:10456000051229E90AFD051229E913FD051229E9B9
:1045700031FD051229E93BFD051229E945FD05122A
:1045800029E958FD051229E9E5FD051229E954FE3E
:10459000051229E982FE051229E9D3FE051229E94F
:1045A0001FFF051229E93AFF051229E944FF051208
:1045B00029E955FF051229E998FF051229E96E9F9F
:1045C000061229E9B99F061229E94FF6021229E9D4
:1045D0007BF6021229E999F6021229E9ACF60212D9
:1045E00029E9C7F6021229E926F7021229E954F748
:1045F000021229E960FB021229E9A2FC021229E950
:10460000D4FC021229E93FFD021229E9C3FE02127D
:1046100029E9EBFE021229E900FF021229E910FF45
:10462000021229E950FF021229E992FF021229E938
:10463000A2FF021229E95195061229E96195061295
:1046400029E97F95061229E99A95061229E9C1956B
:10465000061229E9E295061229E9FC95061229E9D4
:104660003496061229E95796061229E9469C061245
:1046700029E98C9C061229E9E2F5051229E9F2F5EF
:10468000051229E910F7051229E942F7051229E96F
:1046900064F7051229E98CF7051229E9A5F7051237
:1046A00029E9E1F7051229E94AF8051229E986F80E
:1046B000051229E9CDF8051229E9FAF8051229E9C8
:1046C00026F9051229E90891061229E93F910612F7
:1046D00029E96792061229E96A92061229E9AB973D
:1046E000061229E91D98061229E95B98061229E9A4
:1046F0009C98061229E9D6F7041229E9DCF704127E
:1047000029E923F8041229E92FFA041229E95FFAAA
:10471000041229E9C9FA041229E984FB041229E9DF
:10472000CBFB041229E9FEFB041229E988FC0412E0
:1047300029E99FFC041229E9ACFC041229E9B6FC22
:10474000041229E956FE041229E948FF041229E956
:10475000A6FF041229E9EAB1051229E900B20512FF
:1047600029E9B2B2051229E9DCB3051229E9D1B46D
:10477000051229E968B5051229E9A3B5051229E949
:1047800015B6051229E973B6051229E983B6051293
:1047900029E9AAB6051229E9FCB6051229E96BB880
:1047A000051229E970B8051229E992B8051229E91C
:1047B000FCE9051229E91AEA051229E95EEA05125F
:1047C00029E984EA051229E9A6EA051229E9BEEADF
:1047D000051229E9D6EA051229E9EEEA051229E9C6
:1047E00094EB051229E9D6EB051229E9E0EB051255
:1047F00029E9F5EB051229E9FCEC051229E917ED89
:10480000051229E920ED051229E929ED051229E90A
:1048100032ED051229E93CED051229E9B9ED051241
:1048200029E9D0E0051229E915E5051229E931E564
:10483000051229E936E5051229E91AF2051229E9D6
:1048400030F2051229E9CEF3051229E919F405120F
:1048500029E983F4051229E982F5051229E9B1F560
:10486000051229E9C3F5051229E98DFE031229E98C
:104870000080061229E95C80061229E99C80061254
:1048800029E99E81061229E9B681061229E9CB8120
:10489000061229E9F781061229E92E82061229E972
:1048A0003E82061229E95482061229E9798206120B
:1048B00029E90483061229E9B97F001229E9EDA349
:1048C000031229E907A3031229E97FA2031229E9A8
:1048D000CCA1031229E97B9F031229E9509F0312FF
:1048E00029E9F19E031229E9629D031229E9F09C4E
:1048F000031229E9D79C031229E99A9C031229E99A
:104900008C9C031229E9219C031229E9E69B0312DE
:1049100029E9579B031229E9099A031229E98F997A
:10492000031229E9CC98031229E9C297031229E955
:104930007997031229E95397031229E98F960312F5
:1049400029E9D994031229E97994031229E94AA89B
:10495000031229E992A7031229E9D6A6031229E92D
:104960003DA5031229E90DA5031229E9D1A40312DB
:1049700029E9BDA4031229E94A94031229E94794BD
:10498000031229E93294031229E9EF93031229E96A
:10499000A9A4031229E9D693031229E9DE9203128E
:1049A00029E99D92031229E96A92031229E9D8DDC7
:1049B000021229E9FE91031229E995A4031229E9BB
:1049C000CB91031229E97091031229E93F91031257
:1049D00029E9088E031229E91A8D031229E9D48BDB
:1049E000031229E9808B031229E9748B031229E948
:1049F000DB8A031229E9A989031229E9FA8603123D
:104A000029E99D84031229E95184031229E9368397
:104A1000031229E9CB82031229E9F381031229E960
:104A2000AF81031229E90080031229E96B80031288
:104A300029E93280031229E93BF20400000080FBDF
:104A40008F000100130987000100120924000200F1
:104A50003C15250002003E152600020040152700E7
:104A600002004215280001004415290001004515E7
:104A7000840004004615860001004A152A00010042
:104A80004B152B0001004C152C00010050152D007A
:104A90000800FA082E00010051152F0001005215E0
:104AA000300001005315310001005415320001009F
:104AB00002093300010003093400010055153600D6
:104AC00001000409380001005615390001004F1596
:104AD000830002006815630001000F0964000100F3
:104AE0004D15650001004E156D00010010097100A3
:104AF0000800F20866000100671543000100581520
:104B0000440002005915450001005B1546000200F3
:104B10005C15470008000709480001005E154B00BE
:104B200001005F15040001006A15A10001006C1569
:104B3000370001006B158800010014093C000100DA
:104B400005093D0001005715490002006015670086
:104B5000010011094D00020062154E0001006415AC
:104B60004F00020065153E0001000609000000002C
:104B700000000001363601010001020100010301BD
:104B800000010401060605020000070100340801C7
:104B9000000F090401010D0100FF0E0800001702BB
:104BA0000000190100FF1A0100011B0100FE1C0199
:104BB00000081D0200001F01000120010001210268
:104BC00000002301000F240200002601000127013C
:104BD0000008280200FF2A0100072B0102402C01D7
:104BE00000002D0100012E0100012F0100FF300106
:104BF0000B1C310800003A0100083B01000F3C018A
:104C000000013D0100FF3E04000042040000460494
:104C100000004A0400004E04000052040000560444
:104C200000005A0400005E20FFFF3600010006006D
:104C300000000F0000000000000000000000000065
:104C400003FFFF00000403FFFF0000FFFF0FF4015C
:104C50000005C4040320000100000B000000000058
:104C600000000003010F0000000000000000000031
:104C70000000000000000000000000000000000034
:104C80000000000000000000000000000000000024
:104C90000000000000000000000000000000000014
:104CA0000000000000000000010371030103010384
:104CB00001030103010322030203010310030003A4
:104CC000000300030003000300030003420300038A
:104CD0002403060300030003040312032503230334
:104CE0002503230304030403000300030003440318
:104CF0000003000323030003650321003503810340
:104D0000000305030003000300030003250323033E
:104D100003007100300160001100700031022003B7
:104D20005004800010006100000014006300730054
:104D30007200620043000000130006000000000043
:104D40000400120000000000000000000400040045
:104D5000370037003C024400000000000000000063
:104D600065000000350081000000050000008300A0
:104D70000000010171010101010111010101310175
:104D8000010101018001100161013B001400630178
:104D900073017201620143010001130106013D012B
:104DA00035000401120100010001000100010401AD
:104DB0000401330133013C0144013201360000019A
:104DC000000165010001350081010001050182013A
:104DD00083010001030271023001600211027002BE
:104DE0000102020202028002100261023A00410046
:104DF000630273027202620243020002130238006D
:104E0000000200020402120200020002000200027C
:104E100004020402370037003C0244020002390059
:104E20000002000265020002350281020002050252
:104E3000820283020002030471040204600411046C
:104E4000700402040204010402041004610400045A
:104E5000140463047304720462044304000413041E
:104E60000604000400040404120400040004000406
:104E7000000451046400000400040004440400041D
:104E80000004000400046504000435048104640087
:104E9000050400048304000400000B4113007B4060
:104EA00001000B410200FD3F0300034004000940E4
:104EB00005000F4006001B4030003F4031003940E4
:104EC00032004B40330051403500574034005D40C4
:104ED0003600634011006F401400754015002D40EE
:104EE0001F003340FFFF0000015131068731088168
:104EF000310B9F3110BB300AB1310257310575318A
:104F0000075D310C39310D453164BD2EFF000007BE
:104F1000ECFDFDFDECDCDCCCBCACAC9C9C8C7C7C6E
:104F20006C6C5C5C5C4C4C3C3C2C2C1C1C03EAF513
:104F3000E5D5D5C5B5A59595858575756565555531
:104F400045453535252515150500160F00000B15AF
:104F50000B020002220F3300000E01030507090BAC
:104F60000D0F00020406080A0C0D5A6967426565B8
:104F7000416C6C69616E63653039303017181921E6
:104F8000301B1D1F30303016181920231A1C1E30FC
:104F900000034A49434E181A250502000119161844
:104FA0001616182303000C0E020B040B0A07080048
:104FB0000F00393D3F373C3C362C442D02040201A2
:104FC0000101010902E803000000BE040A7F003C61
:104FD00000000000000E00E8033C0008100C0A0C62
:104FE00003150900040009FF1E1E0305010C05043A
:104FF000040810080328C082C08390081CE4F0A3B2
:10500000F07CD57D047A8D7B071246ED122EC312FB
:105010004A23122EC9026DD174F312242D74F51295
:105020002AC889098A088B0AE9705F7402650870CA
:105030003E9007AC7408F0750C00780C122A25EC31
:10504000F50C780C122A25EBF50C780C122A259019
:10505000154612284190154AE0F97C077D09901504
:1050600068126DE2122EED7407122A3402512A746E
:10507000016508600302512D9007AC7408F07B00B5
:10508000AA0AA90A122F2F02512A74016509600980
:1050900074026509600302512DEA60067403650815
:1050A00070409007AC740212514E122C98122EDBF5
:1050B0009007B4E0A2E34010E9700D900820E004EE
:1050C000F06404700312515874036508705C900812
:1050D00021E0F8740128F0E8C39405404D125158BE
:1050E0008048740165087045740165099007AC70CB
:1050F0002E740AF07401122CC7E4F07402122CC74B
:105100007403F004122CC7E4F0A3F0A3F0A3F0742E
:1051100008122CC7E4F0AA18AB1912316380257469
:105120000A12514E122C98122F11E960179080AC80
:105130001228417A017B009007A9E0F9123DB7746B
:1051400004122A34740B122A347F050226BDF09013
:10515000154AE0F990154622901546E4F0A374F83C
:10516000F0A374FFF0A37407F02274F612242DE963
:10517000FFEAFE7AD1F9123C6D8A828B83E5824583
:1051800083702A7A027B00123C4FEA4B700E7A1031
:105190007B009007A9E0F9123C9180148A828B83EE
:1051A00074D1F0EFA3F0EEF9123C5B8003EFA3F0B3
:1051B0000253C074F712242D890890070612749EBA
:1051C000FF901538E0F47003A3E0F4703690071DEB
:1051D000E0901538F0A3E4F080298E828F83A3A39A
:1051E00012788C60168E828F83A3A3A3E0F5838848
:1051F00082A312788CFAA908123FE58E828F83125F
:1052000077B4FFEE4F70D3901538E0F47003A3E04D
:10521000F4600A901538E0FAA908123FE512326BE3
:105220009007771259311232650275D674F1122443
:105230002D890A8C08750900750B00740F122CC794
:1052400012608A7411122CC71259588049AE0E127E
:1052500052F8F50CA3E0F50DAE0BEE2EFEE433FF95
:10526000EA2EF582EB126643650C7004A3E0650D2F
:105270007019AE09EE2EFEE433FFEC2EF582ED3F01
:10528000F583E50CF0A3E50DF00509050EE50EC369
:10529000950840B9050BE50BC3950A5005750E003E
:1052A00080EBA909026CEE74F412242D890B7D00A9
:1052B000740C122CC712608A80010DEDC3950B503F
:1052C00032750A008002050AE50AC39C50ECED2500
:1052D000E0FEE433FFEA2EF582EB3F125308F509B6
:1052E000AE0A1252F865087004A3E0650970D77918
:1052F0000180027900026A95EE2EFEE433FFE82E6B
:10530000F582E93FF583E022F583E0F508A3E0228A
:1053100074F612242D1253AB7003A3E06D70177551
:1053200008B27509077808122A21EEFA12411174A1
:1053300002122A34801F7508027509807808122A23
:10534000218C088D097808122A2112539E124135AA
:105350007404122A34806974F612242D1253AB702F
:1053600003A3E06D70177508BF7509077808122A46
:1053700021EEFA1241177402122A34801F750803B5
:105380007509807808122A218C088D097808122A5C
:105390002112539E1241357404122A348022125C69
:1053A000F9F583E0FD7C801267172212664C1277B4
:1053B000C6FCE439FD900777E06C227402122A34AF
:1053C0007F020226BD74F612242D74FE122AC8EA4A
:1053D000FEEBFF851882851983E4F0A3125B881227
:1053E0006663E0FCA3E0FBECFA88828983A3A3E078
:1053F000F9750900750800600574FF697005750886
:1054000082803D900777E06A7003A3E06B701AAA70
:1054100018AB1912382FE9F50985188285198312FE
:105420006AA0701C7508838017900912E0600464FC
:105430000170057508818008E064027003750880BA
:10544000851882851983125958A908EEFAEFFB12C4
:10545000411DE5096011851882851983126AA060D3
:1054600006126DDC123CF70253BB74F212242DEAD3
:10547000FEEBFF750A00750B001254DC12326BEA6A
:1054800065087003EB65097012123841E914F50ADA
:1054900079017AE87B071238478003750B80126622
:1054A0003DF50C780C122A25750CE8750D07780C63
:1054B000122A21780A122A257808122A21E50BF5EA
:1054C000087808122A251264FE126640F97A057BD4
:1054D000801241237407122A340262461276FF12A8
:1054E000608E888289831277C5F508E439F5092230
:1054F00074F612242DE9FE7F0080298A828B8312A4
:10550000530AF8E4C8F9E50828E439F509EF25E07D
:10551000F8E433F9EC28F582ED125D02EA2402FA90
:1055200050010B0FEFC39E40D20253C074E8122407
:105530002D74FB122AC88A168B1785188285198349
:10554000E4F07403122CC7E4F0A3F004122CC7E4B7
:10555000F0A3F012607B3517125B5AF50B850A82B7
:10556000F5831277C1FEE439FF850A82850B83A398
:10557000A3E0FA850A82850B83A3A3A3E0F9EAF5E9
:1055800008E439F509E50A2404F50A5002050BEE92
:10559000FAEFFB123307E964016016EEFAEFFB1233
:1055A0003307E9703D900777E06E7003A3E06F600A
:1055B0003112685A122A25E4F508F5097808122AEA
:1055C000217808122A2590077712284575088078D7
:1055D00008122A251259371241237407122A34025D
:1055E000592712595E8810602B1273DB123CF1743C
:1055F00003122CC71259317403122CC7126AA0600F
:10560000137403122CC7125950A9101240158A0A9C
:105610008B0B800375100012595E880F6027127380
:10562000DB123CF17401122CC71259317401122C97
:10563000C7126AA0600F7401122CC7125950A90F2B
:105640001240158003750F00900706805D850A8261
:10565000850B83A3A3A3A3A3A3A3A3E4F0A3F0AA0E
:105660000AAB0B851482851583A3A312596E127899
:105670008CF9123C5B851282851383E0C0E08518AB
:1056800082851983E0F874E828F582E43407F5830D
:10569000D0E0126AA404F0E511A2E05007AA12AB10
:1056A00013123CF7851482851583E0F514A3E0F509
:1056B00015E51445157003025894851482851583E9
:1056C000A3A312788C60DD851482851583A3A3A320
:1056D000A3A3A3A3A3E0A2E050CA851482851583E7
:1056E000A3A3A3A3126AA0851482851583A3A36034
:1056F0001F12788CFA7901851482851583A3A3A3E0
:10570000A3126D1712261E8A128B13751101800FBA
:1057100012596EA3A3E0F512A3E0F513751100E58D
:105720001245137003025697851282851383A3E0F6
:1057300065087004A3E06509600F74FF65087004D4
:1057400074FF65096003025697851282851383A34F
:10575000A3A3A3A3A3A3122845851282851383A321
:10576000A3A3A3A3A3E0FC7405122CC7126DE2A9A6
:1057700010123FF77402122A34E9703C85128285B8
:105780001383A3A3A3A3A3A3A3A3A3A31228458521
:105790001282851383A3A3A3A3A3A3A3A3A3E0FCC3
:1057A0007403122CC7126DE2A90F123FF774021294
:1057B0002A34E97003025697E50F2510C333240AF3
:1057C000FA7B00123C4F8A0A8B0BEA450B700302EE
:1057D00056758A828B8374D2F0851682851783A3CF
:1057E000A312608A8A828B83A3A3E8F0A3E91276CE
:1057F000BCA3E5101277CDE50FF0E510603CEA247C
:1058000005FAE4350BFBE50A240AF8E4350BF98ABE
:10581000828B831260947403122CC7125973122A5C
:105820001DAC10EC2CFCE433FD8A828B83126DE2FC
:10583000123C2B7403122A34800D8A828B83A3A31B
:10584000A3A3A3E4F0A3F0E50F700302564DA81044
:10585000E828F8E433F9E50A28F8E50B39F9E824F3
:105860000AFAE439FB850A82850B83A3A3A3A3A3C9
:10587000A3A3A31259317401122CC7125973122A0F
:105880001DAC0FEC2CFCE433FD123C2B7403122AEC
:105890003402565F851882851983E0602712685AA2
:1058A000122A257508E87509077808122A21740359
:1058B000122CC7126863122A2590077712284575A3
:1058C00008008029EEFAEFFB123307E9702F126807
:1058D0005A122A257508E87509077808122A2175D1
:1058E00008007808122A25900777122845780812B0
:1058F0002A251259371241237407122A34740312CD
:105900002CC7126AA0600B7403122CC7126DE2122E
:105910003CF77401122CC7126AA0600B7401122CA0
:10592000C7126DE2123CF77405122A347F1002266A
:10593000BDEAF0A3EBF022E5162402FCE43517FDE6
:10594000E51612648E3517F583E0F97A067B80221E
:10595000125958AA0AAB0B22E0FCA3E0FD22850AEB
:1059600082850B83E0F8A385820A85830B22126D62
:1059700017A322E0F50CA3E0F50D750E00780C22BC
:1059800074F112242D74F4122AC88A088B09ECFED3
:10599000EDFF740B122CC77403F0122AA21246ED0D
:1059A000123265EAFCEBFD7403122AA21246E7E903
:1059B000600FEE241312664064036010E06401601F
:1059C0000B8518828519837484025B128E828F8303
:1059D000A3A3A3A3A3A3A3A3E06018F46015EE24DC
:1059E0001312664064037016EE24141266406003BE
:1059F000F4700B8518828519837482025B1212750C
:105A00008AE064217002A3E06003025AE9851882EB
:105A1000851983748C125B8864036003025AD37403
:105A200001122AAA12622E12499FE96003025AD378
:105A3000123F798A0A8B0BEA450B7003025B138EC7
:105A40000C8F0D750E00780C122A1D7C157D00122E
:105A50003C2B7403122A34850882850983A3A3E5AD
:105A60000A2415FCE4350BFD74091229621271E950
:105A7000C0E0E50A241EF582E4350BF583D0E01280
:105A8000609AC0E0E50A241FF582E4350BF583D067
:105A9000E0F0E50A2420F582E4350BF5837405F087
:105AA000EE240BFE50010FFAEFFB1238E97D007C6B
:105AB000007900EEFAEFFB1240DB9080AC12284137
:105AC0007A007B109007A9E0F9123DB77404122AFE
:105AD000348078125B50122A25125B621249C3741B
:105AE00001122A34E9702C8014125B50122A2512FC
:105AF0005B621249BD7401122A34E9700D85188267
:105B0000851983E4F0123F4980098518828519833D
:105B10007488F01271E9F50A780A122A25740112C4
:105B20002A9A880A890B780A122A21E508240CF59A
:105B300082E43509125B5A4480F50B780A122A2157
:105B40001265C01240CF7405122A34740C026CEB3B
:105B5000EE12623BE0F50A780A22F583E0F50AA32B
:105B6000E022EE240BFCE43FFD8E828F83A3A3A3EF
:105B7000A3A3A3A3A3A3126E1F8E828F83A3A3A3A9
:105B8000A3A3A3A3A3E0F922F01276FFE022C08230
:105B9000C08374F3122AC8851882851983E4F0043F
:105BA000122CC71259317403122CC7AA82AB83126C
:105BB0002DEBAA18AB19122E21740D122A34026D86
:105BC000D174F612242D126648FAA3E0F9EAF8908F
:105BD00007BAE058F508A3E059F509E5084509605A
:105BE0001C7808122A2190077712284512663DFD7D
:105BF0007C0012671312412F7404122A340253C01E
:105C000074F412242D74FF122AC8EAFEEBFF8518E3
:105C100082851983E4F0900906E06021EE240B12DE
:105C20006640640160178E828F83A3A312608AEEA0
:105C30002415126640687003A3E0696003025CF4F7
:105C40001264EE126088E8FAE9FB88828983A3A3D4
:105C5000A3A3A3A3A3A3E0FC88828983A3A3A3A3F4
:105C6000A3A3A3A3127766EC28F508E439F509ECA1
:105C700045096010EC9471E994085008900912E00D
:105C80006402700A85188285198374808038122E08
:105C90005D8A0A8B0BA80AA90BE8496021888289D2
:105CA00083A3A3A3A3E06016C394035011E82412B6
:105CB000125CFFE82414125CFF123F49800985182A
:105CC000828519837481F0125CF9126861122A25A9
:105CD0007401122A9A880889097808122A217508FD
:105CE0001F7509807808122A211264F41240CF74BB
:105CF00005122A347401026A92EE1275B13F22F540
:105D000082E439F583E508F0A3E509F02274EA128C
:105D1000242D74DB122AC88A148B15751200751392
:105D200000127884F50EAC18AD197A007B00799CCE
:105D3000122F417A047900122E33EAF50C8518826D
:105D4000851983E02AF0F8E50EC3984003025F2C22
:105D5000E0C3950EF509C394044003750903E509F2
:105D600075F01AA4FAABF0123CF18A128B13EA45D3
:105D7000137003025F2F750D00AE12AF13850E086E
:105D8000807E125F97123C37850A82850B83A3A31E
:105D9000A3A3E0702D850A82850B83126AA0700C84
:105DA000126F2CF0EE2418126F2F8010125FA5F0E6
:105DB000900566E014C0E0125F7FD0E0125FD0E48F
:105DC0008034900566E004C0E0125F7FD0E0125F8F
:105DD000C8C39403EE4003025E931262377402124A
:105DE0005FC864017003025EA0EE2415125FA8F084
:105DF000EE2416125FA8F0EE241AFE50010F050DD6
:105E0000E50DC395094003025ECBE508C3950C4040
:105E100003025EA985080AAA0A7B00122EA58A0A37
:105E20008B0B0508900553125FB11246ED850A826F
:105E3000850B8312608A125F8DE8F0A3E9125FE29E
:105E4000850A82850B83A3A3A3A3A3A3A3A3A3A3D0
:105E5000E0C0E0125F75D0E0F07401122CC7E4F0EE
:105E6000850A82850B8312608A7402122CC7126025
:105E7000947401122AA2122E0FE964016003025DDC
:105E8000827404122CC7AC82AD83125F9D1246ED62
:105E9000025D88125FA6125FC864036003025DE9B9
:105EA000EE2415126F2F025DEFE50CC3950E400531
:105EB000750800801DE50EC3950CF5088014125F6F
:105EC000A5F0EE241AFE50010F050DE50DC395094E
:105ED000505D740E122AAA85080AAA0A7B007987E7
:105EE000122F4105087418122CC7125FB11246ED2B
:105EF000125F97123C37EE2412F8E43FF9740E1249
:105F00002CC7126DE288828983EAF0A3EB125FD07E
:105F10007403125FE2741D122CC7E0C0E0125F75BB
:105F2000D0E0126D497097126F2C8095750900753D
:105F30000A00780A122A257812122A217809122AD0
:105F400025E50EF5097809122A257405122CC7E0FB
:105F5000FD7C0012647A12416B7405122A34E5123A
:105F600045136007AA12AB13123CF77425122A34AA
:105F70007F0E0226BDEE2419F582E43FF58322123E
:105F80005F8322EE2418F582E43FF58322EE24128B
:105F9000F582E43FF583227C087D0079FFEE240A38
:105FA000FAE43FFB22EE2414F582E43FF58374010A
:105FB0002212608E8E828F83E8F0A3E9F07C677DE9
:105FC00005EE12672E3FFB22127721A3A3A3E02246
:105FD000F0EE126F237402F0EE2416F582E43FF522
:105FE0008322F0EE2417F582E43FF5837402F01269
:105FF0005F8374FFF02274F612242D74F9122AC8FC
:106000008A088B0912607B350912784E123C43EAEC
:10601000F8EBF9ECFAEDFB851882851983122CB0A8
:10602000EE2404FE50010F8E828F83E0C0E07404E2
:10603000122CC7D0E0126D20FA7405122CC774011F
:10604000F07406122CC77401F0900781F090078A53
:1060500004127738A312608A900782126094EA9043
:10606000078B12609A900780F0AA18AB19122EE1E4
:10607000E96003122EE774070253BDEA1260802222
:1060800012665D2212748739F58312608E22E0F861
:10609000A3E0F922E8F0A3E9F022F0127696E022DC
:1060A00074F212242D74FF122AC87508007E007F36
:1060B000001231938A0A8B0B1231938A0C8B0DA834
:1060C0000CA90D80050508126084E84970F7900955
:1060D00012E06007640160030261AB1231938A0C25
:1060E0008B0DA80CA90D8003126084E849603688E6
:1060F000828983126DE2900553E06A7003A3E06B1E
:10610000600D12748739F583126DE2EA4B70D988FD
:1061100082898312608A900553E0687003A3E06966
:1061200070030261AB7A167B00123CF18A0C8B0D76
:10613000AE0CAF0DEE4F607390055312608A8E82E5
:106140008F83126094900548E08E828F83A3A3F022
:106150001232EFE98E828F83A3A3A3A3A3F090153D
:106160004B127715F07C677D0512622E1246EDAA60
:1061700018AB1979411247B9851882851983E060F7
:106180000890077712608A800478FE79FF8E828FEC
:1061900083A3A3A3A3A3A3A3126094126236E50A68
:1061A000F0A3E50BF08E0A8F0B050890078BE0F843
:1061B000E508C39850047A008022E508C398FAC322
:1061C000940640027A057900800DE50A127488353C
:1061D0000B125B5AF50B09E9C39840EE750900787C
:1061E00009122A25780A122A21EAF5097809122AC1
:1061F0002590078BE0F5097809122A25AD087C0067
:106200007A827B07900780E0F91241657405122AB3
:1062100034900912E060046401700BEE4F6007EEE9
:10622000FAEFFB123CF7122EE774010254D6EE246B
:106230000BFAE43FFB22EE12623B221274883FF518
:106240008322EEFAEFFB7F060226BD74EC12242DAA
:1062500074FF122AC88A0A8B0B7E008E0E8E0F12D4
:10626000607B350B12788AFFAC18AD197A007B0081
:10627000799D122F41851882851983E0F8EFC39824
:106280004003026326E0C39FFEC3940B40027E0AD4
:10629000EE75F007A4FAABF0123CF18A088B098A7C
:1062A0000E8B0FEA450F607C750C00801A85088202
:1062B000850983A3A3A3A3A37403F0E5082407F52A
:1062C0000850020509050CE50CC39E5059AC08ADF9
:1062D00009850C10E5102FFAE43400FB798B122F9E
:1062E00041850882850983A3A3A3A3A3E0146008C2
:1062F00014601314601F80B5850882850983A3A3E9
:10630000A3A3A3E480B4850882850983A3A3A3A3E0
:10631000A3740180A5850882850983A3A3A3A3A3F1
:10632000740280967E007508007808122A25780E7F
:10633000122A21EEF5087808122A25EFF5087808C8
:10634000122A257405122CC7E0FD7C00E50A1267AD
:106350002E350BFBE50A12648E350BF583E0F9123E
:1063600041717405122A34E50E450F6007AA0EAB81
:106370000F123CF77401122A347F0C0226BD74EA16
:1063800012242D74FE122AC88A148B15750A007502
:106390000B00127884F508AC18AD197A007B0079EF
:1063A000A31249B185080C85188285198312608A69
:1063B000C3E50C98E499507D851882851983E0C364
:1063C000950CFEA3E09400FFC3EE9404EF9400400C
:1063D000067E037F008004EE4F605AEEFAEFFBEA80
:1063E00075F015A4FAA8F075F015EBA428FB123C83
:1063F000F18A0C8B0D8A0A8B0BEA450B6037750905
:1064000000750E00850E10C3E5109EE49F502BAC66
:106410000CAD0D850E12850810E5122510FAE43436
:1064200000FB79A21249B1E50C2415F50C500205C8
:106430000D050E80CF75098B7E00750C00780C124F
:106440002A25780A122A21EEF50C780C122A2578D2
:1064500008122A257405122CC7E0FDAC0912647AD3
:106460001241777405122A34E50A450B6007AA0A1F
:10647000AB0B123CF77402025F6DE51412672E3508
:1064800015FBE51412648E3515F583E0F922240F0F
:10649000F582E42274F612242D74FF122AC8EAFE53
:1064A000EBFF1264EE1275CEA3A3A3A3A3A3A3A331
:1064B000E0F9122F05E9851882851983F075080027
:1064C0007808122A257401122A9A880889097808FE
:1064D000122A217508357509807808122A2112645C
:1064E000F41240CF7405122A3474010253BDEE1227
:1064F00060803F2279011264FEFAE43FFB22EE2421
:1065000002FCE43FFDEE240F2274F412242D74FAF1
:10651000122AC88A088B09EA12748E12749EFFEE42
:10652000FAEFFB122DF1E96013123265EAFCEBFD84
:10653000EEFAEFFB1246E7E96401700A7401122CCF
:10654000C7E4F0A380097401122CC7EEF0A3EF1288
:106550007754A3A3A3A3A3E0F8A2E6500874031200
:106560002CC77401F0E8A2E750087404122CC77419
:1065700001F07405122CC7E4F004122AA2122F3580
:10658000E9851882851983F07A007B0012328975BB
:106590000A00780A122A257401122A9A880A890B9D
:1065A000780A122A21750A34750B80780A122A217A
:1065B0001265C01240CF7405122A347406026A9222
:1065C0007901E5082402FCE43509FDE508240FFA09
:1065D000E43509FB2274F612242D74FF122AC81226
:1065E0006648F509A3E0F508A909122EF3E9851814
:1065F00082851983F0900912E0700B7401650870B0
:1066000005A90912421FEE240B126640702C750872
:10661000007808122A257401122A9A8808890978B4
:1066200008122A217508367509807808122A211265
:1066300064F41240CF7405122A340264E9EE240E89
:10664000F582E43FF583E02212664C22EAFEEBFF7E
:1066500012665C3FF583E0126663E022EE2413F5D8
:1066600082E422F8A3E0F98882898322C082C08371
:10667000900912E07003124225026DD174F41224C5
:106680002D74EF122AC8EAFEEBFF1254DC90077754
:10669000E065087004A3E065097052A818A919887C
:1066A0000A890B780A122A21750A11750B00780ADB
:1066B000122A217C007D007A817B00123D7B7404CC
:1066C000122A34E97027750A00780A122A25740103
:1066D000122A9A880A890B780A122A21AC08AD0975
:1066E0001267131241297403122A348021750A118A
:1066F000750B80780A122A217808122A2112663D29
:10670000FD7C841267131241357404122A3474110B
:10671000026A9212671722EE12672E3FFBEE240FD9
:10672000F582E43FF583E0F922FCEFFDE508240261
:10673000FAE42274F112242D74EB122AC81266486E
:10674000FCA3E0FAE4CAFBEC2AF508E43BF5099067
:106750000777E065087004A3E0650960030268023A
:1067600088828983A3A3E09410500F88828983A331
:10677000A3E085188285198380088518828519838E
:106780007410F0E0C0E07404122CC7D0E01275BFA2
:10679000A3A3A982AA83890C8A0D750E00780C1216
:1067A0002A1D7407122CC7E0FC7D007408122CC748
:1067B000AA82AB83123C2B7403122A347404122A6B
:1067C0009A880A890B780A122A21750A11750B001A
:1067D000780A122A217C007D007A817B00123D75A7
:1067E0007404122A347404122CC7E09007B26005B6
:1067F000E0D2E48003E0C2E4F0851882851983E4E6
:1068000080088518828519837484F0E0C0E07401E3
:10681000122CC7D0E0F07402122CC7E508F0740304
:10682000122CC7E508F0125CF9126861122A25746F
:1068300002122A9A880889097808122A21750814F0
:106840007509807808122A2179031264F61240CF64
:106850007405122A347415026CEBE5161275B13505
:1068600017F583E0F50878082274F412242D74E0FB
:10687000122AC88A088B09AC18AD191240BD9009BC
:1068800012E0640270337402122CC7AE82AF83121E
:106890003265EEFCEFFD1246E7E9601D12326B8AAD
:1068A0000A8B0BA80AA90B851882851983E06870EA
:1068B00003A3E0697003026A901234217402122C5F
:1068C000C7126DD8123337E964017003026A9074FD
:1068D00018122AA21232777402122CC7AC82AD832E
:1068E0007418122AA21246E7E960321232718A0A3B
:1068F0008B0BA80AA90B851882851983E0687003A1
:10690000A3E069601885188285198312608A900552
:10691000491260947A497B05794B1247BF9009125E
:10692000E06007640160030269CE1273ADC082C0EB
:106930008312326B8A088B09D083D082E06508709D
:1069400004A3E06509605C7402122CC7AA82AB83C1
:10695000122E5D8A088B09A808A909E849602688D3
:10696000828983A3A3A3A3E06401600D8882898345
:10697000A3A3A3A3E06402700C7402122CC7AA8222
:10698000AB83122E699005E7126AA0601690090683
:10699000E06401700E126DDC9005E8E0F5838882FA
:1069A00012261E12326B8A088B09A808A9098518BD
:1069B00082851983E0687003A3E069601174021294
:1069C0002CC7126DD8122E3FE96003123F497402A2
:1069D000122CC7126DD812340F7900126DDC1230F0
:1069E00085740B122CC7E4126AA4F8A3E0F9740CA6
:1069F000122CC7126094740B122AA2122E0FE96097
:106A00003F7C087D0079007418122AA2123C37746A
:106A10000E122CC7AC82AD837418122AA21246E75C
:106A2000E9601D7402122CC7AC82AD83740E122C67
:106A3000C7AA82AB83122DEB740B122AA2122E214D
:106A40007402122CC7AC82AD83740E122CC7AA82BA
:106A5000AB83122DEB740B122AA2122E15E96030B3
:106A6000740C122CC712608A851882851983E0681D
:106A70007003A3E069601985188285198312608A02
:106A8000740C122CC7126094740B122AA2122E21BD
:106A90007420122A347F040226BDF582E438F5837F
:106AA000126F6322F0851882851983E02274F11237
:106AB000242D74F6122AC8EAFEEBFF750800900830
:106AC0001E126AA070507A377B00123CF190081EAB
:106AD000EAF0A3EB12729860197C377D00790012FE
:106AE0003C37EEFCEFFD90081E126DE212408DE97E
:106AF000700B8518828519837488026C5412759204
:106B0000126CF37401F07C997D409004D3126DE215
:106B1000124A1D026CE9E0C8126CF37402F0EEFC3C
:106B2000EFFD1271EE12408DE9700C851882851907
:106B3000837488F0750801750AE8750B07780A12E6
:106B40002A21126DF212284512759224281271E141
:106B5000FC126E2512759224141271E1F9123FF1A4
:106B60007404122A34126D00126D2624311271E160
:106B70006043127282FAE433FB123CF190081EE08B
:106B80002432126D3B6022750CE8750D07750E00FE
:106B9000780C122A1D127282FCE433FD126E101260
:106BA0003C2B7403122A34800C8518828519837457
:106BB00088F0750801780A122A21126DE61228451C
:106BC00012759224111271E1FC126E071275922453
:106BD0002B1271E1F9123FF17404122A34127592EA
:106BE0002434126D2624341271E16035127279FA60
:106BF000E433FB123CF190081EE02435126D3B603B
:106C000042750CE8750D07750E00780C122A1D12DE
:106C10007279FCE433FD126DFE123C2B7403122AD0
:106C200034E508A2E04025126D001271E170089071
:106C3000081E12724560157B007A0079001240939D
:106C4000026CE98518828519837488F0851882851D
:106C500019837486F07409122CC774021273F1122E
:106C60006D0F122CC7E8F0A3E9126D20F508780823
:106C7000122A257401122A9A880889097808122A8A
:106C8000217508207509807808122A217901740677
:106C9000122AAAEEFAEFFB1240CF7405122A341220
:106CA000723470427409122CC77402F0126D09120A
:106CB0002CC712729F122A257401122A9A880889F9
:106CC000097808122A217508207509807808122A87
:106CD0002179017406122AAA90081E126DE2124050
:106CE000CF7405122A34124087740A122A347F079F
:106CF0000226BD126CF722242EF582E438F5832299
:106D000090081E12720A24312290081E126D17A3D9
:106D1000A312608E740122E0F8A3E0F5838882223A
:106D20001273F1A3E022F582E438F583126D31C8C5
:106D300022E9F090081EE0F8A3E022F8A3E0340076
:106D4000F988828983EAF0A3EB1275C8126F632277
:106D5000C082C08390081E126AA06075E0C8243506
:106D6000126A9A6006126DFE123CF7127592243276
:106D7000126A9A6006126E10123CF7127592241273
:106D8000126A9A6009126DE6126DE2123CF71275F2
:106D9000922415126A9A6006126E25123CF712753B
:106DA000922429126A9A6009126DF2126DE2123C65
:106DB000F7127592242C126A9A6006126E07123C22
:106DC000F790081E126DE2123CF790081EE4F0A343
:106DD000F0D083D0820229E6AC82AD83851882850B
:106DE0001983126E1F221272072412F582E438F5FD
:106DF00083221272072429F582E438F58322127265
:106E0000072435126E1922127207242C126E1922D1
:106E10001272072432126E1922F582E438F583E0EB
:106E2000FAA3E0FB221272072415126E192274F1E4
:106E300012242DEAFEEBFF8C088D09750A018C0CDB
:106E40008D0D750E00780C122A1D7C177D00123CEA
:106E50002B7403122A34EE2412126F2FF0A3F0EEDB
:106E60002415126F2FF0A3F01273ADE0603AEE24F8
:106E700012F8E43FF9880C890D1273D6123CF11216
:106E80006F506021E5082412126F43122A1DE50895
:106E90002411126F37125F8E126DE2123C2B7403B5
:106EA000122A348003750A00E5081273BB6035EEC0
:106EB0002415F8E43FF9880C890D1273D6123CF1C1
:106EC000126F506055E5082415126F43122A1DE514
:106ED000082414126F37126F1F126DE2123C2B74CC
:106EE00003122A34E50AA2E0402BEE2412F582E4D4
:106EF0003F126A9E6009125F8D126DE2123CF7EE3E
:106F00002415F582E43F126A9E600AEE126F1F128A
:106F10006DE2123CF7A90A026CEE750A0080CB12F2
:106F20006F23222415F582E43FF58322EE2414F525
:106F300082E43FF583E422127582E025E0FCE4332D
:106F4000FDEE22127582E0F50CA3E0F50D780C221F
:106F5000850C82850D83125931850C82850D831233
:106F60006F6322E0F8A3E0F9E8492274EE12242DC1
:106F700074ED122AC8890A8A0E8B0F750C00750DE4
:106F800000750BFF7510FF7511FF7508007509007E
:106F9000851882851983E412729860177403650A54
:106FA00060067402650A7010E0C824301271E16551
:106FB0000F600579000271D77C997D407A007B00D3
:106FC000124A1D7401650A700A8518828519837436
:106FD00085803DE50A60067403650A701990081EF5
:106FE000127214F07403650A7029E50E6029851881
:106FF00082851983801A7402650A701BE50E900859
:107000001E7005127214800812759512722B74028C
:10701000F08004E50A601E12721A701912723E6046
:1070200005126D03800A127245600A1275922434AB
:107030001271E114F012723E602212530AF5091225
:107040007282F8E433F990081EE0FAA3E0CA243211
:10705000127256241D1271FB2425802E1272456077
:107060002E90081EE02417F508A3E03400F509125D
:107070007279F8E433F990081EE0FAA3E0CA2435E7
:1070800012725624061271FB240E1271E1F50B7474
:1070900009122CC77402126AA46003027145E50844
:1070A0004509700302714512721A70047E22800233
:1070B0007E21850882850983126D0F122CC712600C
:1070C00094900822E0C0E01275922430F582E438F2
:1070D000F583D0E0F07412122CC77403F0AC0CAD41
:1070E0000D740A122AA21246ED850882850983A32F
:1070F000E0F50C780C122A25780B122A25740C1254
:107100002A9A880C890D780C122A217810122A21CB
:10711000E5082406F50CE43509F50D780C122A2152
:107120001271E9F97409122AAAEEFA7B00124141A0
:107130007408122A347C997D409004D3126DE212B7
:107140004A1D0271D5126D09122CC712729F122AA4
:10715000257401122A9A880889097808122A21754B
:1071600008207509807808122A2179017406122AEC
:10717000AA90081E126DE21240CF7405122A341232
:107180007234704E1275922419F582E438F5831228
:107190006D11122CC7E8F0A3126D2C2418F582E4AF
:1071A00038126861122A257401122A9A88088909FE
:1071B0007808122A217508207509807808122A217A
:1071C00079017406122AAA1271EE1240CF740512C8
:1071D0002A3412408779017413122A347F0A022656
:1071E000BDF582E438F583E0221276A6E02290080D
:1071F0001EE02417FAA3E03400FB22F50CA3E034D0
:1072000000F50D1272072290081E12720E22E0F88D
:10721000A3E0C82212722474012290081E12722464
:10722000E064012212720E12722B22242FF582E4E6
:1072300038F58322127207126CF7E0640222127290
:107240008890081E221272492212720E2434F5828E
:10725000E438F583E022F582E43AF583E028F8A3E8
:10726000E039F9E824FEF582E934FFF583E0F51012
:10727000A3E0F51190081EE02290081E1272492525
:10728000E02212728825E02290081E12720E24312C
:10729000F582E438F583E022126D32F9E84922E8FC
:1072A000F0A3126D31F5838882A3E0F508780822F7
:1072B000C082C0837B007A857901124093026DD130
:1072C00074F412242D8C088D09EA240F12775A12B7
:1072D00076B012608A8C828D83A3A3126094EA2414
:1072E0000E12775AA3F01274951273E21275A4501D
:1072F000010FFCEFFDE5082406FAE43509FB124610
:10730000EDEE2408FE50010F8E828F83E0C0E01264
:1073100076A2D0E01274A3F8127692E81275A85003
:10732000010FE50824121273B5A3F0E50824151225
:1073300073B51273EBA30EAF83C0E01273ADD0E050
:10734000F06028E50824121273CD123CF112776D1B
:107350006019E50824121273C01273AFE0F91240ED
:10736000158A0A8B0BAE0AAF0B8007E508241112B1
:1073700073B58E828F83E0A3AE82AF83C0E01274B8
:1073800079D0E0F0601FE50824151273CD123CF1AE
:1073900012776D6010E50824151273C01273BBF9E3
:1073A0001240158005127479E4F0026A95E508240C
:1073B0001112758222127582E4F02212747FE0228B
:1073C000127582125958EEFAEFFBE50822F8E435FF
:1073D00009F9880A890BE01273DB2225E0FAE4330D
:1073E000FB22FF12770A8C828D8322A31273F1E0B5
:1073F00022F08E828F832274F612242D8C088D0940
:10740000127495FFEEFCEFFDAA08AB091246EDEEF3
:107410002408FE50010F8E828F831277BB1274A353
:10742000850882850983A3A3A3A3A31275A4500191
:107430000F8E828F83E0F8E50812748EE81275993A
:107440007403687026EEFCEFFDE508240BFAE435C2
:1074500009FB1246ED8E828F83A3A3A3A3A3A3A34C
:10746000A3E0C0E0127479D0E0800A12768612752B
:107470007CE8F0A3E9F00253C0E50812747F221201
:1074800074883509F58322E82414F582E422126019
:10749000801275852212773212749C22F583E0FEE9
:1074A000A3E0221276D112770E2274F212242DEA72
:1074B000FEEBFF750A00EE2410126640C3940C40E8
:1074C0000D1276FB127595240B1271E1F50AA80ACC
:1074D000E828F8E433F9E8240DFAE439FB123CF12A
:1074E0008A088B09EA450970030275731264EE126B
:1074F00076EA8A828B831276CD7078EEFCEFFDEA15
:107500002403FAE43509FB1246EDEE2408FE50018F
:107510000F8E828F83127706850882850983127504
:10752000A750010F12757AE4F0E50A6046E50824D9
:107530000DF8E43509F98E828F83E0C0E012757A88
:10754000D0E012768DC0E012758AD0E01275998570
:107550000A0B8E828F83E0FCA3E0FBEC8882898398
:107560001275B7500109EE2402FE50010F150BE50C
:107570000B70DFAA08AB09026246E508240B1275FE
:107580008222F582E43509F58322E508240C127580
:10759000822290081E12720A2212759D221276D93A
:1075A0000EAF8322A3A3A3A3F0A3E9F0EE2402FE6F
:1075B00022240EF582E422125932E82402F8221223
:1075C00075C3221275C8A322F08882898322126EA5
:1075D0001D8A828B83227F010226BD74F212242D24
:1075E00012772E125308850882F583E0F50DA385E6
:1075F0008208858309A3A3E0F50C1276E53400FB2D
:10760000123CF18A0A8B0BAE0AAF0BEE4F60378E3D
:10761000828F83E50DF0850882850983E0FA127771
:1076200041850882850983A3A3A3A982AA83890827
:107630008A09880A7808122A1D1276E03FFB123C5C
:107640002B7403122A3402624274F712242DEA24A6
:1076500013F8E43BF988828983E0FAA3E0F5838A92
:1076600082127760127681126663A3E0FA888289BB
:1076700083A3A3E0F9EA8C828D83A312609502753F
:10768000D61275C8E02212770EF8E5082212759D11
:10769000E02212769622E508240FF582E43509F5FA
:1076A00083221276A622E5081275B13509F58322E8
:1076B0001276B5A322F08A828B83A3221276C0228F
:1076C000F08A828B83A3A3A322A3A3A3A31276D1C0
:1076D000221276D9AE82AF8322F08E828F83A322CC
:1076E000AC0C7D00EE2404FAE4221276EE22F5833F
:1076F000E0FEA3E0FF8E828F83E0221276FF22124B
:10770000665C3FF5832212770E228E828F83E0FA29
:10771000A3E0F9EA22E08E828F83A3A3A3A3A3A30D
:1077200022F0850A82850B83A3228C088D091277AB
:107730003222EA12665D3B22F0850882850983A326
:1077400022127766EA8E828F83A3F0A3E912775420
:10775000E50CF0221276D9A3A322F582E43BF5834F
:10776000E08C828D8322A3E0F8E4C8F922850A82A6
:10777000850B83125931850A82850B83126F632230
:1077800074F612242D12772AF5831277B41273E25D
:107790001275A850010F1267293509FB1246ED8EAC
:1077A000828F83A3A3A3A3A3A3A3A31277BBA3A3A3
:1077B000F00253C012608EE8FEE922127861A3A3A2
:1077C000221277C522E0FA127766EA28221276C0E2
:1077D000A3A3A3A32274F612242D12772A12784EA3
:1077E000123C43EAF8EBF9ECFAEDFB8508828509D7
:1077F00083122CB0EE2404FE50010F8E828F83E0A2
:107800008508828509831276C9C3940650051278CB
:10781000668037850882850983A3A3A3A3E064FE5D
:10782000600E850882850983A3A3A3A3E0F4701BDF
:10783000127859127599850882850983A3A3A3A399
:10784000E0F47007127873F0A3E9F00253C01274E9
:107850009CFF7904EEFAEFFB228E828F831278610F
:1078600022127866A322E0850882850983A3A3A358
:10787000A3A32212770A850882850983A3A3A3A361
:10788000A3A3A322EA1260803515F583126D17E0D9
:107890002274F712242DE99007C1F07A157B80122B
:1078A00041837A387B009007C1E0F9124183900749
:1078B000E274CDF0A3743FF09007E074D3F0A374AA
:1078C0003FF09007DE74C7F0A3743FF09007CB74CD
:1078D00002F09007C374FEF0A304F07F010226BDFE
:1078E00074F212242DEAFEEBFF54807003027A0436
:1078F000805279001233738A0A8B0B750C00780C56
:10790000122A257808122A21780A122A2190059D28
:10791000127D7B9007C2E0F9123FBB7405122A3436
:107920009007D9E060179080C41228417A087B0044
:107930009007C1E0F9123DB77404122A34AA08ABCB
:1079400009123C559007C1E0F9123C678A088B097F
:10795000E508450970030279FC850882850983E002
:1079600024CF603E14607E245F70D2E508240CF5BD
:1079700082E43509F583E0F50AA3E0F50B780A12F5
:1079800026710000020038009979158090793D79C0
:10799000AA08AB09123FAF80A4AA08AB09123FA9FD
:1079A000809B9007CEE0C39404509290055CE0F970
:1079B0009080C8122C98122F4DE97081850882851D
:1079C0000983127EF39007D0127C6B8508828509AB
:1079D00083A3A3127EF39007D2127C6B9007D97415
:1079E000FFF002793D9007D9E0F460030278F2AA33
:1079F00008AB09123FB59007D9E480E5EEFAEF64D1
:107A000080027A92EEA2E050259007DDE0900548D2
:107A1000F07ADD7B0779E11247BF123F3790059D71
:107A2000E4F0A3F07901123373EE64018062540232
:107A300060399007CC127EF5E84960259007CCE0CC
:107A400024FFF0A3E034FFF09080CC1228417A02AA
:107A50007B009007C1E0F9123DB77404122A34800C
:107A6000059007CEE4F0EE64028025EE5408602510
:107A70009007D9E060179007D8E0F99007D4122C4E
:107A800098122F4DE970069007D9E014F0EE6408C3
:107A9000FAEFFB80047A007B007F060226BD74F4B7
:107AA00012242D74F7122AC8EAFEEBFFAC18AD19A8
:107AB0001240C37404122CC7E0C39406505A127CBF
:107AC000586003027C3A7405122CC7E07003027CF4
:107AD0003AC394064003027C3A7404122CC7E0F9BE
:107AE000851882851983122C98122F4DE9600302A4
:107AF0007C3A127C449007C2127EFB127C687405AB
:107B0000122CC7E014F08518828519837CD47D0778
:107B10007409122962027C3AE064FE7076740612DF
:107B20002CC7127C4F4003027C3A7406122CC7E02B
:107B3000F91232B979008518828519837808122CD8
:107B400070E97808122A69E508A2E0400709E9C34C
:107B5000941B40E2900548E0697003027C3AE9908A
:107B600007DDF0900539E075F064A4F508A8F0E4AD
:107B700028F5093395E0F50AF50B7808122A197AE9
:107B8000017B009007C1E0F9123DB77404122A345A
:107B9000027C3AE0F4705C7406122CC7127C4F40F1
:107BA00003027C3A7406122CC7E0F91232B9851828
:107BB00082851983122CA4E8494A4B6027851882D4
:107BC0008519837808122C709005567808122ADEE1
:107BD0006012851882851983122CA4900556122CE8
:107BE000B0123F377407122CC7E0FAA3E0FB123F34
:107BF000C18047127C5870428E828F83A3A3127C6F
:107C0000637508007808122A257808122A25E4F5F9
:107C1000097808122A217808122A217808122A21C4
:107C20009080D01228417D007C807AC37B07127C33
:107C300044F912417D740C122A347409122A347FDB
:107C4000040226BDEE240FF582E43FF583E022E036
:107C5000F890059FE0C39822EE240BF582E43FF5EF
:107C600083E022E0F8A3E0F99007C3E8F0A3E9F08D
:107C70002274F712242D74FD122AC8EAFEEBFFAC21
:107C800018AD191240B7851882851983E0701874F1
:107C900001122CC7E05440600E8E828F83A3A3E0B4
:107CA000FAA3E0FB123FC17403122A340278DB749A
:107CB000F212242D8A0C8B0D7A00850C828B83A303
:107CC000A3A37808122C70900548E07808122A695E
:107CD000E508A2E05009E0F8E50C28127D6CFA797D
:107CE00000850C828B83A3A3A37808122C70E978FB
:107CF00008122A69E508A2E05068E50C29127D6C9B
:107D0000C39A505E90059B127C6375081078081228
:107D10002A25780C122A219007D21228459007D0E4
:107D2000127D7B7900123FBB7405122A349007CF75
:107D30007401F09007CEE070209007CC743CF0A363
:107D4000E4F09080CC1228417A027B009007C1E0D9
:107D5000F9123DB77404122A349007CEE004F00201
:107D60007A9909E9C3941B50F6027CE1F582E43B61
:107D7000F583A3A3A3A3A3A3A3E022E0FCA3E0FDB8
:107D80007AC37B072274EC12242D89118A128B137B
:107D9000ECFEEDFF751000750800750900790074A0
:107DA00016122CC7E0F50AA3E0F50B850A82850BB5
:107DB00083A3A3A3780C122C70E9780C122A69E52E
:107DC0000CA2E05002051009E9C3941B40DDE51048
:107DD0006055FA7B00123CF18A088B09EA4509607C
:107DE000467A007900850A82850B83A3A3A3780CC9
:107DF000122C70E9780C122A69E50CA2E05021E5FA
:107E00000A29F582E4350BF583A3A3A3A3A3A3A3B7
:107E1000E0C0E0E5082AF582E43BF583D0E0F00A13
:107E200009E9C3941B40BE750C00780C122A257416
:107E300019122CC7E0F50C780C122A257808122AA2
:107E4000217418122CC71228458E0C8F0D780C1235
:107E50002A21850A82850B83A3A3A3122841AD1092
:107E6000850A82850B83A3A3E0FCAA12AB13A91198
:107E700012417D740C122A34E50845096007AA08EE
:107E8000AB09123CF77F0C0226BDC082C08390056F
:107E90009BE06A7003A3E06B600B90059BEAF0A384
:107EA000EBF0123F37D083D0820229E674F6122419
:107EB0002DEAFEEBFF7A067B00123C4FEA4B602E68
:107EC0008A828B837431F08E828F83127EF58A8250
:107ED0008B83A3A3E8F0A3E9127EFB8A828B83A3A2
:107EE000A3A3A3127C6B9007C1E0F9123C5B7F0255
:107EF0000226BDA3A3E0F8A3E0F922F08E828F83CF
:107F0000A3A3E0F8A3E0F92274F412242D8A088BCD
:107F1000097A227B00123C4F8A0A8B0BAE0AAF0B08
:107F2000EE4F60628E828F837432F08508828509FD
:107F300083E08E828F83A3A3F0850882850983A3C3
:107F4000122CA48E828F83A3A3A3122CB085088247
:107F5000850983A3A3A3A3A3E0F508A3E0F509750E
:107F60000A007808122A1D7C1B7D00EE2407FAE423
:107F70003FFB123C2B7403122A34EEFAEFFB9007FE
:107F8000C1E0F9123C5B027C3FC082C0839007CF06
:107F9000E060238A828B83A3A3A3E070198A828B7B
:107FA00083A3E0701190059DE4F0A3F079011233F2
:107FB000739007CFE4F0027EA5C082C0838518824B
:107FC000851983E0F8A3E0F9E84960128A828B837F
:107FD000ECF0A3E824FF18E934FFF94870F2D083ED
:107FE000D0820229E67409F5D575D4167409F5D343
:107FF00075D21ED2B80229E6851A87000229E6FF4B
:108000003D48C1360F31294A132D173EA33F59472A
:108010003B47334300000000000000000000000068
:108020000000000000000000000000000000000050
:108030000000000000000000000000000000000040
:108040000000FFFFFFFFFFFFFFFF0008000400022A
:108050000001FFFFFFFFFFFFFFFF00000000000027
:108060000000FFFFFFFFFFFFFFFF02050200080106
:108070007400000000000000000000000082003AD0
:10808000003B0002000206020400000019E0FCFFB1
:10809000F8FF0000E71F030080510100FA00000014
:1080A000100E0000000000FF30000000E803000098
:1080B0000943388664000000E20400005802000012
:1080C000BC0200003200000000F8FF0760EA000078
:1080D00000000000020000000B0000000100000092
:1080E0000A0000003C000000FEFFFFFF1F00000030
:1080F00008000000975118006AAEE7FF965118007B
:108100009F020000E9FFFFFF0000FF0000000000E9
:10811000000000000A74F712242DE99005A0F090E9
:108120000555E4F01246C39005B4E4F0A3F09005C1
:10813000A1F0A3F01233C7900912E060046401704B
:1081400006122E2D122FEF1246C9900516E4F0A349
:10815000F01247FB02B14F74F012242DEAFEEBFF40
:10816000548060689005A0E0F9123C678A088B098A
:10817000EA4509604F7C0080010CEC75F003A4F81F
:10818000A9F074E828F582744E39F583E493F4601D
:108190002CE493F88508828B83E06870DCAA08ECF5
:1081A00075F003A4F874E928F582744E39F583E478
:1081B00093C0E0740193F583D08212261EAA08AB07
:1081C00009123C55EEFAEF6480028448EF542060B7
:1081D0001E1232298A088B09EA4509600A123145C4
:1081E000AA08AB09123C55EEFAEF642002844890CD
:1081F0000912E064027024EEA2E0501F90055AE0DC
:10820000640F70117900123115E9600990153C1264
:10821000D33312312DEE640102834EEE54207003ED
:1082200002831F750C007A207B009005A0E0F912F4
:108230003DC9EA4B4C4D70179080D41228417A20EA
:108240007B009005A0E0F9123DBD7404122A347C35
:108250000079047A007B001231F38A088B098018B8
:10826000850882850983A3A3A3A3A3A3A3A3A374BF
:1082700001F0850A08850B09E508450960777C004F
:108280007904AA08AB091231F38A0A8B0B750C0129
:10829000E5082404F8E43509F98882898312EF247B
:1082A00012EA7970CD850882850983A3A3A3A3A3CD
:1082B000A3A3A3A3A3E0640170A685088285098314
:1082C000A3A3A3A3A3A3E054047095850882850902
:1082D00083A3A3A3A3A3A3A3A3A37406128B4A708F
:1082E0000374B7F0E0FA85088285098312862612A6
:1082F00031270282721231C37C0079017A007B003F
:108300001231F38B09EA45097010E50C700C7A20E4
:108310007B009005A0E0F9123DC3EE6420802FE0C1
:1083200060076401600302841EEE5410600812307E
:108330002BEE64108018EE544060081230A3EE64F7
:1083400040800BEE5480600B122EF9EE6480FAEF41
:10835000028448EF540160169005D312CB79600671
:1083600012C5E312261EEEFAEF6401028448EF54B0
:10837000086047122FFB900902E0640170349009F5
:1083800003E0602EF508E4F509F50AF50B9080ACE2
:10839000780C122C707808790C12233E7808122A77
:1083A000197A007B089005A0E0F9123DBD74041213
:1083B0002A34EEFAEF6408028448EF5410601290F9
:1083C00005B2E06005E4F0122FFBEEFAEF641080D6
:1083D00077EF544060489005DD12CB796039900505
:1083E000E312CB796031900906E0640170299005B1
:1083F000DD12C5E012261E9005E312C5E012261E0E
:108400009080CC1228417A007B409005A0E0F912C0
:108410003DBD7404122A34EEFAEF6440802AEF5412
:1084200002600A123391EEFAEF6402801BEF5404EB
:10843000601912CA8312C895790190055312D3337B
:10844000122F77EEFAEF6404FB80047A007B0002BF
:10845000C120C082C08374EA122AC87C167D0079CC
:1084600000AA18AB19123C377408122CC77402F01A
:108470009005491297701284917409122CC712C882
:10848000957413122CC7E412C9DF1247E9741680E1
:108490000EE8F0A3E9F090055312D0F4227408120C
:1084A0002A3402C15874F712242D74DF122AC8EA44
:1084B000FEEBFFEE4F602DAC18AD1912324D740675
:1084C000122CC7E0601E7417122CC7E0FD74011255
:1084D0002CC7E0FCEEFAEFFB7900122DA9E960044D
:1084E00079A480027900742102B14C74F412242D15
:1084F000EAFEEBFF8E828F83A3A3A3A3A3A3E05482
:10850000406016128B3E123307E960077AFF7BFF4B
:108510000285ED12C5DC0285E0900912E060076477
:108520000160030285C6900540E0A2E14003028598
:10853000C68E828F8312862012C9A5A3A3A3A3E0AF
:10854000FA88828983A3A312D5068E828F83A3A380
:10855000A3A3A3A3A3E05410600479408002790090
:10856000750AFE750BFF780A122A2112B61412281A
:1085700045AC08AD09128B3E1230017404122A3446
:10858000E5086A7003E5096B600B12B6196A70039F
:10859000A3E06B704E750A00780A122A2579028EC4
:1085A000828F8312B204AA08AB09123349740112F4
:1085B0002A347508CDAA088E828F8312862612313E
:1085C00027E9604C8057900912E06402600FE06078
:1085D00004640170DD900540E0A2E140D5900549BA
:1085E00012D33374FE6A700374FF6B60C512C5DC6E
:1085F00012DA27123307E98E828F83600512AA3AB6
:10860000800312AA4F12AA581247EFE9F50870A585
:10861000EE4F60097901EEFAEFFB1231CF02BEEDA9
:10862000E0F812B2462212EDEFE0F92274F61224BD
:108630002DE9FEEAFF7A0F7B00123C4FEA4B601FE8
:108640008A828B83740CF0EEA3A3F0EF8A828B8373
:1086500012AE8D9005A0E0F9123C5B7900802FEE00
:10866000F91231F98A088B09A808A909E849601CA0
:1086700088828983A3A3A3A3A3A3A3A3A37406129D
:10868000E669E0F91230B5EEF91231D5791002C47D
:10869000CC74F412242D90055AE0640F7030EA4B2C
:1086A000602C900555E064086005E06404701F8A42
:1086B000088B09E4F50AF50B7808122A197A017B70
:1086C000009005A0E0F9123DB77404122A34029814
:1086D0005B74F212242DEAFEEBFF8C088D09890AE7
:1086E000740E122CC712978A850C82F583E4F0A3CE
:1086F00012C89BE0F91232E3E9602612D326123346
:1087000007E96402701B8E828F83A3A3A3A3A3A394
:10871000A3A3A312B8AC850C82850D8312C89580E3
:1087200003750A0012B03E14602514603A14605BB1
:1087300014606314603F14607D24FE70030287D0D0
:108740001470030287E41470030287F70288057827
:108750000C122A21AC08AD09EEFAEFFB12301374AB
:1087600002122A34028800AC08AD09EEFAEFFB12BF
:10877000301902880F12D326123307E960030288EA
:1087800005EEFAEFFB12306702880FA90AEEFAEF46
:10879000FB12334F806A12BB5464027068E50A70A2
:1087A0000A12DAE07003A3E0697064EEFAEFFBA945
:1087B0000A1232D7804A12DAE07003A3E0697045EA
:1087C00012BB546402703EEEFAEFFB1232BF803FE0
:1087D0009005D512CB796037EEFAEFFB12C5E312A4
:1087E000261E802B12DAE07003A3E0697017EEFA00
:1087F000EFFB12335B8018EEFAEFFBA90A12336726
:10880000E9F50A800A750A007AD37B001242CDA9E5
:108810000A02D10574F412242D74DB122AC88A08C6
:108820008B098A828B83A3A3E0F91231F98A0A8B20
:108830000BAE0AAF0BEE4F700302894585088285A7
:108840000983A3A882A983E0C0E012C863D0E01224
:10885000E68064F16033850882850983A3E064CDF6
:108860006027850882850983A3E0641A601B850858
:1088700082850983A3E064E9600F85088285098306
:10888000A3E064E16003028A2F900912E0600764AC
:1088900001600302895E8E828F83A3A3A3A3A3A397
:1088A000A3E05408700302895E8E828F83A3A3A382
:1088B000A3A3A3A3A3A37405F0900912E06004642A
:1088C000017053850882850983A3E064E9604790BD
:1088D00005D912CB79600612C5E312261E9005DB7E
:1088E00012CB796031900540E0A2E1502912CD51C0
:1088F000A3A3A312B0548882898312D3331233F70F
:10890000EA4B6012850882850983A3E0F99005DBB4
:1089100012C5E012261E8E828F83A3A3A3A3A3A356
:10892000A3A3A3E0640270108E828F83A3A3A3A3EA
:10893000A3A3A3A3A37406F0850882850983A3A338
:10894000E0F91231D51231C3900912E064027009C6
:1089500090154012D33312312D74250298587900A6
:108960001231CFE97003028A2F900912E060076488
:10897000016003028A04900540E0A2E14003028AFC
:108980000412CB74607E8E828F8312D333740412F0
:108990002AAA12CD6E12324D850882850983A3E082
:1089A00064E97020128B2D122A258508828509839F
:1089B000A3E0F50A780A122A2512D5171232837419
:1089C00002122A34740D122CC712CB6A12E9A512B6
:1089D000C8957409122CC7E06004794080027900C0
:1089E000740F122CC712B054740D122CC712D3334B
:1089F00012300DE9600E8E828F83A3A3A3A3A3A3DD
:108A0000E04420F0EE2404F50AE43FF50B8E828F5B
:108A10008312ACE6E0F9850A82850B8312D3331208
:108A200046D5850A82850B83EAF0A3EB0288B885D8
:108A30000882850983A3E0C0E07402122CC7D0E04D
:108A400012A4CCEEF0A3EF128B4AC0E07403122CF8
:108A5000C7D0E012E27AE0AA18AB19702E122F5399
:108A6000900912E06004640170247402122CC7E0C3
:108A7000701C128B3E123307E970369005D912CB69
:108A800079602E12C5E312261E80031232DD7402B5
:108A9000122CC7E064E97019128B2D122A25750A71
:108AA000E9780A122A2512D5171232837402122A83
:108AB00034900912E0600764016003028916900592
:108AC00040E0A2E140030289168E828F83A3A3A314
:108AD000A3A3A3A3A3A3E0640270398E828F83A310
:108AE000A3A3A3A3A3E05404602A128B3E1233076E
:108AF000E98E828F83700F12C5E074FFF0A312AD70
:108B0000017405028937A3A3A3A3A3A3A3A3A374FA
:108B100003028937850882850983A3E064E960033D
:108B2000028916EEFAEFFB12336D0289168E828FE0
:108B30008312D0F4E8FAE9FB750A01780A228E82E2
:108B40008F8312B21FFAA3E0FB22F0E50812EDE5D5
:108B50003509F583E02274F412242DEAFEEBFF754B
:108B600008007509008E828F83A3A3A3A3A3E060EE
:108B70003B75080812D32679FF122D1F8B0BEA458F
:108B80000B601075082C8E828F83A3A3A3A3A3E090
:108B9000D2E0F08E828F83A3A3A3A3A3E054036447
:108BA000016003028C60430811028C60EE241812ED
:108BB000BB576049EE241A12BB576003F4701D12B4
:108BC000DAE07003A3E0697006750822028C6090F9
:108BD0000555E064046003028C60801CEE241BF5E4
:108BE00082E43F12B63C241A12BB57FAEE24191243
:108BF0009830123079E97068750901806312D326C4
:108C0000123307E96402700375080112DAE0700399
:108C1000A3E0697006E508D2E1F508E50860158E65
:108C2000828F83A3A3E07006E508D2E58004E508FF
:108C3000D2E6F50812D326123307E964017006E57F
:108C400008D2E0F5088E828F83A3A3E0601212B0F1
:108C50003EF91232E3E964016006E508C2E0F50876
:108C6000900912E0600464017012E508A2E1400C72
:108C7000E509A2E04006E508D2E7F50802BEED747A
:108C8000EC12242D74CD122AC8EAFEEBFF8518825F
:108C9000851983129B4C75100075110075090090A1
:108CA0000912E06402701C8E828F83A3A3A3A3E049
:108CB000601190153E12CB79600990153E12D333A6
:108CC00012312D7405122AAA8E828F83A3A3A312B8
:108CD000CB6C12D33112324DE97003028E0279014E
:108CE0007407122CC7E0C394024001197409122CB6
:108CF000C7E0C3940240027900740E122CC7E064EE
:108D0000F87003A3E0F47003028E02740E122CC7F5
:108D1000E064F97003A3E0F47003028E02740E1293
:108D20002CC7E064FA7003A3E0F47003028E0274AF
:108D30000E122CC7E064FB7003A3E0F47003028EF4
:108D4000027408122CC7E0F8900543E06860030243
:108D50008E02E9A2E04003028E0212B8A37424122C
:108D60002CC712C9CE241C12B8A67412122CC7121A
:108D7000C895740B122CC7E0601D741C122CC7E040
:108D8000FD7406122CC7E0FC8E828F8312D33179DA
:108D900001122DA9E9703D7405122AA212313FE992
:108DA000F508740B122CC7E0702E90053DE060288A
:108DB000742255086422602074425508644270147D
:108DC0007422122CC7129747600E7422122CC712FD
:108DD000974D60047ACF802CE9A2E6506E9009127C
:108DE000E0600464017025900540E0A2E1501D742C
:108DF00022122CC712B0471228CA01010A238E0082
:108E0000028E7AD37B001242CD02972B7422122C51
:108E1000C712B04724FD600B14600824FD600424D1
:108E2000FD70DF7422122CC7129792700E742212FA
:108E30002CC712C5E2A3E0640D60107405122AA2CB
:108E4000123343E96401700302972BEE242DF5825F
:108E5000E43FF583129E247003A3E069701E750A37
:108E600000780A122A25780A122A25EE242F129851
:108E70003012975E1232837402122A34740B122C51
:108E8000C7E07003028F2912975E1233F78A0A8BAC
:108E90000BEA450B7003028FD27406122CC7E0F860
:108EA0008E828F83A3A3E028F8A3E03400F9E8249E
:108EB0000D129735F88A828B83A3A3A3E068600F15
:108EC000E88A828B83A3A3A312DBC4129798F0795C
:108ED000047406122CC712A2BBE02AF8A3E03400E7
:108EE0008882F583A3AA82AB83123C438A0C8B0D44
:108EF0008C0E8D0F850A82850B83A3A3A3A3780C08
:108F0000122983400302972B9080DC780C122BCB24
:108F1000850A82850B83A3A3A3A3E50CF0A3E50D2B
:108F2000F0A3E50EF0A3E50FF0900912E0640260F3
:108F300015E060076401600302906C900540E0A2B8
:108F4000E15003029066900555E064046008E06417
:108F500009600302972BE508A2E5400302900DEE9D
:108F6000242F12BB57C0E07402122CC7D0E0129716
:108F7000B8C0E07403122CC7D0E01297B0C0E07400
:108F800004122CC7D0E0F07416122CC7E0640170F4
:108F9000267410122CC71297537003A3E069701740
:108FA000740E122CC712D333123307E96402700710
:108FB0007416122CC7E4F01297A6122841740612F8
:108FC0002AAA7409122AA2122F597404122A3402EE
:108FD000972B90059AE064016003028F2974221296
:108FE0002CC71297477009E508A2E65003028F29A3
:108FF0007412122CC7E0F47003A3E0F4600CEEFCD2
:10900000EFFD7405122AA212314B02972BA2E650F3
:10901000527422122CC712CD687016741C122CC701
:10902000E06402703E7405122AA279001232D780E1
:10903000327422122CC712974D7014741C122CC754
:10904000E06404701E7405122AA21232CB801474DC
:1090500022122CC7129792700A79007405122AA264
:1090600012334F02972B900912E06013E064016005
:109070000302972B900540E0A2E1400302972B7476
:1090800016122CC7E0601CEE240212B603129CEDEF
:109090001412AE83129CEDC0E07416122CC7D0E0FF
:1090A000F07006E508C2E7F508E508A2E35061752F
:1090B0001110A2E25018740A122CC7E054E3F074A5
:1090C0000A122CC7E0131313541FF8E0802CA2E4FB
:1090D000502A740A122CC7E01313543F5407F86047
:1090E00009740768600B18E87007C3E508C2E7F564
:1090F00008E8333354FCF8E054E348F0740A122CC7
:10910000C7E0C0E08E828F83A3A312ADD3D0E0F07E
:10911000900555E064046008E0640960030291EC86
:10912000740E122CC712DAED7003A3E069601F748D
:109130000E122CC712D333123307E96402600F7486
:109140000A122CC7E054036401600302972B7407D2
:10915000122CC7E07041EE242F12BB57C0E07402FE
:10916000122CC7D0E01297B8C0E07403122CC7D0FD
:10917000E01297B0C0E07404122CC7D0E01297A19F
:109180001228417406122AAA7409122AA2122F590F
:109190007404122A3480527422122CC712CD6870C3
:1091A00016741C122CC7E06402703E7405122AA2C9
:1091B00079001232D780327422122CC712974D7068
:1091C00014741C122CC7E06404701E7405122AA2C9
:1091D0001232CB80147422122CC7129792700A7923
:1091E000007405122AA212334F02972B746155089E
:1091F00070030292F3E508A2E0506D12B04B7405C3
:10920000122AA21230A9E9705C12327DE9F50974C4
:1092100016122CC7E0700F7410122CC712975370DF
:1092200003A3E0696042A90912B04B7405122AA297
:109230001230AFE96024E508A2E3500C851882855E
:10924000198374FFF0A3800C740E122CC712977050
:10925000E8F0A3E9F0751004800EE508C2E5F50812
:10926000750900800353089FE508A2E5503FEE24EE
:109270002F12BB57C0E07402122CC7D0E01297B86F
:10928000C0E07403122CC7D0E01297B0C0E07404A1
:10929000122CC7D0E01297A11228417406122AAAF4
:1092A0007409122AA2122F597404122A34E508A252
:1092B000E640030295C6A818A919880A890B780AFE
:1092C000122A21A90912973E122AA21231337402DE
:1092D000122A34E9F50970030295C67422122CC7CC
:1092E00012B047640160030295C674104510F51072
:1092F0000295C67407122CC7E06401705D742212D7
:109300002CC712B0476405701EA818A919880889CF
:10931000097808122A2112973C122AA212313374BA
:1093200002122A3402972B7422122CC712979270C1
:1093300029740E122CC712D333122E4BE9601BA8CE
:1093400018A919880A890B780A122A2112973C1247
:109350002AA21231337402122A347416122CC7E076
:1093600070257407122CC7E06401700C7422122C53
:10937000C7E0F8129792600CEEFCEFFD7405122A1C
:10938000A212314B02972B1231C9E9600302972BCD
:10939000741D122CC7E070030294417420122CC774
:1093A00012B054741F122CC7E0FA741E122CC7E0BE
:1093B000F9123079E9607D741F122CC7E0701E74B9
:1093C0000E122CC712977012BC3AFAA3E0FB122EB1
:1093D000578B0BEA450B60030295C0805174201235
:1093E0002CC712D333741F122CC7E0F912307385C7
:1093F000188285198312DA277808740D122CC7E0B9
:1094000060027810740C122CC7E06004740828F80D
:10941000740A122CC7E0600108088E828F83A3A310
:10942000E028FAA3E034008A82F583E014F0751096
:10943000400295C07508007808122A25790B02951C
:1094400079740E122CC712C8917409122CC7E060EF
:1094500003029594E508A2E3500302959474071261
:109460002CC7E06401607A7900851882851983121F
:10947000D3331230CD8A0A8B0BA80AA90BE84960B6
:109480001C88828983A3A3A3A3A3E06401605288FC
:10949000828983A3A3A3A3A3E064026044EE242DE6
:1094A00012B04E85188285198312D3331233F78A8E
:1094B000828B83E5824583600FA3A3E0F912341504
:1094C000E96005C3940840197410122CC712D333F5
:1094D000122E4BE9700302956F7409122CC77404A5
:1094E000F0E4F5097809122A25741E122CC7AC8203
:1094F000AD83740F122CC712D333740A122CC7E039
:10950000F91230DF7401122A34E9600F7510208ED1
:10951000828F83A3A312B047543FF0741D122CC74F
:10952000E06023740E122CC712B054741E122CC7A4
:10953000AA82AB8312324785188285198312DA27F3
:1095400074404510F5107407122CC7E064016015D3
:1095500079007410122CC712B054740E122CC7125A
:10956000D33312307FE508A2E35037794080357558
:1095700008007808122A257902740F122CC712B03D
:10958000547411122CC712D3331233497401122AA6
:109590003402972BE508A2E340030294E1744002F1
:1095A00094E279007410122CC712B054740E122C6D
:1095B000C712D33312300DE9600674204510F51040
:1095C00012327DE9F509851882851983E064FE7001
:1095D00003A3E0F47003750900900905E0640160DD
:1095E00003029679EE241312BB57F47003A3E0F440
:1095F0007003029679740E122CC7C3E094F9A3E0AD
:1096000094FF507512B8A37410122CC7E068700351
:10961000A3E06960647410122CC712D333122E5762
:109620008A0A8B0BA80AA90BE849604D88828983B6
:10963000A3A3A3A3E06401600D88828983A3A3A3ED
:10964000A3E0640270337426122CC7740112DF9DEC
:10965000F8A3E0F97431122CC712C8957426122AA7
:10966000A2122E1BE960127429122CC7AA82AB83A6
:10967000122E69E96003123F49E508A2E7400302A0
:10968000972BE509700302972B8E828F83A3A3A3E8
:10969000A3E0FA7B00123CF18A0A8B0BEA450B70BF
:1096A0000302972BEE2404F512E43FF5138E828F0C
:1096B00083A3129780122A1D851282851383E0FCF2
:1096C0007D00123C2B7403122A347407122CC7E05D
:1096D000C0E07402122CC7D0E0F07403122CC7E46F
:1096E000F0A3F07402122A9A880C890D780C122AC1
:1096F000217810122A21E509F5087808122A251286
:10970000CA75122845851282851383E0F974071201
:109710002CC712B054AA0AAB0B12323B7407122AA0
:1097200034E96007AA0AAB0B123CF77433122A34EF
:109730007F0C0226BDF582E412E7CA22790012CA24
:109740007912B05874072212B21F64062212B22591
:1097500064072212D0F4EE241312B6206822EE24FD
:109760002BF582E43FF58312B642241312984B2264
:10977000E012977522F8A3E0F985188285198322F3
:10978000A312978A750E00780C22E0F50CA3E0F581
:109790000D2212B225640322A3E4F0A3F0A3F0A3E8
:1097A00022F01297A622EE2425F582E43FF58322CB
:1097B000F0EE243112B62022F0EE243012B6202230
:1097C00074F412242DEAFEEBFF8C088D0990090237
:1097D000E0600F12DAE07003A3E0697005122FFB5E
:1097E000804C790012D3261230CD8A828B83E58299
:1097F00045836032A3A3A3A3A3A3E054186027E585
:1098000008241C12C878122845E508241312C878C9
:10981000122845EE24181298301298351230E5744B
:1098200004122A3480087900129835123025802BD2
:1098300012B620F9228E828F83A3A3A3A3A3A3A38E
:10984000A3A312B642240B12984B22F582E43FF5F3
:109850008312E9A0FB227418122A347F040226BD69
:1098600074F012242D74EA122AC88A0A8B0BEA2497
:1098700002F50EE4350BF50F0A0AFB122E5D8A087D
:109880008B09AE08AF09750801850A82850B83A391
:10989000E0F509750C01AC0EAD0F740B122CC7AAC4
:1098A00082AB831246ED7413122CC7129B4C7415B5
:1098B000122CC77402F07408122CC7E4F09014E55F
:1098C000E0700EEE4F700AE50970067508C3029A43
:1098D000A0900555E0640860067508C2029A9C8550
:1098E0000A82850B83A3A3A3A3A3A3A3A3A3A3E09B
:1098F000A2E1500EA2E35005750C04800C750C0318
:109900008007A2E35003750C02EE4F70030299AC7E
:109910008E828F83A3A3A3A3E06404600D8E828F45
:1099200083A3A3A3A3E06403700C7404650C602CF0
:109930007403650C60268E828F83A3A3A3A3E064C7
:1099400002600D8E828F83A3A3A3A3E06401703510
:109950007402650C60067401650C701C8E828F8326
:1099600012D333123325E970438E828F8312A637C8
:10997000122CC712C89580348E828F83A3A3A3A311
:10998000E06402600D8E828F83A3A3A3A3E0640131
:10999000700A8E828F8312A79E12261EE50A240269
:1099A000FAE4350BFB122E697E007F007413122C33
:1099B000C7E064FE7003A3E0F4704E122E27E97036
:1099C00048E5096023900592E06402701B9014EC56
:1099D00012D333123325E9700F9014EC12A637120C
:1099E0002CC7E8F0A3E98020850A82850B83A3A316
:1099F000A3A3A3A3A3A3A3A3E05402F91230377433
:109A000013122CC7EAF0A3EBF07413122CC7E06416
:109A1000FE7003A3E0F470057508C7807FE509F5C3
:109A20000D780D122A25850A82850B83A3A3A3A393
:109A3000A3A3A3A3A3A3E0F9E50A2402FCE4350B46
:109A4000FD7414122CC712D333122F7D7401122A05
:109A500034E97048A90CE50A2402FCE4350BFD74D6
:109A600013122CC712D333122E398A0E8B0FAE0E5F
:109A7000AF0FEE4F601E74026509700D8E828F83EA
:109A8000A3A3A3A3A3E0D2E3F07415122CC7E4F0C0
:109A9000F50880087413122CC7129B4CE509700955
:109AA000AA18AB191247CB800AFCA90CAA18AB194B
:109AB0001232C5E9F8EE4F6053E50960208E828FBF
:109AC00083A3A3A3A3A3E0D2E6F074026509700DFB
:109AD0008E828F83A3A3A3A3A3E0D2E5F0850A829D
:109AE000850B83A3A3A3A3A3A3A3A3A3A3E0A2E69D
:109AF000500D8E828F83A3A3A3A3A3E0D2E7F08EA1
:109B0000828F83A3A3A3A3A3A3E004F0E5087003BB
:109B1000E86034FC7D007A017B101246CFEE4F6086
:109B20000CE50A2402FAE4350BFB122E69741312B9
:109B30002CC7E064FE7003A3E0F4600B7413122CD6
:109B4000C712A79E12261E741602C11D74FEF0A332
:109B500004F02274F712242D74F7122AC8EAFEEBDF
:109B6000FF900555E06403600DE064016008E06467
:109B7000096003029C7D8E828F83A3E06003029CB8
:109B8000537C007D007A027B001246CF129C828AB1
:109B9000828B8312B8AC90054612C8957953124750
:109BA000BF790090055312D333122F77900555E0FB
:109BB0006409600990055312D3331233F18518827A
:109BC000851983740112C9DF79421247BF90055588
:109BD0007404F07401122AA2794A1247B97401126E
:109BE0002AAA7A4B7B051246ED900912E0600464C4
:109BF00001701F900549E064FE7003A3E0F4602A41
:109C000079007401122AAA90054912D333122E3911
:109C10008018E06402701390054612B0547A037BFA
:109C2000001246CF12A55E1246CF900540E0A2E397
:109C30005004D2F08002C2F012C9D579521247BF47
:109C4000900912E06402703290153C12D333123145
:109C50002D80278E828F83A3AE82AF83FC7D007A16
:109C6000037B101246CF8E828F83E0F9900553124A
:109C7000D333122F77900555E4F01231997409020D
:109C8000B14CEE2402FAE43FFB22C082C08390056F
:109C90001612CB79701F900555E014600924FC6002
:109CA0000A14600C800F90051F803490051B802FD4
:109CB00090051D802AE849600890051712A2C4701B
:109CC0000C8A828B83A3E0F9122F5F801D9005160A
:109CD000129CED64027005123385800E9005D71238
:109CE000CB79600612C5E312261E02C158E0F812B5
:109CF0009CF322A3E0C82406F582E438F583E02231
:109D000074F412242D74FB122AC88A088B097A0F66
:109D10007B00123C4F8A0A8B0BAE0AAF0BEE4F70E2
:109D200003029E1F8E828F83740212C9DF79501244
:109D300047B9850882850983A3E06003029E0290EB
:109D40000553E0F47003A3E0F46044900553E0642D
:109D5000FE7003A3E0F46037851882851983129E94
:109D6000247003A3E0696027850882850983A374B2
:109D7000EAF07A467B0579531247BF7A497B057929
:109D80004B1247BF7A537B0579501247BF807385CA
:109D9000188285198312DBB112C8957A467B057942
:109DA000531247B990054612ACF712C8957A497B11
:109DB00005794B1247B97A487B0579E11247B9908A
:109DC000055AE0C3940F501D900548E0C0E07402AE
:109DD000122CC7D0E0F07404122CC77401F00412E6
:109DE0002AA21247E3750A00780A122A25780A1275
:109DF0002A25901572E0F912A9E612328374021234
:109E00002A3485088285098312D646A3F090055529
:109E10007403F0EEFAEFFB9005A0E0F9123C5B74DE
:109E20000502985812DBB5E0682274F412242D74F0
:109E3000E8122AC8EAFCEBFD8C828D83A3A3A3A3BE
:109E40007808122C707808122C02900556780812A7
:109E50002B6C7F7F7E7F79009005567808122C70DE
:109E6000E97808122A69E508A2E0502978009005EF
:109E7000A18014850882850983A3A3E06970010885
:109E8000E508241412C87812A6C170E7E8C39F50F1
:109E900004E8FFE9FE09E9C3941B40BC8C828D8372
:109EA000A3A3A3A3122CA4E8494A4B607DEC24048D
:109EB000F508E43DF509850882F583122CA4900588
:109EC00056122CB07C187D007900AA18AB19123CF0
:109ED00037850882850983122CA485188285198309
:109EE000122CB07404122CC77401F090055CE0C011
:109EF000E07405122CC7D0E0F07407122CC7E412EE
:109F0000C9DF1247D7807090055312D333122FAD9B
:109F10008A0A8B0BA80AA90B900553E8F0A3E91253
:109F2000CB86687003A3E069602D9005A112A6C1DD
:109F30006025850882850983129E247003A3E06949
:109F4000700C850882850983A3A3E06E60B9E508DB
:109F5000241412C87880D6EE900548F012317BE9BF
:109F60006015900555E4F090052112CB79600879D1
:109F7000C412C5E312261E02985674F412242D74DE
:109F8000E8122AC88A828B83A3A3A3A3A3A3A3A3B3
:109F9000A312B8ACE8FAE9FB7900900556780812EC
:109FA0002C70E97808122A69E508A2E05031EA2904
:109FB000F582E43BF583E0F89014EBE0C398501F82
:109FC000750801750900750A00750B00E97808121B
:109FD00029C17808122C029005567808122B6C09BA
:109FE000E9C3941B40B4900556122CA4E8494A4B8F
:109FF000604E7C187D007900AA18AB19123C37908E
:10A000000556122CA4851882851983122CB074046D
:10A01000122CC77401F07407122CC77401F090055C
:10A020005CE0C0E07405122CC7D0E0F07407122C7D
:10A03000C7E412C9DF1247D79005557406F0801E99
:10A04000900555E4F0FCFD7A047B101246CF900594
:10A050002112CB79600879C412C5E312261E02983A
:10A060005674F512242D74D1122AC88A088B098AD5
:10A07000828B8312B8B0741C122AAA8A828B83A3A3
:10A08000A3A3A3A3A3A312B1FB12D32E1231AB74CB
:10A090001C122CC7E0702C850882850983A3A3A31A
:10A0A000A3A3A3A3A3E0C3940B40188E828F83A322
:10A0B000A3A3A3A3A3A3A3E06402700712C863E051
:10A0C000F4600302A2B6900555E06402700302A199
:10A0D00098E06406700302A19890051612CB79608F
:10A0E0000812A2C4700302A1CD900555E064086077
:10A0F00008E06404600302A2B6741E122CC712A208
:10A10000BBA3A3A3A312B8B0900516E0F84960075B
:10A11000129CF364026077900553E06E7003A3E035
:10A120006F600302A2B674016A60167423122CC712
:10A13000AC82AD837A677B051246E7E9600302A231
:10A14000B67A007B029005A0E0F9123DC9EA4B4CBB
:10A150004D600302A2B6900556122CA48518828584
:10A160001983122CB090055CE0C0E07404122CC777
:10A17000D0E0F07405122CC77401F07406122CC7DD
:10A18000740212C9DF122EE1E9600302A2B3EEFAF3
:10A19000EFFB12337F02A2B690051612CB79702D19
:10A1A0007508007808122A257808122A25EE24104E
:10A1B000F582E43FF58312CB6DA3A3A3A3A3A3A3CE
:10A1C000A3A312ADC81232837402122A348E828F76
:10A1D0008312B8AC7407122CC7E8F0A3E912AD01E2
:10A1E00012B8AC7409122CC712C9CE240D12BB5779
:10A1F000C0E0740B122CC7D0E0F012C86312ACDAC6
:10A20000740F7808122C52740C122CC7E508F074E5
:10A2100020122CC7E0C0E0740D122CC7D0E0F074FF
:10A2200022122CC7E0C0E0740E122CC7D0E0F074EC
:10A230001D122CC7E0C0E07410122CC7D0E0F074DF
:10A240001E122CC7E0C0E0740F122CC7D0E0F0EE55
:10A25000241012BB57C0E07411122CC7D0E0F07468
:10A2600021122CC7E0C0E07412122CC7D0E0F074A9
:10A270002E122CC7E0C0E07413122CC7D0E0F0748B
:10A2800023122CC7A982AA8389088A09750A007833
:10A2900008122A1D7C087D007417122CC7AA82ABF5
:10A2A00083123C2B7403122A347407122AA2122F31
:10A2B000718003122EE7742F02EF33E0FA8E828F43
:10A2C00083A3A322129CF464012274F612242D7439
:10A2D000C9122AC89005D112CB79600612C5E312C3
:10A2E000261E900555E06408700302A3879005922E
:10A2F000E064027023904FE1E493900537F0904FB3
:10A30000E1E493900535F090055E7401F0129798A2
:10A3100004F0A3E4F0A3806C900566E0F8740B28C9
:10A32000F582E4340EF583E0FA900537F0740C28DA
:10A33000F582E4340EF583E0F9900535F07508FFF9
:10A340007509FFEA7808122BDEE508F4FCE509F44C
:10A35000FD3395E0FE90055EECF0A3EDF0A3EEF08A
:10A36000A3F07508FF7509FFE9C39A7808122BDE80
:10A37000E508F4FCE509F4FD3395E0FEA3ECF0A359
:10A38000EDF0A3EEF0A3F07C237D007900741412AD
:10A390002AA2123C37900566E07009741E122CC781
:10A3A00074018006741E122CC7E412A4CC740FF042
:10A3B0009014EA12C9DF79461247BF7401122CC704
:10A3C000E4F090154BE0C0E07402122CC7D0E0F02E
:10A3D000900543E0C0E07403122CC7D0E0F0740491
:10A3E000122CC7E4F07405122CC7E4F07407122C89
:10A3F000C7E4F0900566E0C3940F500CE0C0E07431
:10A4000006122CC7D0E080077406122CC7740FF018
:10A410007C677D057408122CC7AA82AB831246EDB7
:10A420007C037D0079FF7410122CC7AA82AB8312C3
:10A430003C3790059FE0C0E07413122CC7D0E012A7
:10A44000C7D77401122AA21231A57AA37B057945D8
:10A450001247BF1232B390055AE0C0E0741C122CB0
:10A46000C7D0E0F090055BE0C0E0741D122CC7D0AF
:10A47000E0F0900548E0C0E0741A122CC7D0E0125A
:10A4800084957418122CC712C8957420122CC7E436
:10A49000F090055DE0C0E0741F122CC7D0E0F074AE
:10A4A00034122CC7E4F07429122CC7E4F07A467BEE
:10A4B0000579531247BF7A497B05794B1247BF7420
:10A4C00014122AA21247DD743702C4C912A4D02282
:10A4D000F085188285198322C082C0838A828B838B
:10A4E000A3E09005556004E4F080707408F09005D6
:10A4F00066E0702890052112CB796008790012C5BA
:10A50000E312261E90055312B0547A057B001246C2
:10A51000CF90055312D3331233F180187900122FE4
:10A520006B90054612B0547A067B001246CF12A5F6
:10A530005E1246CF9005DD12CB79601F900906E0D0
:10A54000640170179080CC1228417A007B409005FE
:10A55000A0E0F9123DB77404122A3402C1589005E4
:10A560004912B0587A047B002274F412242D74EA44
:10A57000122AC8EAFEEBFF129C82122E5D8A088B1B
:10A5800009EA4509700302A6328A828B83A3A3A33A
:10A59000A3E0640160278A828B83A3A3A3A3E06462
:10A5A00002601A8A828B83A3A3A3A3E06403600DD5
:10A5B0008A828B83A3A3A3A3E064047075EE2402B4
:10A5C000FCE43FFD740B122CC7AA82AB831246ED4C
:10A5D00085088285098312A637122CC712C8957484
:10A5E00015122CC77401F07408122CC7E412C9DFCD
:10A5F0001247D1890AAC0A7D007A077B001246CF48
:10A60000850882850983A3A3A3A3A3E0C2E012C0A7
:10A61000C4A3A3740112E2895001097A027B0012DB
:10A620002246E8850882850983A3A3A3A3A3A3A345
:10A63000A3F0741602985812D0F474132274F21214
:10A64000242D74F8122AC8EAFEEBFF8C0A8D0B89C0
:10A650000C908062AC18AD197408122962F50DEEE9
:10A66000FCEFFDAA18AB191246E7E97003750D015E
:10A670009005A1801AEEFCEFFDE508240BFAE43505
:10A6800009FB1246E7E97023E508241412C8781282
:10A69000A6C16024E50DA2E040DB85088285098320
:10A6A000E0650A7004A3E0650B70DD85088285090A
:10A6B00083A3A3E0650C70D0AA08AB09740802D18B
:10A6C0000212ACDEE508450922C082C0839005A1D4
:10A6D00002C15574F712242D9005A112E9A0800C37
:10A6E00012D3BF12B8B3123CF7EEFAEFFBEA4B708D
:10A6F000EF9005A1E4F0A3F002B14F74F412242D01
:10A70000EAFEEBFFEE241312BB576403700CEE2439
:10A710000BFAE43FFB122E5D800EE06402707C12A7
:10A72000C86312D333122E578A088B09E5084509EE
:10A7300060698E828F83A3E0700F8508828509830C
:10A74000A3A3A3A3A3A3E4805164F1600A8E828F24
:10A7500083A3E064E17027850882850983A3A3A30E
:10A76000A3A3A3E06401701685088285098312A75C
:10A770009E12261EEE240BFAE43FFB122E6985087A
:10A7800082850983A3A3A3A3A3A3E0600E85088207
:10A79000850983A3A3A3A3A3A314F002985B129833
:10A7A0005190052F12C8A92274F112242D8A088B0A
:10A7B00009ECFEEDFF890A12D633EEF8EFF9A30E8D
:10A7C000AF838A828B83A3A3E0C454F0FA88828982
:10A7D00083E04A12A88912D64712A884E033335482
:10A7E000FCF88E828F83E04812A884A3E0333333D1
:10A7F00054F8F88E828F83E048F0EEF8EFF9A30E5C
:10A80000AF838508828B83A3A3A3A3A3A3E0A2E0C5
:10A81000E4331313FA88828983E04AF0E5082407B9
:10A82000F50CE43509F50D750E00780C122A1D7C27
:10A83000087D00EEFAEFFB123C2B7403122A34EE73
:10A840002408FE50010FE508240FF50CE43509F546
:10A850000D780C122A1D7C037D00EEFAEFFB123CF2
:10A860002B7403122A34E50AC3940F4012E508241E
:10A8700012F582E412DEBD8E828F83A3A3A3F07F44
:10A88000070226BD12A889A322F08508828B83A324
:10A89000A3A32274F112242DEAFEEBFF890A8C088F
:10A8A0008D098E828F83E08C828D8312B652AE82A8
:10A8B000AF83E012BEF212C0E0C412BEF212A95D74
:10A8C000E054038C828D8312C0DEA2E2E4338C82DA
:10A8D0008D8312C0DD131313541F12BEF212C0DC9D
:10A8E000A2E7E4338C828D83A3A3A3A312A95D8E78
:10A8F0000C8F0D750E00780C122A1D7C087D00E56A
:10A90000082407FAE43509FB123C2B7403122A349D
:10A91000EE2408FE50010F8E0C8F0D780C122A1DAC
:10A920007C037D00E508240FFAE43509FB123C2B7B
:10A930007403122A34E50AC3940F40158E828F8364
:10A94000A3A3A3E0C0E0E508241212C878D0E080F9
:10A9500008E508241212C878E4F002A87FA3A31225
:10A96000B6560EAF832274F512242D8A088B098AFD
:10A97000828B83A3AE82AF83E0F9122F958E828FF4
:10A9800083E064EB6024850882850983A3E064E1A9
:10A990006018850882850983A3E064F1600C85084E
:10A9A00082850983A3E0641A70098508828509837A
:10A9B000A3E4F090153C12D33312312D750A0178BF
:10A9C0000A122A25850882850983A3E0F5087808FC
:10A9D000122A25790012A9E61232837402122A344F
:10A9E0001231C302EF3690055312B0589005491248
:10A9F000985122C082C083E99005B37003E48002BD
:10AA000074018065E0F902C15874F712242DEAFE42
:10AA1000EBFF8E828F8312C9A712DA0C12DA27128B
:10AA20003307E98E828F83600512AA3A800312AA47
:10AA30004F12AA581247EF02B14F12AA41E4F0A3F5
:10AA400022E0F8A3E0C8240DF582E438F583221251
:10AA5000AA417401F0A3E422F07C1B7D318E828F29
:10AA60008312985122EAF0A3EBF002C15874F61257
:10AA7000242D9005B3E0701B7C0079017A007B00E7
:10AA80001231F3EA4B600C8A828B8312CB7960031C
:10AA900012312102C4CCC082C08379041231EDE9A5
:10AAA000F8904FEEE493C398401079FF1231EDE92E
:10AAB000F8904FEDE493C398500479018002790037
:10AAC00002C15874F012242D8A088B09890B750C69
:10AAD000008A828B83A3A3A3A3A3A3A3A3E0F91259
:10AAE00031F98A0E8B0FAE0EAF0F750A01EE4F6073
:10AAF0000302AB9385088285098312ACE6A3A3A366
:10AB0000A3A3A312BC2C12D3331231E18A0C8B0DF8
:10AB1000AE0CAF0DEE4F700302ACCC8E828F83A3D0
:10AB2000A3A3A3E4F0A3F0E508240CFAE43509FBA1
:10AB30008A828B83E0C0E012E27FD0E0F012331310
:10AB4000EE240D12DA21E50812DEAF350912B8AA9B
:10AB500012B61412C895750C01EE240612BB5B5494
:10AB60007FF0A3E054FC12E6805404600302AC0AB8
:10AB7000901544E0F50875090074077808122BDE7B
:10AB80008E828F83A3A3A3A3A3A3E04508F0A3E031
:10AB90004509F08E828F83A3A3A3A312ACD87407B8
:10ABA0007808122C52E5085407F508E50B606B8E07
:10ABB000828F83A3A3A3A3A3A3A3A3A3740212C0FE
:10ABC000E112AFC3600B90054112ACF7A3A312C80A
:10ABD00095E508700302AC98EE240612EDB8547F98
:10ABE000FCA3E054FCFDE50824FFF508E434FFF580
:10ABF0000974077808122BDEEC4508F8ED4509F9D1
:10AC00008A828B8312C89502AC988E828F83A3A30D
:10AC1000A3A3A3A3E0448002AB92E5087005750AE4
:10AC20000080758E828F83A3A3A3A3A3A3E05420E7
:10AC3000600C123C49EA547F7900245F80198E82AF
:10AC40008F83A3A3A3A3A3A3E05410601A123C49CB
:10AC5000EA540F7900240A5001098E828F83A3A33E
:10AC6000A3A3F0A3E9800D8E828F83A3A3A3A37473
:10AC700001F0A3E412AD017404F07A207B0090058A
:10AC8000A0E0F9123DC9EA4B4C4D700C7A207B00D4
:10AC90009005A0E0F9123C91E50CA2E050318E82C3
:10ACA0008F83A3A3A3A312D337F9EEFAEFFB1231DC
:10ACB000E7E9601B12B14412CB77600912B233127C
:10ACC000D333123CF7EEFAEFFB123CF7750A00A9FA
:10ACD0000A02C1208E828F83A3A312ACDE22E0F58C
:10ACE00008A3E0F50922A3A3A3A3A3A312B0588548
:10ACF0000882850983A32212D0F48E828F83A3A3B6
:10AD00002212C885A3A3A32274F412242D74F7126F
:10AD10002AC87E001231F9EA4B700302ADC18A8263
:10AD20008B83A3A3A3A3A3A3A3A3A3E064066003AD
:10AD300002ADC18A828B83A3A3A3A3A3A3A3E0FF35
:10AD40008A828B8312ADD3E0C0E07408122CC7D086
:10AD5000E012B21812C892123217EF5408606085E0
:10AD6000188285198312B0547A007B001231DB8B74
:10AD70000BEA450B704912EF2D1248077C007D004D
:10AD80007A007B0080258E828F8312B047F4700397
:10AD9000A3E0F4602A90055312ADC8124801E9649B
:10ADA0001A601C7C007D00EEFAEFFB1231DB8A0A90
:10ADB0008B0BAE0AAF0BEE4F70CC790012480D7EB4
:10ADC00001EEF9740902985812B0588E828F8312DE
:10ADD00098512212B89E12ADDA222408F582E43886
:10ADE000F58322C082C083EA4B70059005B48006CB
:10ADF0008A828B83A3A312AFF760258A828B83A3F9
:10AE0000A3A3A3A3A3A3E0540860E5EC4D60158AB7
:10AE1000828B8312B0476C7003A3E06D70D2800404
:10AE20007A007B0002C15874F212242DEAFEEBFF77
:10AE3000890A8C088D097A117B00123CF1EA4B607B
:10AE40003E8A828B83A3A3A3A3A3A3A3A3A3E412F9
:10AE5000B20CA3E50A12DBC4A3A3A312F00E8A82EC
:10AE60008B83A3A3A3A3E4F0A312B22D12AE8D1281
:10AE7000DA1412B722E4F012AE82A3A3F0A3F00218
:10AE8000D105A312AE8722F08A828B8322A3F0120F
:10AE9000EDE43BF583E4F02274F412242DEAFEEB9A
:10AEA000FF89088C0A8D0BEE4F700302AF4C7401C2
:10AEB0006508701279011231EDE9F8904FF3E493CF
:10AEC000C3985022801674046508701479041231F6
:10AED000EDE9F8904FEEE493C398500A7911806E33
:10AEE0007402650870668E828F83A3A3A3A3A3A3B5
:10AEF000A3A3A3E50812BE5D12D62B8E828F83A377
:10AF0000A3E4F0A3F09005B412CB7960178003E0BE
:10AF1000F8A312C9AEA3A312AFF788828983A3A3B3
:10AF200070ED80039005B412DA187A207B0090054A
:10AF3000A0E0F9123DC9EA4B4C4D700C7A207B0021
:10AF40009005A0E0F9123C917900800279C1029845
:10AF50005BC082C083E9F879009005B4801D8A82C5
:10AF60008B83A3A3A3A3A3A3A3A3A3E068600574F7
:10AF7000FF687001098A828B83A3A312AFF770DE8A
:10AF800002C15874F712242DEA4B70059005B48065
:10AF9000068A828B83A3A312AFF760208A828B83F9
:10AFA000A3A3A3A3A3A3A3A3A3E06970E4EC6010ED
:10AFB0008A828B83E012AFC370D780047A007B0053
:10AFC00002B14F12AA42E0540422C082C08390050D
:10AFD000B480068A828B83A3A312AFF760128A82A1
:10AFE0008B83A3A3A3A3A3A3A3A3E06970E5800419
:10AFF0007A007B0002C158129851EA4B2274F71272
:10B00000242DEAFCEBFD9005B480068A828B83A395
:10B01000A312AFF760218A828B8312B0476C700352
:10B02000A3E06D70E68A828B8312862212CA94A2F4
:10B03000E0E43370D680047A007B0002B14FEE2446
:10B040001DF582E43FF58312B21F22EE2413F58230
:10B05000E43FF58312B0582212B05C22E0FCA3E07A
:10B06000FD2274F212242D8A0A8B0B8C0C8D0D7527
:10B070000800750900EA450B60309005B480068E23
:10B08000828F83A3A312B8B3EE4F601EAC0CAD0D3C
:10B09000EEFAEFFB850A82850B8312261EE9640116
:10B0A00070DDEEF8EFF988088909AA08AB0902D12A
:10B0B0000579000229E674F712242D9005B412B820
:10B0C000AC7C007D00800DE8FCE9FD88828983A3CB
:10B0D000A312B8ACE8496030EA687002EB6970E727
:10B0E0009005B412D333E86A7002E96B88828983D1
:10B0F000A3A3700812B8AC9005B4800912B8AC8C48
:10B10000828D83A3A312C895804574F712242DEA7B
:10B11000FEEBFFEE4F602B12321112B239123CF7E8
:10B120008E828F8312D333123CF712B14412CB7745
:10B13000600912B23312D333123CF7EEFAEFFB126E
:10B140003CF7800BEE240DF582E43F22122A347F77
:10B15000010226BD74F712242D8A828B8312B20459
:10B160009005B412B8AC7508007E008033888289DF
:10B1700083A3A3A3A3A3A3A3A3A3E0640570180EB2
:10B1800088828983E0FFA3E0F5838F82E06C7003FF
:10B19000A3E06D7002050888828983A3A312B8AC6E
:10B1A000E84970C9904FEA12E3D45008904FE61274
:10B1B000D274400F8A828B83A3A3A3A37401F0A34C
:10B1C000E4800C900541E0F812B1FBE8F0A3E9122D
:10B1D000B22D740512B20CE0440812B218F47003D8
:10B1E000A3E0F4600E90055312D52E124801E964D5
:10B1F0001A7005790112480D02B14FA312B5FCA3D4
:10B20000A3A3A32212B21FFCA3E0FD2212B21022BC
:10B2100012DBCCA3A3A3A32212AE8712B21F22E09B
:10B22000F812B22522A3E0F5838882E02212B21040
:10B23000A3A32212B144F5832212B24012984F22E6
:10B240008E828F83E0F8A3E0C8241FF582E43822C1
:10B25000C082C083EAFCEBFDEC4D6017EC24FBF5EB
:10B2600082ED34FF12CB77700712B2AAE0F46007C8
:10B27000123C55790580309005A0E0C0E012B2AADA
:10B28000D0E0F0904FDEE493F97AB67B05123C8B68
:10B29000E9640170107A007B209005A0E0F9123C6F
:10B2A0009179008002790402C158EC24FFF582ED07
:10B2B00034FFF5832274F412242DA2AFE433F50891
:10B2C000C2AF9005B612B8B3EE4F603AEE24FBF56C
:10B2D00082EF34FF12CB777A007B209005A06007C5
:10B2E000E0F9123C918005E0F9123C97E4F50AF58B
:10B2F0000B780A122A21EEFCEFFD7AB67B05123C90
:10B30000857402122A34E508A2E092AFEEFAEFFB50
:10B3100002985B74F012242D74DB122AC8EAFEEB4B
:10B32000FF750B00750A007508FE7509FF1231C91B
:10B33000E9600302B5EFEE241512BB576046901585
:10B340005FE0C43354E0F8E0333354FC48C0E0120B
:10B35000D318D0E012B65212D33279FF122D1F8BC0
:10B360000DEA450D6011750B017508FF12B6194401
:10B370000412C8B2D2E0F0900912E06004640170D7
:10B3800003750A408E828F8312D331123307E9602E
:10B390000312C985EE241312BB57700D904FE9E4D8
:10B3A00093C0E012CA75D0E0F08E828F83E0A2E7EE
:10B3B000500454038019EE241412BB5770129005E8
:10B3C00032E0C0E012ED96D0E0F0900532E004F0FB
:10B3D00012EDAF701990154DE0600D90053DE070D5
:10B3E0000D8E828F83E07006EE241112C9889009B9
:10B3F00012E0600464017048900540E0A2E1504012
:10B40000E50BA2E040218E828F8312D331123307E5
:10B41000E9602D8E828F83E0600DEE240B12B04127
:10B42000F91232E3E9601912B628700302B5A0EEF2
:10B43000241312EDB2600302B5A012B61954FBF04A
:10B440008E828F83E06401700DEE240B12B0416494
:10B4500002700312B63512B628600302B519E50B67
:10B46000A2E0500302B519900912E0600764016080
:10B470000302B519900540E0A2E1400302B519E5C9
:10B480000AF50B780B122A25EE2406FCE43FFD8E0C
:10B49000828F8312D331EE24121298301230DF746F
:10B4A00001122A34E9600612C98512B62E8E828FE7
:10B4B00083A3A3A3A3A3A3E0603CEE2402F50CE4C2
:10B4C0003FF50D850C8212B63C2407FAE43FFB12CF
:10B4D00032478A088B09850C82850D83E0650870E8
:10B4E00004A3E06509700C8E828F83A3A3A3A3A39A
:10B4F000A3E4F012B6358E828F83E064016008A960
:10B500000A12B64712307FA90A8E828F8312B6477D
:10B5100012300DE9600312B62EAC18AD19EEFAEF39
:10B52000FB1232418A0A8B0B74FE6508700474FFAB
:10B530006509700312ACD4EA450B700302B5F38EB3
:10B54000828F83E0C0E07401122CC7D0E0F0740257
:10B55000122CC712DA187401122A9A880C890D78F5
:10B560000C122A2112B614122845EE240E12BB57D3
:10B57000F50C780C122A25900546122845740712FE
:10B580002CC7E0F9AC08AD0912323B7407122A341B
:10B59000E9FE74106E705EAA0AAB0B123CF7805580
:10B5A000EE241312BB57C0E07415122CC7D0E01262
:10B5B000EE13740D122CC712C9CE240412B6031256
:10B5C000B8AC740F122CC712C9CE241412BB57C0CA
:10B5D000E07416122CC7D0E012E27512B5FC12B05E
:10B5E000547404122AA21230AFE9600302B4407905
:10B5F0001180047E10EEF9742502C11DE0F98A82E3
:10B600008B832212B60722F8E43FF9E8FAE9FB8AB5
:10B61000828B8322EE12C99A2212B61D22EE240FCB
:10B62000F582E43FF583E02212B61D54402212B6A3
:10B630001D4420F02212B61D4440F022F58312B6BC
:10B64000422212B05CEE22A3A3A3A312D34312980A
:10B65000512212B65622F08E828F83A322C082C05E
:10B660008374DC122AC88A828B83A3A3A3A312B893
:10B67000AC740E122CC7E8F0A3E912D0EB740C12D4
:10B680002CC712C89512B722E0C0E0741A122CC75A
:10B69000D0E0F012B72C3B12B8AA7420122CC712BB
:10B6A000C895EA12D3203BF583E0C0E07408122C61
:10B6B000C7D0E0F0EA241CF582E43B12B8AA741269
:10B6C000122CC712C895EA2411F582E43BF583E0F9
:10B6D000C0E07409122CC7D0E0F0EA2412F582E42D
:10B6E0003BF583E0C0E07407122CC7D0E012A4CC75
:10B6F00074FFF07401122CC774FFF07402122CC78F
:10B7000074FFF09080D01228417404122AAA7407A2
:10B71000122AA2122F597404122A347900742402B6
:10B72000849FEA240DF582E43BF58322EA12EDE5DD
:10B730002274EE12242D74EF122AC88A0E8B0F8CFD
:10B74000088D09890C750A107A217B00123CF112D0
:10B75000D14BE849700302B897750B007C217D003E
:10B760007900851882851983E0FA123C3774261215
:10B770002CC712B8B3900912E060046401703EAAAD
:10B7800008AB09122E578A108B11A810A911E8498D
:10B79000602388828983A3A3A3A3E06401600D884A
:10B7A000828983A3A3A3A3E064037009EE544070CD
:10B7B0000474044FFFEF54046003750B01900553AC
:10B7C00012D33385188285198312B89E2409F58215
:10B7D000E43812DA257423122CC712B8AC740F1295
:10B7E0002CC7E8F0A3E912B8B912EDDB12B8B91210
:10B7F000ADDA740212BC3612C5E1E508F0A3E50922
:10B8000012B8B912EDA6E50CF07425122CC7E0F5BC
:10B810000885188285198312EDEBE50812B8B92462
:10B820001FF582E438F583E50EF0A3E50FF074060A
:10B83000122CC712DA187408122CC7E508F0742805
:10B84000122CC712C5E0C082C083740C122CC7AC86
:10B8500082AD83D083D0827403122962A90BAA1807
:10B86000AB191231CFE964017021900912E0600434
:10B8700064017012E50BA2E0500CA9081231F9EA3C
:10B880004B600312321D750A00800C8518828519E1
:10B890008312D333123CF7A90A741102BE6A12D084
:10B8A000F9C822EE2413F582E43FF58312D0F42286
:10B8B000A3A3A3E0FEA3E0FF2212D15AC82274EE94
:10B8C00012242DEAFEEBFF8C088D098E828F83A354
:10B8D000740812C9C1E060088E828F83A37410F0CF
:10B8E00012BB5460098E828F83A3E02408F0EE24FB
:10B8F0001512BB5760088E828F83A3E004F08E82FE
:10B900008F83A3A3A3A3A3A3E060198E828F83A335
:10B91000A3A3A3A3A3A3E0C3332402F88E828F833F
:10B92000A3E028F0EE241112BB576005750B0E80C2
:10B9300003750B008E828F83A3E0F8EE240D12BBFB
:10B940005728250B8C828D83F0EE241112BB576093
:10B950001190053EE0F9122DAF850882850983E03C
:10B9600029F0850882850983E0C39475400975082C
:10B970000075090002BB4DE0FA7B00123CF18A0819
:10B980008B09EA4509700302BB4D8E828F83E0FA72
:10B9900090054312BB657402780C122BDEEA450C4D
:10B9A000FAAB0DEE241212BB575403F50C750D00C3
:10B9B0007406780C122BDEEA450CFCEBFDEE241528
:10B9C00012BB576004780180027800EE2416FAE476
:10B9D0003FFBE8F9ED49FDEE241112BB57F50C745D
:10B9E00009780C122BDEED450DFD8A828B8312BB8C
:10B9F00065740B780C122BDEED450DFD12BE3A126C
:10BA0000BB65740C780C122BDEED450DFD8E828F1C
:10BA100083A3A3A3A3A3A312BB65740A780C122B60
:10BA2000DEECF8ED450DF9E8850882850983F0E93B
:10BA3000A3F0EE240212BB5B85088285098312BB4A
:10BA400089F0EE2404F8E43FF98882898312C08BE0
:10BA5000A312BB89A3A3F0EE241312BB6CF0EE2457
:10BA60001412BB6CA3F0750A088A828B83E0601500
:10BA7000EE241812B04EE5082408FAE43509FB124A
:10BA800046ED750A1012BB54601BEE241A12B04E1C
:10BA9000850A0CE508250CFAE43509FB1246ED741D
:10BAA00008250AF50A8E828F83A3A3A3A3A3A3E08C
:10BAB0006058EE2407F510E43FF511851082F583F8
:10BAC000E0C0E012C871D0E012BB79E0C0E012C85B
:10BAD00071D0E012BB79129780122A1D85108285E1
:10BAE0001183E025E0FCE433FD850A0CE508250C14
:10BAF000FAE43509FB123C2B7403122A34851082B8
:10BB0000851183E0C333250AF50AEE241512BB57CD
:10BB10006008C0E012C871D0E0F012C863129781CB
:10BB2000122A1DEE240D12BB57FC7D00850B0A8ED8
:10BB3000828F83A3E0F8E50828F8E43509F9E825C1
:10BB40000AFAE439FB123C2B7403122A34AA08AB1C
:10BB50000902BE6DEE241712B62022F8E43FF988E0
:10BB6000828983E022E0F50C750D0022F582E43F26
:10BB7000F58312BB92A3A3A322F0050A8E828F83C2
:10BB8000A3A3A3A3A3A3A3A322A3A312DFA312BBD4
:10BB9000922212C08FA3A32274F412242D74FD12DA
:10BBA0002AC88A088B09ECFEEDFF7401122A9A88D4
:10BBB0000A890B780A122A217402122AAAEEFAEFD5
:10BBC000FB12305B7402122A34E9705785188285A3
:10BBD0001983E0850882850983F07401122CC7E07F
:10BBE000F812BC2CA3A312BC3A60291485088285E4
:10BBF0000983A312BC3612D70C7401122CC7E0289B
:10BC0000F8A3E039F9E824FEF582E934FFF5831260
:10BC1000E9A0800C850882850983A3E4F0EEFAEFA1
:10BC2000FB80047AFE7BFF7403029858A3E0F98539
:10BC300008828509832212BC4222E8F0A3E912BCE3
:10BC4000422212BC462212A4D0E02274EE12242D0D
:10BC50008A0A8B0BECFEEDFF750F01E9C3940850C7
:10BC60000302BDD28E828F83E912AE8312C0B61258
:10BC70003253E96003750F0012C0988E828F8312D1
:10BC8000C0E8EE12B72D3F12C0D2C0E0EE2411F58D
:10BC900082E43FF583D0E012C0CAC0E0EE2412F582
:10BCA00082E43FF583D0E012B652740812BE5DA361
:10BCB000A3A3E06018E50A2408F8E4350BF912CADA
:10BCC0007512C8958E828F83A3E02408F08E828F30
:10BCD00083A3A3A3A3A3A3A3A3E0601C8E828F834B
:10BCE000A385820885830912C0ABEE241512E257A2
:10BCF000A3E912CB862408F08E828F83A3A3A3A38B
:10BD0000A3E0600F12BE448E828F83A3A3A3A3A3DC
:10BD100012BE64EE241912C988EE241B12C988A32E
:10BD2000F0EE241812BB57700302BDC212BE44FAD3
:10BD3000EE2419F582E43FF583EA12BE64F8E50AC1
:10BD400028F582E412E24EF812CB8AE812BE64E8CB
:10BD5000C39AEE5068241912BB57F8904FDDE49354
:10BD6000C398500575110C8008EE241912BB57F5C5
:10BD7000118E828F83A3E0F8E50A28F50CE4350BD9
:10BD8000F50D750E00780C122A1DAC11EC2CFCE49C
:10BD900033FD7AAB7B12123C2B7403122A34EE244F
:10BDA0001BF582E43FF58374ABF0A37412F0E51148
:10BDB000C333F8850882850983E028800412C9818D
:10BDC000E4F08E828F83A3E0F88E828F83E0C398A5
:10BDD000500479008062A3E0FAE50A28F8E4350B04
:10BDE000F9EE241D12E257A3E912C0E1C39AC0E0A4
:10BDF00012BE3AD0E012C880603CEE2417F8E43F4F
:10BE0000F9880889098882F583E024F2F0EE241D80
:10BE100012BB5B240EFAA3E03400FB8882898312F4
:10BE2000DA2790053EE0F9122DAFE9F88508828502
:10BE30000983E0C398F0A90F8033EE2417F582E45C
:10BE40003FF583228E828F83A3858208858309E054
:10BE5000F8E50A28F582E4350BF583E02212B656A0
:10BE6000A3A3A32212CB9404F022122A347F0A0245
:10BE700026BD74F412242D8A088B09EA12BEF9F04B
:10BE8000EA1313543F12BEF2A3A3A3F0EAC41313A0
:10BE900012BEF9A3A3F0EB12BF0412BF0C74097811
:10BEA0000A122C5212BF0212BF0B740A780A122C0B
:10BEB00052E50A5401C0E0EC2418F582E43DF58314
:10BEC000D0E012BF11740B780A122C5212BF02A3D9
:10BED00012BF0B740C780A122C5212BF02A3A3A338
:10BEE000A3A3A3A3A3F0740D7808122C52A90802EF
:10BEF000985B540F8C828D832254038C828D83A394
:10BF0000A322E50A54018C828D8322A3A3A3A3A3B9
:10BF1000A3F08A0A8B0B22C082C08379008A828BAD
:10BF200083A3A3A3A3A3A3E090053D600EE070222A
:10BF30008A828B83A3A3E070198016E060148A8242
:10BF40008B8312D32A900546E06A7003A3E06B60EE
:10BF5000010902C15874F012242D8A0A8B0B890C36
:10BF60008C088D098A828B8312C0B612325312C09C
:10BF70009885088285098312C0E8E50812B72D3537
:10BF80000912C0D2C0E0E508241112C878D0E0122E
:10BF9000C0CAC0E0E508241212C878D0E012EE3E14
:10BFA000740812C0C4E0601EE50A2408F8E4350BEA
:10BFB000F9E508241312C87812C895850882850906
:10BFC00083A3E02408F0850882850983A3A3A3A3A3
:10BFD000A3A3A3A3E0601B850882850983A312C0E5
:10BFE000A7E508241512C878E8F0A3E912C0E124F7
:10BFF00008F0850882850983A3A3A3A3A3E06019A1
:10C00000850882850983A3AE82AF8312BE4F85085F
:10C010008285098312C0DC04F0AA08AB09123259E8
:10C02000E9F50D7061850882850983A3A3A3A3A305
:10C03000A312C08B701AE0FAE50A2AF8E4350BF96E
:10C04000E508241D12C87812C895E50CC39A802A09
:10C0500012C0A7E8240EF8500109E508241D12C8F3
:10C060007812C89590053EE0F9122DAF8E828F832D
:10C07000E0F8E50CC39824F2C399C0E0E508241762
:10C0800012C878D0E0F0A90D02C12012C08F22E0C2
:10C09000850882850983A322850A82850B83A3A351
:10C0A00012C0FEE0F9EA22AE82AF83E0F8E50A288A
:10C0B000F8E4350BF922E0FAA3E0F8E4C8F9EA283D
:10C0C000E439FB2212EE21A3A32212C111A3A3A3E0
:10C0D000E022F583E812C10AA3A3E022A3A3A3A34D
:10C0E000A3F08E828F83E022A3A3A3A3A3A3A3A381
:10C0F000A312C10A12C0FEA3A3E0F9EAF822E0FAF3
:10C10000850A82850B83A3A3A322F0A3E912C111A0
:10C1100022F0850A82850B83A3A3A3A322122A34CB
:10C120007F080226BDC082C0837AC47B0579E212F3
:10C1300047B97AC47B058020C082C08390054680C1
:10C1400014C082C083900549800BC082C083794AA5
:10C150001247B9800312D333D083D0820229E67408
:10C16000F612242D9005CCE0FE04F0EEF91231F920
:10C170008B09EA450970EDEE60EAF902C4CC74EE71
:10C1800012242DEAFEEBFF8C0E8D0F890A750B0031
:10C19000750C001233F78A088B097412122CC7E051
:10C1A000F5107413122CC7E0F50DEA45097017E578
:10C1B0000D600302C2A2A90AAC0EAD0FEEFAEFFBAE
:10C1C00012341B02C3B0E50D700302C2689009125D
:10C1D000E060046401700E9005D912CB79600612FC
:10C1E000C5E312261EE510700B850882850983E4DD
:10C1F000F002C29D900912E060076401600302C270
:10C20000C5900540E0A2E1400302C2C59005DB12E3
:10C21000CB79600CA910AA08AB0912C5E312261E3F
:10C22000850882850983E0FA12E26A500109C3EAAF
:10C2300098E499A2D265D033500985088285098394
:10C24000E004F0850882850983E0F8904FF4E493D8
:10C25000687072750B01EEFAEFFB1230EB85088205
:10C26000850983A3E4F0805DE5107021EA2402F5DE
:10C2700082E412DEBD850A0E250EF8E4340013E8D0
:10C2800013F070098A828B83A3A37401F08A828BD6
:10C2900083A3A3E0F8901572E0C3985028750C01B1
:10C2A00080237401650D701DE5106019900912E07E
:10C2B00060046401700F900540E0A2E15007EEFABF
:10C2C000EFFB1230EB900912E06402600FE06004B3
:10C2D0006401702A900540E0A2E140227401650DDE
:10C2E000701CE5109005EB6013E004F0901545E03C
:10C2F000F89005EBE0C3984005750B01E4F0E50C00
:10C30000A2E092F0E50BA2E072F0400302C3B0900D
:10C310000912E0600464017041900540E0A2E15020
:10C3200039EEFAEFFB122E578A088B09A808A909E3
:10C33000E8496026E50CA2E0500D88828983A3A31A
:10C34000A3A3A3E0C2E0F0E50BA2E05063888289DA
:10C3500083A3A3A3A3A3E0D2E0F0E50BA2E0505097
:10C36000900912E060046401701D900540E0A2E1B4
:10C370005015EEFAEFFB122E45E9600BEEFAEFFBDB
:10C380007900122F8F8029900549E06E7003A3E099
:10C390006F701DEEFAEFFB7901122F8F900912E0FA
:10C3A0006402700C7A017B009005A0E0F9123DC395
:10C3B00002BE6D74F412242D74016A4B700E7A0162
:10C3C0007B009005A0E0F9123C91803790153C125B
:10C3D000DA27EA4B60218A088B09E4F50AF50B7825
:10C3E00008122A197A017B009005A0E0F9123DB7E6
:10C3F0007404122A34800C7A017B009005A0E0F9C5
:10C40000123DC302985BC082C08390153E02AA65AC
:10C41000C082C08390154002AA6574F612242D755F
:10C4200008327509057808122A217C6E7D007A2170
:10C430007B00123D697402122A34E9F508122DD3EB
:10C44000E94208900912E0600464017006122E812E
:10C45000E9420890070F12CB79600912C5E3122652
:10C460001EE94208122D43E9FE124273E9F8E5087D
:10C470004E48F9805774F612242D1246C9750832B9
:10C480007509057808122A2175086E750900780863
:10C49000122A217C007D007A217B00123D757404F4
:10C4A000122A34122DD9900912E06004640170033D
:10C4B000122E8790071112CB79600612C5E312265F
:10C4C0001E122D4912427F8003122A347F02022657
:10C4D000BD74F612242D74FF122AC87E007508322E
:10C4E0007509057808122A217C6E7D007A217B006F
:10C4F000123D697402122A34E9600302C5B4780857
:10C50000122A2175086E8E097808122A217C007D76
:10C51000007A217B00123D7B7404122A34E9600307
:10C5200002C5B4900546E064FE7003A3E0F4700316
:10C5300002C5B40E900555E064086005E06404701F
:10C540006F851882851983EE12C9DF79421247BFC1
:10C550007A5D7B0579431247BF7A5A7B057947128A
:10C5600047BF7A4B7B05794A1247BF7A497B0579E9
:10C570004B1247BF7A537B0579501247BF7A467BEF
:10C580000579531247BF7A5B7B0579541247BF7A0E
:10C59000487B0579E11247BF900540E0A2E35004D3
:10C5A000D2F08002C2F012C9D579521247BF80047E
:10C5B0001246C91E122DDF900912E060046401705A
:10C5C00003122E9990071312CB79600612C5E3125D
:10C5D000261E122D55EEF9740102C4C98E828F8376
:10C5E000E0F8A3E0F58388822274F612242DE9FE98
:10C5F000A2E050267508327509057808122A2175BF
:10C60000086E7509007808122A217C007D007A21C5
:10C610007B00123D757404122A34EEA2E35003121B
:10C620002DE5900912E0600464017008EEA2E1506B
:10C6300003122E9FEEA2E2500E90071512CB7960E6
:10C640000612C5E312261E02C4CC74F612242D7401
:10C65000EC122AC87401122AAA9014EAE0F97AA30B
:10C660007B051231AB900592E06402707C74051278
:10C670002CC7E4F07407122CC7E4F07A04F9122EE8
:10C68000338A08904FE1E493FAC3E5089AEB9400EB
:10C69000400302C71F122E27E9600302C71F904FF5
:10C6A000D312C77B60157A047903122E33904FE1C1
:10C6B000E493FC904FD312C78550087405122CC721
:10C6C0007401F0904FD112C77B60157A0279011284
:10C6D0002E33904FE1E493FC904FD112C785503F29
:10C6E0007407122CC77401803590055E122CA4E8E3
:10C6F000494A4B600474018001E4C0E07405122CC7
:10C70000C7D0E0F0900562122CA4E8494A4B6004BF
:10C7100074018001E4C0E07407122CC7D0E0F090EF
:10C7200014EAE0F97CA37D057401122AA21231A556
:10C730007AA37B0579451247BF7407122CC7E070B6
:10C74000117405122CC7E07009851882851983E4DD
:10C7500080088518828519837401F09014E6E0F84A
:10C760009014E5E058F8851882851983E05812C9BD
:10C77000DF79411247BF741402C4C9E493F874010D
:10C7800093F9E84922E493F8740193F9ECC398F81B
:10C79000E499F9C3EA98EB992274F712242D74ED09
:10C7A000122AC8E9FE90059FF0AC18AD199014EA62
:10C7B000E0F97AA37B051231AB7412122CC7EE128A
:10C7C000C7D7AA18AB191231A57AA37B05794512F0
:10C7D00047BF741302B14CF09014EAE0F97CA37DDA
:10C7E000052274F412242DEAFEEBFF9014ECE064B1
:10C7F000FE7003A3E0F470687A167B00123C4F8A47
:10C80000088B09EA450960588A828B83740112C833
:10C81000808A828B83A3600474028002740112C830
:10C820009BA3E08A828B83A3A3A3A3A3A3A3A3A315
:10C8300012C8B1FCA3E0FDEA2402FAE43509FB12B8
:10C8400046EDE508241312C878E4F0AA08AB099075
:10C8500005A0E0F9123C5B12C86312D0E412C8953F
:10C8600002985B12C86722EE240BF582E43FF58341
:10C8700022850A0CE508250CF582E43509F58322AA
:10C8800012C885E022F08E828F83A3A3A3A3A3A363
:10C8900022E0129775E8F0A3E9F022F0EE241DF5EE
:10C8A00082E43FF58312C8A92212D0F9F583888269
:10C8B00022A3F0EE241512B6202274F212242D7455
:10C8C000FD122AC88A088B09890A8C0B7401122C64
:10C8D000C7740412C9DF1232E98A0C8B0DAE0CAF9B
:10C8E0000DEE4F700302C976EE12B72D3F12C9A5A7
:10C8F0007407F0A3A882A983E5082413FAE4350994
:10C90000FB8A828B8312C9B68A828B8312C9B5E5F2
:10C910000812D32012DEBD8882898312C9C1740136
:10C92000F0E508240BF8E43509F9EE12C98112C9C3
:10C93000CE12EDBE12326512DA1EEE241312EDC0D5
:10C940007403650A60067401650A700712C9917460
:10C9500004800412C991E4F09014EC12ACF712C8F0
:10C96000957401650B7006EE241112C988EEFAEF7A
:10C97000FB122ECF800279109014EC129B4C02D146
:10C980000012EE0A22EE2412F582E43FF583E4F071
:10C990002212C9997440F0A322EE12DEAF3FF58354
:10C9A0002212EDE43BF58312C9AB22E0F8A3E0F9D3
:10C9B0008882898322A3E088828983F0A308A983DF
:10C9C00022F0EE2416F582E43FF58322A3A3E8F0DB
:10C9D000A3E9F0EE22A2F0E433851882851983F0F2
:10C9E000AA18AB192274F412242DEAFEEBFF7A0088
:10C9F0007B049005A0E0F9123DC312CA8312C895CA
:10CA00009005557409F01232658A088B09AC08AD9F
:10CA10000912CA7512D3331246E7E9640170537ADA
:10CA20000F7B00123C4F8A088B09EA450960438A54
:10CA3000828B837402F012CA8DFC88828983A3A33F
:10CA4000E0FBEC8A82850983A3A312DA2888828915
:10CA500083A3A3A3E08A8285098312C8B1FAA3E065
:10CA6000FB794A1247BFAA08AB099005A0E0F9126A
:10CA70003C5B02985B12CA7922EE2413F582E43FF4
:10CA8000F5832290051812D0F490154022EE241D53
:10CA9000F582E43FF58312CD5EE02274F412242D7A
:10CAA00074FD122AC88A088B097401122CC77402FB
:10CAB00012C9DF1232E98A0A8B0BAE0AAF0BEE4FB6
:10CAC000700302CB6512EE29700888828983A374F3
:10CAD00020F0850882850983A3A3A3A3A3E06401B2
:10CAE000700988828983A3E0D2E6F08508828509EF
:10CAF00083A3A3A3A3A3A3E06401700A888289830C
:10CB0000A3E0D2E7800312EDA012EE1A7019850897
:10CB100082850983A3A312CB796006EE241612ED59
:10CB2000C012EDFC12C895850882850983A3A3A3D2
:10CB3000A3A3A3A3E06401700312EDD1850882854D
:10CB4000098312D333123307E9600312EDCA12EDE1
:10CB5000BD12326512CB7F12CB6B12C9CCFAEFFB40
:10CB6000122ECF8002791002BC27E0F8A3E0F98EE4
:10CB7000828F832212B240F58312D0F4E849221248
:10CB8000CB8AEAF0A3EB12CB9422EE241AF582E4CE
:10CB90003FF58322F0850882850983E02274F5122F
:10CBA000242D74F3122AC8890AEAFEEBFF750800E7
:10CBB0007509007C0D7D007900AA18AB19123C376D
:10CBC000EE12D7143FF58312CD4A741F58600C7AC9
:10CBD000D37B001242CD790002CC9CE8A2E550083C
:10CBE000740C122CC77401F0E8A2E75008740B1201
:10CBF0002CC77401F0E8A2E6740A5008122CC7741E
:10CC000001F08008122CC7E0640170138E828F83BC
:10CC1000A3A3A3A3A3A3A3E06032EE241380128EE8
:10CC2000828F83A3A3A3A3A3A3A3A3E0601EEE24E8
:10CC300015F582E43FF58312A6C16010AC08AD097A
:10CC40007402122CC7AA82AB831246ED12C863127B
:10CC5000C891740A122CC7E06401703712D32612EF
:10CC60003307E97035EE240B12B8A6900549E06849
:10CC70007003A3E0697023E5084509601612326568
:10CC8000EAFCEBFD7402122CC7AA82AB831246E7C2
:10CC9000E96007AA18AB19122F89A90A02EF3174AB
:10CCA000F712242D74D2122AC8EAFEEBFF8E828F6F
:10CCB00083129CEDA2E0400302CD4512CD51E05419
:10CCC000FE12E678740D122AAA12CD6E12325FE9B6
:10CCD0007073742A122CC712CD6870697C0D7D00A8
:10CCE0007900AA18AB19123C377416122CC712C857
:10CCF00091742A122CC712CD4AA2E55008740B1267
:10CD00002CC77401F0E8A2E75008740A122CC7740B
:10CD100001F0E8A2E65004742080027422122CC7AD
:10CD200012B0547402122CC7AA82AB831246ED8E45
:10CD3000828F83A3A3E0C0E0740C122CC7D0E01252
:10CD4000C9DF122F83742E02B14C12C8A9A3E0F8D8
:10CD5000228E828F8312CD5EA3A3A3A3A32212D01F
:10CD6000F9F988828983A32212B21F640422EA247B
:10CD70001EF582E43BF583E0F9EA241FF582E43BEB
:10CD800012984F22E9F87900740468600A740A68FE
:10CD900060057403687001090229E674F612242DF7
:10CDA0008A828B837420F0A3A37401F0122ED58A9B
:10CDB000088B09AE08AF09EE4F60168E828F837420
:10CDC00001F0900593E0700912EDBD12326512DAA0
:10CDD0001EEEFAEFFB02C4CCC082C0839005430272
:10CDE000AA04C082C0839014EB02AA04C082C0834C
:10CDF000E99014EB02AA69C082C0839005B874015F
:10CE0000F0E9A2E350037403F0E9A2E15004E0D298
:10CE1000E2F002C15874F612242D79007C008A08D1
:10CE20008B097808122703F8FF0746CE44CE44CE7C
:10CE300044CE44CE3CCE40CE46CE41CE7C0480068D
:10CE40000C0C80027C089005B8E05C60030980034C
:10CE5000EC60010902C4CC74F412242DEAFEEBFF4D
:10CE60008908122E5D8A0A8B0BA80AA90BE8496073
:10CE70004188828983A3A3A3A3E06036C3940550AD
:10CE80003174016508601A88828983A3A3A3A3E093
:10CE90006401600D88828983A3A3A3A3E064027068
:10CEA0000A8882898312A79E12261EEEFAEFFB12D1
:10CEB0002E6902985B74F612242D8A828B83E070AF
:10CEC00012A312CB79600C8A828B8312D33212495F
:10CED0009980047A007B0002C4CCC082C083900594
:10CEE00092E06402700B900555E064087003123301
:10CEF0002B02C158C082C0837C00EC12CFA7700304
:10CF0000A3E06B7011904FE4E493C0E012CF76D0B1
:10CF1000E0F079C580510CECC3940340DD7C00EC5B
:10CF200075F003A4F8A9F074BC28F5827405129773
:10CF30003864FE7003A3E0F4600F0CECC39403406C
:10CF4000DE7C00EC12CF6A7015EC12E31112DA27C6
:10CF5000904FE4E49388828983F0790080090CEC97
:10CF6000C3940340DE79C702C15875F003A4F8A941
:10CF7000F012CF76E02274BB28F582740539F58370
:10CF800022C082C0837D00ED12CFA77003A3E06BA7
:10CF9000700912CF716004790180090DEDC394030B
:10CFA00040E5790002C15875F003A4F8A9F074BCFB
:10CFB00028F582740512E7CA6A2274F212242D74CD
:10CFC000DD122AC8EAFEEBFF750A00900912E06044
:10CFD000076401600302D0DE900546E06E7003A393
:10CFE000E06F701EEE4F700302D0D29005CD12CBD1
:10CFF00079700302D0D2750A0112C5E312261E020F
:10D00000D0DE122E578A088B09EA4509700302D038
:10D01000D28A828B83A3A3A3A3E0640160108A82D7
:10D020008B83A3A3A3A3E06402600302D0D285187C
:10D0300082851983E412D0EB740B122CC7E8F0A39D
:10D04000E912C9DF122E1BE9700302D0D2850882D3
:10D0500085098312D0E412C895790012303785080B
:10D060008285098312DA277403122CC7AC82AD8340
:10D070007418122CC7AA82AB831246ED85088285EC
:10D08000098312B8AC7420122CC712C895742212EE
:10D090002CC7E4F07C02850882850983A3A3A3A39F
:10D0A000E0F9740D122AA21232C58508828509831F
:10D0B00012B8AC7401122CC7E8F0A3E912C9DF1250
:10D0C0002E21750A01E508240C12C878129799F0F0
:10D0D000800C90055312B63EFAEFFB1233DFA90A1B
:10D0E0007423801E12D0F49014EC2212AE8712D05A
:10D0F000F222A3A312D0F9F922E0F8A3E022A90AB0
:10D100007403122A347F060226BDC082C08374FED7
:10D11000122AC8900912E060046401702979019014
:10D12000052B12C5E012261E12D14B900546E8F0E1
:10D13000A3E912C9DF79531247BF85188285198385
:10D1400012D333123EEF740202849F851882851930
:10D1500083EAF0A3EB12D15AF92212BC46F8A3E0FD
:10D160002274F512242D74F3122AC88A088B09EC54
:10D17000FEEDFF750A12EA45097005790002D26ECC
:10D18000900546E065087004A3E065097019123245
:10D1900065EAFCEBFDEEFAEFFB1246E7E970057578
:10D1A0000A018003750A00851882851983E4F0045A
:10D1B000122CC7E508F0A3E50912C9DF122E0FE90A
:10D1C00060297403122CC7AA82AB83122DF1E96483
:10D1D000017018750A017403122CC7AC82AD83EE7E
:10D1E000FAEFFB1246E7E9701E801F7412650A70A1
:10D1F00019900592E064027011EEFCEFFDAA08ABF5
:10D2000009122E3FE96003750A00EEFCEFFDAA0843
:10D21000AB091233FDE9F8740A687005750A0180DC
:10D220004274A0687037EEFCEFFDAA08AB09123417
:10D230000F7E008023EE75F017A4F8A9F012E7E046
:10D240007004A3E06509700F12E91C122DF1E9705A
:10D250000612E4BB1233EB0E12D27140D874016592
:10D260000A70097900AA08AB0912333DA90A02EF36
:10D2700031904FDCE493F8EEC3982274F612242D1B
:10D28000EAFEEBFF8908900912E060046401701E59
:10D2900012332BE508F5097809122A25790DEEFCE1
:10D2A000EFFD7AFC7BFF1233497401122A3402C469
:10D2B000CC74F712242DEAFEEBFF8E828F83A3A39A
:10D2C000A3A3A3A3A3A3E0601312D318129842123E
:10D2D0003337E96401700512C863802D8E828F8315
:10D2E000A3A3A3A3A3A3A3E0602912CA7512D337F3
:10D2F000FAA3E0FB123337E9640170178E828F8343
:10D30000A3A3A3A3A3A3A3A3A312D33312331F796D
:10D31000018002790002B14FEE12D3203FF5832243
:10D320002415F582E4228E828F83A3A3A3A3A3A353
:10D33000A3A3A31298512212D343A3A3A3A3A3A3ED
:10D34000A3E02212B05C8E828F83A3A32274F21218
:10D35000242D74FD122AC88A088B09ECFEEDFF8982
:10D360000B750A017401122CC7740412C9DF123242
:10D37000E9EA4B60477411122CC7E0601AEA2417DF
:10D38000F582E43BF583E412DBD38A828B83E0D21F
:10D39000E7F012D3BFE4F012C9A1740312D62DEE48
:10D3A00088828983A3A3F0EF88828983A3A312AE26
:10D3B00082A3A312F00E122ECFE9F50A02D0FEEAE4
:10D3C0002414F582E43BF5832274F012242DEAFE46
:10D3D000EBFF890A750B0112CA8DF50C88828983CF
:10D3E000A3A3E0FA8882898312D50612BB54640491
:10D3F000600A7AD37B001242CD02D501E50C1228D7
:10D40000CA02000216D4030BB6D4030C9DD40D75CA
:10D41000D40EB6D4B4D4900912E06007640160035E
:10D4200002D4B6900540E0A2E1400302D4B67900F0
:10D43000AB091230CDEA4B60318A828B83A3A3A360
:10D44000A3A3A3E05418602212C8631228458A825D
:10D450008B83A3A312284579008E828F8312D52552
:10D460001230E57404122A34802E7901AA08AB091F
:10D47000122F9B8041900912E06004640170379084
:10D480000540E0A2E1502FAB09123319AA08AB09FD
:10D4900012331FE964C5701E750B008019900912C4
:10D4A000E060046401700F900540E0A2E1500712B3
:10D4B0003F138002880AEE2409F50EE43FF50FAC15
:10D4C00008AD09A90C850E82F58312D333122FB350
:10D4D000850E82850F8312D333123307E96022EE63
:10D4E000241112BB57C39402401712C86312DAED1D
:10D4F0007003A3E069600AE50BA2E05004A90A806A
:10D5000002790002C120A3A3A3E0F8E4C8F9EA2845
:10D51000F508E439F50922E508240CF582E435091B
:10D52000F58312B5FCA3A3A3A3A3A3A3A3A312B043
:10D53000588A828B831298512274EE12242D74F52E
:10D54000122AC88A0A8B0B890C8C0E8D0F7E01EE75
:10D55000122CC7740AF0741D122CC7E0F50DE97087
:10D560000FE50DC333240AC0E0EE122CC7D0E0F063
:10D57000AA18AB191232E98A088B09EA4509700327
:10D5800002D62212B72C350912D7AF740912D7BBB5
:10D59000450D12D64DAC0EAD0FEEFAEFFB1246ED77
:10D5A000EE2408FE50010FE50C70247C00741E125E
:10D5B0002CC712B8AC8012EC12DAD9E82AFAE93B8F
:10D5C000FB12D633A30EAF830CECC3950D40E8E5F8
:10D5D00008241712C8787401F0123265E508241A7D
:10D5E000F582E4350912DA257403122AAAAA0AABD5
:10D5F0000B122DF7E96019E508241612C87874019A
:10D60000F07403122A9AE508241812C87812C895F3
:10D6100085088285098312D629AA08AB09122ECF64
:10D62000E9FEEEF9740B02BE6AA3A3E50AF0A3E5D6
:10D630000BF0228A828B8312D64712D64D8A828BB8
:10D640008312D646F022A3E08E828F8322F0A3AE0F
:10D6500082AF832274F012242D74F8122AC88A082B
:10D660008B0912D713350912D834F50B880AA3AEEB
:10D6700082AF83EEFCEFFDAA18AB191246EDEE2443
:10D6800008FE50010FAC18AD197A677B051246E70A
:10D69000E9607474E0550A7067AA0BEA2AFA7B0005
:10D6A000123CF18A0C8B0DEA450D605B7C00801EFC
:10D6B0008E828F8312C0B6EC12D70CE50C28F5824F
:10D6C000E50D3912DA25EE2402FE50010F0CECC3F1
:10D6D000950B40DC780C122A21780B122A25740352
:10D6E000122AAA7900E508240B12C87812D3331243
:10D6F00033617403122A34AA0CAB0D123CF7800775
:10D700007AD37B001242CD740802C11D25E0F8E4F3
:10D7100033F922EA241DF582E42274F012242D8AC2
:10D720000A8B0B890C8C088D099007E412CB796069
:10D730007B7410122CC7E0F50D12D70CE8240EFAFA
:10D74000E439FB123C4F8A0E8B0FAE0EAF0FEE4F3B
:10D75000605A8E828F8374D4F0A3A3E50AF0A3E508
:10D760000B12BE5DE50CF0AC08AD09EE2405FAE441
:10D770003FFB1246ED12B233E50DF07411122CC7C7
:10D7800012DBBD7808122A1DAC0DEC2CFCE433FD35
:10D79000EE240EFAE43FFB123C2B7403122A34EE03
:10D7A000FAEFFB9007E412C5E012261E02C120F535
:10D7B00083E0FEA3E0FF8E828F8322F0A3E50CC4FA
:10D7C0003354E02274F612242D74F8122AC8890802
:10D7D00012D7133B12D834F98809A3AE82AF8374F1
:10D7E00001697042EEFCEFFDAA18AB191246EDEE8E
:10D7F0002408FE50010FAC18AD197A677B0512465C
:10D80000E7E9602974E05509701C8E828F83A3E0DC
:10D81000FA8E828F83A312C0B88E828F83E0F912B2
:10D820003379A90880097AD37B001242CD7900743C
:10D830000802C4C9F583E02401FEA3E03400FF8E92
:10D84000828F83E0F8741F582274F612242D74DF3F
:10D85000122AC8EAFEEBFF12CB7460508E828F83CF
:10D8600012D333AC18AD1912CD6E12324D740912A9
:10D870002CC712DAED7003A3E069603012C5DC1228
:10D8800028457508FE7509FF7808122A21741C12B4
:10D890002CC7E0F9740D122CC712B054740F122C5F
:10D8A000C712D3331230E57404122A34742102C42F
:10D8B000C974F712242DE9FC7A007B007E00800BEE
:10D8C00012D953E02AFAA3E03BFB0E904FE112D2AB
:10D8D000745029EE75F016A4F8ADF0EDF912E7CF0B
:10D8E000F460E7741D28F582740E3912CB7760DA84
:10D8F000EC60CD12D953E4F0A3F080CE7E00800B13
:10D9000012D940E02AFAA3E03BFB0E12D271502D4F
:10D91000EE75F017A4F8ADF0EDF912E92D7003A340
:10D92000E0F460E674F028F582740F3912CB77606A
:10D93000D9EC60CC12D940E4F0A3F080CD02B14F15
:10D94000EE75F017A4F8EDF974F028F582740F392C
:10D95000F58322EE75F016A4F8EDF9741D28F58212
:10D96000740E39F5832274EC12242D890CEAFEEB37
:10D97000FF90059FE0C3950C503B1232B99005CF44
:10D9800012DA18900539E0F508E4F509F50AF50B07
:10D990009080B47810122C707808791012233E7899
:10D9A00008122A197A007B029005A0E0F9123DB70F
:10D9B0007404122A3402973074F612242DEAFEEB16
:10D9C000FF9005B9801388828983E06E7003A3E01D
:10D9D0006F603688828983A3A312CB7970E87A04BA
:10D9E0007B00123CF18A088B09A808A909E8496064
:10D9F000188882898312DA189005B912DA0CA3A369
:10DA000012DA279005B912C89502C4CC1298518831
:10DA1000828983228A828B83EEF0A3EFF022EE24A8
:10DA20001AF582E43FF583EAF0A3EBF02274F412D6
:10DA3000242D7E009005B980070E88828983A3A3D8
:10DA400012CB7970F4EE12DAD9123CF18A088B0904
:10DA5000EA4509607E7F009005B98021888289832C
:10DA600012B054EF12DAD9E5082AF582E5093BF540
:10DA700083ECF0A3EDF00F88828983A3A312CB7906
:10DA800070DA90059B12DAED7003A3E069780870F4
:10DA90001C122A21EEF50A780A122A257C677D05D8
:10DAA000790090059B12D333123361801A122A2118
:10DAB000EEF50A780A122A257C677D057900900523
:10DAC0009B12D3331233557403122A34AA08AB09BC
:10DAD000123CF7122EE702985B25E0FAE433FB22B2
:10DAE0008E828F83A3A3A3A3A3A3A3A3A312D0F483
:10DAF000900546E06822C082C08380128A828B83B0
:10DB0000A3A312B8AC9005B912C895123CF79005C2
:10DB1000B912AFF770E602C15874F512242D9005C2
:10DB20005312B8B39005CF12DBB112C8957ACF7BF0
:10DB30000579501247BF9005CF12DBBD801512E367
:10DB40006F65087004A3E06509600612E4C3123330
:10DB5000EB050A12DBA65018E50A12E4AF7003A326
:10DB6000E06F70DA74E528F582740F12F00B80E133
:10DB70009005CF12B8B39007E612CB7960257A06EC
:10DB80007B00123C4FEA4B601A8A828B8374D5F07B
:10DB9000A3A3E412DBC40412DBD39007E612C5E0B2
:10DBA00012261E02EF36904FDCE493F8E50AC39884
:10DBB0002212DBB52212D0F9F99005532212ACDE05
:10DBC000750A002212DBC82212DBCC2212AE87A318
:10DBD000A3A32212DBC8A3EEF0A3EFF022C082C001
:10DBE000839005D174A3F0A37433F09005D3749D92
:10DBF000F0A37433F09005D574BBF0A3743302AA7C
:10DC000069C082C083900546E064FE7003A3E0F41F
:10DC1000600E900540E0A2E150061234031233A9D1
:10DC200002C15874F012242D900594E06053F50C55
:10DC3000E4F50DF50EF50F9080AC7808122C707895
:10DC40000C790812233E123C498A088B09A808A9BE
:10DC500009904FCDE49358F508A3E49359F509E4EE
:10DC6000F50AF50B780C7908122B92780C122A1908
:10DC70007A007B019005A0E0F9123DBD7404122AE0
:10DC80003402C12074EE12242D7E007F008E0A8E95
:10DC90000B122EAB8E0D803E850D08AA087B00125C
:10DCA0002EA58A088B09A808A909E8496026888258
:10DCB0008983A3A3A3A3E060046404701788828906
:10DCC00083A3A3A3A3A3A3A3A3A3A3E0F91234153F
:10DCD000E960010F050D904FE1E493F8E50DC3985D
:10DCE00040B61233D98A0E8B0F8E0C8023AA087B84
:10DCF000001233E58A088B09A808A909E849600ED3
:10DD0000E8240F129735F9123415E960010E050C5D
:10DD1000850C08C3E508950EE4950F40D0EF2EFE64
:10DD2000700302DE1D8E0875090074027808122B3C
:10DD3000DEAA08AB09123CF18A0A8B0BEA450B708C
:10DD40000302DE1B750C008E08750900740278084A
:10DD5000122BDEAC08AD0979FF123C37750D00803F
:10DD60005D850D08AA087B00122EA58A088B09EA9A
:10DD7000450960488A828B83A3A3A3A3E06004645F
:10DD80000470398A828B83A3A3A3A3A3A3A3A3A311
:10DD9000A3E0F9123415E96023050C780A122A2150
:10DDA000EEFD850882850983A3A3A3A3A3A3A3A350
:10DDB000A312DEC31233AF7402122A34050D904F42
:10DDC000E1E493F8E50DC3985006E50CC39F40913C
:10DDD000750C00850C08C3E508950EE4950F503DC1
:10DDE000AA087B001233E58A088B09EA45096027F7
:10DDF000EA12DEAF12DEBDF9123415E96019780AB5
:10DE0000122A21EEFDE508240E12C87812DEC31294
:10DE100033AF7402122A34050C80B87E00750E628E
:10DE200090053EE0600CF9122DAFE9F87454C398E8
:10DE3000F50E75F003E50E84F50D94204003750D85
:10DE40001F850A08850B09750C00E50E6006750C28
:10DE500020750E00E50DC39E5004AF0D8008EEFF47
:10DE6000E50CD2E6F50CAC08AD09AA0CEFF91233BB
:10DE7000B5E9F50FE50CA2E6401A1F7800800BE526
:10DE8000082404F5085002050908E8C39F40F0EF94
:10DE9000CEC39EFEE97006E50CA2E650AAE50A454F
:10DEA0000B6007AA0AAB0B123CF7A90F02BE6D2448
:10DEB0000FF582E42274782508F58274133509F58C
:10DEC00083E022E0FC850882850983129851227440
:10DED000F212242DEAFEEBFF89088C098D0A7C00E2
:10DEE0007D00740E122CC712D3338C0B800DEAFC0C
:10DEF000EBFDEA2404FA50010B050BE50BC3950A70
:10DF0000400302DF9A8A828B83E0F47003A3E0F47B
:10DF10006077EC4D600C8C828D83C3E09EA3E09F04
:10DF200050CC8A828B8312E2DEEE98EF9950BFEAE2
:10DF3000F8EBF988828983E0F47003A3E0F46010C1
:10DF4000E82404F8500109050BE50BC3950A40E3EA
:10DF5000E8FCE9FDE824FCF8E934FFF988828983CC
:10DF600012978A8C828D83E50CF0A3E50D12DF9D5C
:10DF70008C828D83A3A312E672E08C828D83A3A38F
:10DF8000A3F0C3EA98EB9940C712DA148A828B8314
:10DF9000A3A3E50912DBC4E508F002D10512DFA353
:10DFA000A3E022F088828983A32274F212242D74C4
:10DFB000FD122AC889088A09ECFEEDFF750A017571
:10DFC000F003E9A42402C0E07401122CC7D0E012CF
:10DFD000C9DF1232E9EA4B607812C9A17408F07403
:10DFE0001F55084509A3F0E82402F8500109750AF5
:10DFF0000080388E828F83E088828983F0A3A88294
:10E00000A9838E828F8312C9B58E828F83A3A3E0EA
:10E010005407C4FC8E828F83A3A3A3E054074C1241
:10E02000C9B7EE2404FE50010F050AE50AC395089E
:10E0300040C18A828B83A3A374FCF0A374FFF0EA2F
:10E040002413F582E43BF5837401F0122ECFE9F539
:10E050000A02D0FE74F112242D8A0A8B0B75080077
:10E060007AFE7BFF7CFE7DFFE50A12D714350B128A
:10E07000CA94F509741F5509F50CE82402F85001FB
:10E0800009E509A2E7406FE50A2417F582E412E2E8
:10E090004EFE75F003E50CA424026E7059E50C6089
:10E0A0000B88828983E0FEA3E0FBEEFA750D008009
:10E0B0001DE05407F50EA3A882A983EEFC90054647
:10E0C000E06E7003A3E06F7003850E08050DE50D8B
:10E0D000C3950C502B88828983E0FEA3E0FCE4CC3E
:10E0E000FDEE2CE43DFFE82402F850010988828906
:10E0F00083E0548860BB7AD37B001242CD02E243B6
:10E10000E508700BA9091233C1E9700302E243125A
:10E11000E26012D333122E578A0C8B0DAE0CAF0D6A
:10E12000EE4F605A8E828F83A3A3A3A3A3A3A3E47D
:10E13000F0904FF493F88E828F83A3A3A3A3A3A39D
:10E14000A3A3E0C398402412E26A5001097A027B3B
:10E1500000122246E88E828F83A3A3A3A3A3A3A3C6
:10E16000A3F0E508C39407500205088E828F83A3AD
:10E17000A3A3A3A3A3A3A3A3E508F002E2437CFF08
:10E180007DFF12E26012D3331233CD8A0C8B0DAEB9
:10E190000CAF0DEE4F704F1233D38A0C8B0DAE0CBB
:10E1A000AF0DEE4F700302E2437C177D0079001241
:10E1B0003C3712E26012CB6A1284918E828F83A365
:10E1C000A3A3A3A3A3A3A312C9CC12B61574AA1226
:10E1D000E2895001097A027B0012224612B233E82A
:10E1E00012E2757401F0904FF4E493F8EE240D12EE
:10E1F000BB57C398401912E26A5001097A027B00AA
:10E2000012224612E254E508C39407500205081290
:10E21000E8DBE50812E27AE4F0129C82122DF1E9C3
:10E220007021850A82850B83A3A3A3A3A3A3A3A321
:10E23000E06010E50A12D320350B12B63C129C8325
:10E240001246ED02A87F7478250AF5827413350B07
:10E25000F583E022EE240DF582E43FF583E8F02219
:10E26000E50A12EDE5350BF58322904FF4E493793E
:10E27000002401F822F012E8DF22F012E27F22EE01
:10E28000240CF582E43FF58322F0904FF4E4937977
:10E29000002401F82274F712242DE9FE74FE6A703E
:10E2A0000374FF6B603474605E6460602DEEA2E501
:10E2B000401CA2E6900546500DC3E09AA3E09B5097
:10E2C00019790002B14FC3E09AA3E09B40F3900597
:10E2D0004612E2DEEC98ED9940E7790180E512D034
:10E2E000F4C32274F712242D7E00800712E4BB12BF
:10E2F00033EB0E12D27140F47E00EE12E311129B4A
:10E300004C88828983E4F00EEEC3940340EC02B1A2
:10E310004F75F003A4F8A9F074BB28F8740539F917
:10E3200088828983A32274F712242D7F0080010F35
:10E33000904FDCE493F8EFC398502DEF75F017A4DD
:10E34000F8A9F012E7BB6A7003A3E06B70E112E377
:10E350006F6C7003A3E06D600A74FF6C700374FF50
:10E360006D70CC12E4C380047A007B0002B14F12BE
:10E37000E3732274E528F582740F12E7CA2274F65B
:10E3800012242D7CFF7DFF7AFE7BFF1233CDEA4BFA
:10E39000703C7508008032E50875F017A4F8A9F004
:10E3A00074EA28F582740F129738600512E7B0708E
:10E3B0001674DB28FE740F39FF8E828F8312D333DD
:10E3C0001230EBEEFAEFFB050812E3D140C902C4AC
:10E3D000CC904FDCE493F8E508C39822C082C08358
:10E3E0007A007B007D00801012E9257003A3E0F421
:10E3F00060050AEA70010B0D904FDCE493F8EDC361
:10E400009840E502C15874F412242D8A088B09EC57
:10E41000FEEDFF800B1233EBEEFCEFFDAA08AB091B
:10E420001233CDEA4B70EE02985B74F612242D7D08
:10E43000007E0080020D0E12D2715018EE12E926F5
:10E440007003A3E0F460EF8D08EA65084B70E612F4
:10E45000E4C380047A007B0002C4CC74F712242D3C
:10E46000EAFEEBFFEE4F601A7C177D007900123C4C
:10E47000378E828F8374FEF0A30412AD01A31412B1
:10E480009B4E02B14F74F712242DEAFEEBFF750884
:10E49000008014E50812E4AF7003A3E06F60061279
:10E4A000E4C31233EB050812E3D140E702B14F7524
:10E4B000F017A4F8A9F012E3736E22EE75F017A41A
:10E4C000F8A9F074DB28FA740F39FB2274F41224D3
:10E4D0002D8A088B09ECFEEDFF900912E0600464C0
:10E4E000017020900553E06E7003A3E06F7014126A
:10E4F0002E578A0A8B0BA80AA90BE8496005E82465
:10E5000008801AEEFCEFFDAA08AB091233CD8A0889
:10E510008B09A808A909E8496009E8240DFAE4393B
:10E52000FB80047A007B0002985B74F412242D8A2D
:10E530000A8B0BECFEEDFF7508007509008034E5D1
:10E540000912E915122DF1E96027E50975F017A404
:10E55000F8A9F012E7DA7004A3E0650B7003750800
:10E560000AEEFCEFFD12E91C1246E7E960034308DE
:10E57000A00509904FDCE493F8E509C3985004E541
:10E580000860BC02BEED74F612242D7E00805C8E05
:10E5900008AA087B00122EA58A088B09A808A909D9
:10E5A000E849604688828983A3A3A3A3E06401604D
:10E5B0003988828983A3A3A3A3E06402602CE824A2
:10E5C00007129735FA74012AF0900595E0C39A5026
:10E5D0001988828983A3A3A3A3A3A3A3A3A3A3E4CA
:10E5E00012E669A312E6781230EB0E904FE112D2D8
:10E5F00074409C7E008059EE75F017A4F8AAF0EAEA
:10E60000F912E92D7003A3E0F4604474DB28F87478
:10E610000F39F9E8240C129735F8740128F09005A9
:10E6200095E0C3985029EE75F017A4F8EAF974DB69
:10E6300028F8740F39F9E812DEAF39F583E4F0E811
:10E64000240EF582E439F583E412E6781230EB0EFD
:10E6500012D27140A27B00EB12CF6A600214F00B61
:10E66000EBC3940340F102C4CC12E672A3A3A3A3AC
:10E67000A32212DFA3A3A32212E680FAA3E0FB22C7
:10E68000F088828983E02274F312242D8A088B0992
:10E69000ECFEEDFF750C007B007C01740D122CC7A5
:10E6A000E0F50AA3E0F50B8010123C49E50CF5F00B
:10E6B000EA84ABF0750C007C007D0080010D904F6A
:10E6C000DCE493F8EDC398504912E9257003A3E008
:10E6D000F460EA12E7E07004A3E0650960DF12E786
:10E6E000BB6E7003A3E06F60D412E7DA7004A3E09E
:10E6F000650B60C912E7B060C4C3940750BFEC0556
:10E700000C70BAE50CC39B40B474DB28F582740F1F
:10E7100080787A0080010A904FE1E493F8EAC39888
:10E720005070EA75F016A4F8A9F012E7E664FE70DE
:10E7300003A3E0F460E012E7E665087004A3E06577
:10E740000960D312E7E66E7003A3E06F60C812E7BA
:10E75000E6650A7004A3E0650B60BB741628F582B9
:10E76000740E12973860AFC3940750AA12E7CF64B3
:10E770000160A3E06402609EEC050C7099E50CC397
:10E780009B4093740D28F582740E39F58312D333B0
:10E790008019E50C6011EB700E7401650C600302CA
:10E7A000E6A97B0102E6B47AFE7BFF7F050226BD67
:10E7B00074E928F582740F12E7CA2212E7BF2274A7
:10E7C000DB28F582740F12E7CA2239F583E0227440
:10E7D0001128F582740E12E7CA2212E7BF650A22D9
:10E7E00012E7BF650822740D28F582740E12E7CA7D
:10E7F0002274F512242D8A088B09ECFEEDFF750AB0
:10E80000008002050A12DBA65022EEFCEFFDE50AAD
:10E8100012E9151246E7E960EAE50A75F017A4F86F
:10E82000A9F074DB28F582740F12F00B02EF36E9C1
:10E83000F87907C3940D400479018019E8C394075F
:10E8400040047903800FE8C394034004191980053C
:10E85000E8700279000229E674F012242D8A088BF0
:10E86000098C0A8D0B890C1233D38A0E8B0FAE0ED6
:10E87000AF0FEE4F60627C177D007900123C378E3F
:10E88000828F8312F00E8E828F83A3A3A3A3A3A3F0
:10E89000A3A312D629E50C600712B614E50C800577
:10E8A00012B6147401F09005D312CB79601590055F
:10E8B0009AE06401700612E8DBE4800C12E8DB7475
:10E8C00007800512E8DB740112E2895001097A021F
:10E8D0007B0012224612E25402C12012E8DF22EE2F
:10E8E000240EF582E43FF5832274F712242D7E0076
:10E8F000801BEE12E9267003A3E0F4600F12E91CFE
:10E90000122DF1E9700612E4BB1233EB0E12D27134
:10E9100040E002B14F75F017A4F8A9F074DD28FAB1
:10E92000740F39FB22ED75F017A4F8A9F012E7BFB8
:10E9300064FE22C082C0839005D7742DF0A3743486
:10E94000F09005D97433F0A37434F09005DB74397A
:10E95000F0A3743402AA6974F712242DEAF8EBF9D3
:10E9600090051612E9A0CA2406F582E43AF583E080
:10E97000702B88828983A3A3A3A3A3A3A3A3A31219
:10E98000284590051612E9A5122C9888828983A340
:10E99000E0F9122FA77402122A34122EE702B14FA7
:10E9A000E0FAA3E02212E9A0F5838A8222C082C0A5
:10E9B0008390059D12EA70F090059D12CB79700549
:10E9C000790112337302C15874F612242D74FC12AB
:10E9D0002AC8E9FE904FE5E493700874E16E600385
:10E9E00002EA6BEA2408F8E43BF98882898312EA98
:10E9F0007012EA79700E90059DE4F0A3F07901128F
:10EA000033738067900914E06061FA90059D12E20B
:10EA1000DEEA98E499505479001233738A088B091E
:10EA2000AC08AD09ECF8EDF9E875F064A4F8AAF0CB
:10EA300075F064E9A42AF990059D12D33312224E91
:10EA4000E8941AE9940040239007DE12CB79601B0A
:10EA500090059D12C8917402122CC7ECF0A3ED1220
:10EA6000C9DF9007DE12C5E012261E740402C4C975
:10EA7000E02401F0A3E034002212E680F8A3E0F9DC
:10EA8000E84922C082C08374F8122AC890805AAC28
:10EA900018AD197408122962AC18AD191246E7E9CD
:10EAA0006401700479008002790102849D74F61279
:10EAB000242D740C122CC712B8B3743A6E7001EF87
:10EAC0006006743B6E4F7023740A122CC7122845DF
:10EAD0008C088D097808122A21EAFCEBFDEEFAEF8A
:10EAE000FB123D7B7404122A348002790A02C4CCE2
:10EAF000C082C0839005DD74B1F0A3742EF0900540
:10EB0000DF74B7F0A3742EF09005E17457F0A3748E
:10EB100034F09005E3745DF0A37434F09005E5746F
:10EB200063F0A37434F09005E77469F0A37434F0D3
:10EB30009005E9746FF0A37434F0745744346003A3
:10EB400012345702C15874F412242D74E9122AC8E1
:10EB50008A088B097404122CC77402F004122AA2CA
:10EB60001232E98A0A8B0BAE0AAF0BEE4F7003022A
:10EB7000ED8C12EE29700888828983A37420F085B9
:10EB80000882850983A3A3A3A3A3E0640170098875
:10EB9000828983A3E0D2E6F0850882850983A3A356
:10EBA000A3A3A3A3E06401700A88828983A3E0D2AF
:10EBB000E7800312EDA012EE1A701985088285090C
:10EBC00083A3A312CB796006EE241612EDC012EDDA
:10EBD000FC12C895850882850983A3A3A3A3A3A3D8
:10EBE000A3E06401700312EDD185088285098312C8
:10EBF000D333123307E9600312EDCA12EDBD1232AE
:10EC00006512CB7FFAA3E0FB8E828F83A3A312DA77
:10EC100027123307E9600312C985EE241312BB578C
:10EC2000700D904FE9E493C0E012CA75D0E0F08E09
:10EC3000828F83E0A2E7500454038019EE2414125B
:10EC4000BB577012900532E0C0E012ED96D0E0F0B4
:10EC5000900532E004F012EDAF701990154DE060B0
:10EC60000D90053DE0700D8E828F83E07006EE24DE
:10EC70001112C988AC18AD19EEFAEFFB1232418AB5
:10EC8000088B09EA4509700302ED807A217B0012A6
:10EC90003CF17406122CC712DA277406122CC71224
:10ECA000CB79700302ED74900912E0600464017086
:10ECB0000812B614A3E04404F07401122AA2795099
:10ECC0001247B97401122CC712B8AC7406122CC7C3
:10ECD00012E9A0CA2409F582E43AF58312C8959096
:10ECE000054612B8AC7415122CC712C895740612DA
:10ECF0002CC712B89E12EDDBF07406122CC712ADB1
:10ED0000D3740212EE137406122CC712E9A512BCBA
:10ED10003AC0E07406122CC712B89E12EDA6D0E0DD
:10ED2000F0EE240E12EDB8C0E07406122CC712EDFE
:10ED3000EBD0E0F07406122CC712862012F00CEE15
:10ED4000240F12B8A6740C122CC712C8958A828B95
:10ED500083E0C0E0740E122CC7D0E0F07406122AD3
:10ED6000A21231BDE9F50A7406122CC712D3331270
:10ED70003CF78003750A10AA08AB09123CF7800320
:10ED8000750A10EEFAEFFB123CF78003750A10A922
:10ED90000A7417029858EE2414F582E43FF5832292
:10EDA00012CA79740122241EF582E438F58322EE1A
:10EDB000241112B62064012212B607E022EE2417B5
:10EDC000F582E43FF5837401F02212B61D4404F08D
:10EDD0002212C9997401F0A3E4F02212EDE538F58E
:10EDE00083740222EA240BF582E42212EDEF221250
:10EDF000D0F9C8240CF582E438F583228508828591
:10EE0000098312D0F2EE12EE0A222418F582E43FB2
:10EE1000F5832212B65612D0F32212EE21E06401DD
:10EE20002212EE42A3A3A3A32212C86712C9AB7495
:10EE300004F0A3E412EE3EA3A3A3E064012212EEC9
:10EE40004222F0850882850983A32274F612242DBC
:10EE50007E00801F7C047D0079FF8E088D0974027E
:10EE60007808122BDE74782508FA74133509FB1222
:10EE70003C370E904FEB12D27440D902C4CC74F5DB
:10EE800012242D74F7122AC8750A00801E850A08FC
:10EE900075090074027808122BDE747A2508F58251
:10EEA000741312C87B12EF24F0050A904FEB12DBAB
:10EEB000A9506D850A0875090074027808122BDEC6
:10EEC00012DEB5F47003A3E0F460DE850A0875096C
:10EED0000074027808122BDE747A2508F582741308
:10EEE000350912CB7770A67408122CC77402F0850E
:10EEF0000A087509007808122BDE74782508FE745C
:10EF0000133509FF8E828F8312C89112EF2D12489C
:10EF1000077C047D0079FFEEFAEFFB123C37808915
:10EF20007409800FE024FFF0A3E034FF2212F09B6D
:10EF300022740D122A347F030226BD74F012242D90
:10EF400074F7122AC8EAFEEBFF8C088D09750CFFD6
:10EF50007408122CC712F08D124801E9641A70036C
:10EF600002F007750E00800B74FF650C7003850EB0
:10EF70000C050E904FEBE493F8E50EC398504885CE
:10EF80000E0A750B007402780A122BDE12E246F4A8
:10EF90007003A3E0F460D1850E0A750B007402784B
:10EFA0000A122BDE12E2466E7003A3E06F70C27588
:10EFB0000F007402780E122BDE747A250EF582741F
:10EFC00013350FF5838030E493650E702D74FF6563
:10EFD0000C602E850C0A750B007402780A122BDE69
:10EFE0007478250AF87413350BF98882898312DA4C
:10EFF0001888828983A3A312F00E7901740902C1D3
:10F000001D12EF2D124807790080F139F583E508CC
:10F01000F0A3E509F02274F412242D74F7122AC823
:10F02000EAFEEBFF7408122CC712F08D1248077528
:10F030000A008002050A904FEB12DBA9504C850AAA
:10F040000875090074027808122BDE12DEB5F47020
:10F0500003A3E0F460DE850A0875090074027808ED
:10F06000122BDE12DEB56E7003A3E06F70C67C0457
:10F070007D0079FF8D0B7402780A122BDE747825DF
:10F080000AFA7413350BFB123C3702ADC37402123B
:10F09000A4D0EEF0A3EFF012F09B2290055312B033
:10F0A0005CAA18AB1922C082C08374F8122AC885E2
:10F0B000188285198312DA277402122CC7E4F0A390
:10F0C000F07404122CC77401F07405122CC774017B
:10F0D000F07406122CC7E4F07407122CC7E412C9AE
:10F0E000DF12345102849D74EE12242D8A088B099C
:10F0F000ECFEEDFF750C00EE65087003EF6509602E
:10F100000C123D6F8A0A8B0BEA450B7006750C01D9
:10F1100002F1A3EEFAEFFB123D6F8A0E8B0FAC0EDD
:10F12000AD0FEC4D6007EEFAEFFB123D81E4F50EFA
:10F13000F50F780E122A21AC0AAD0BEEFAEFFB1296
:10F140003D697402122A34E96059AA0AAB0B123CD9
:10F15000F18A0E8B0FEA450F6046780E122A21784D
:10F160000A122A217C007D00AA08AB09123D7B749B
:10F1700004122A34E9701D780E122A21780A122A04
:10F18000217C007D00EEFAEFFB123D757404122A1B
:10F1900034E96003750C01AA0EAB0F123CF7800333
:10F1A000750C10A90C02BE6D74F712242D90071770
:10F1B0008008EAFEEBFF8A828B8312FC9BEA4B609D
:10F1C0003BEA2408F582E43BF583E014F070E31297
:10F1D000FE39EA687002EB698A828B83700B12FE3B
:10F1E0004212F911123CF780C412FE3C8E828F83CA
:10F1F00012F911123CF78E828F8380BE12F7846061
:10F200001AE0C812F77BE01412F773E0700D12FCDD
:10F2100098123CF7900719E4F0A3F090071712F743
:10F2200087700512F78460269080AC1228417A0816
:10F230007B0090071DE0F9123DB77404122A34E9EF
:10F24000600C7A087B0090071DE0F9123C917F0169
:10F250000226BD74F612242D74FA122AC8EAF8EBBD
:10F26000F97E0088828983A3A3E0602B14603414A4
:10F27000603114603414602524F460331470030288
:10F28000F35314700302F34D14700302F359147016
:10F290000302F39502F3E212391902F3E412391F63
:10F2A00002F3E412392502F3E412392B02F3E48865
:10F2B000828983A3A3E0FFE82403F8500109888230
:10F2C0008983A3AA82AB8388828983E06063146008
:10F2D0005514602F1470668A828B83A3A3E0F98A89
:10F2E000828B83E0FCA3E0FBECFA124783E9600821
:10F2F0007403122CC7E480077403122CC77401F046
:10F30000E080328A828B83E0F9123829EA4B600C64
:10F31000124789851882851983E48029851882859A
:10F3200019837401801F8A828B83E0F912477780EA
:10F330000312477DE9851882851983800885188224
:10F34000851983740212FF52EFFA02F3DB12393D82
:10F3500002F3E412394302F3E488828983A3A3A36E
:10F36000A3E0C0E07401122CC7D0E012F96EA3A391
:10F37000A3A3E0C0E07402122CC7D0E0F074011225
:10F380002AA288828983A3A3A3E0F912385912FF25
:10F390004B7A1380469081107401122AAA740212CB
:10F3A000296204122AA288828983A3A3A3E0F91206
:10F3B00038537401122CC7E0C0E07404122CC7D07B
:10F3C000E0F07402122CC7E0C0E07405122CC7D024
:10F3D000E0F07404122AAA7B037A1479641238F5D7
:10F3E00080020E0EEEF97406122A347F020226BD48
:10F3F00074F212242D74FF122AC88A088B0912F4A1
:10F4000098F50A7A067B00123CF18A0C8B0DAE0C43
:10F41000AF0DEE4F603F8E828F83A3741DF0A374F7
:10F4200007F0EEFCEFFDE5082403FAE43509FB12D2
:10F430003907E9851882851983F0700FEEFAEFFB22
:10F440001237F3E9851882851983F0E06007EEFA38
:10F45000EFFB123CF7AC18AD197B01AA0A796412D4
:10F4600038F57401122A347F060226BD74F712247F
:10F470002D74FF122AC812F498FE8A828B83A3A3EC
:10F48000A3E0F91237F912FF4BEEFA79641238F55E
:10F490007401122A3402F24E851882851983741081
:10F4A00012F9852274EA12242D74F2122AC88B0DE7
:10F4B000851882851983740112F967E0F5128A8232
:10F4C0008B83A3A3E0F50FEA2403F50C5002050D8E
:10F4D0007402650F7071850C82850D83E0F8740AE3
:10F4E000122CC7E812F7557403687021850C088543
:10F4F0000D09750A007808122A1D7C087D00740524
:10F50000122AA2123C2B7403122A34800912F91712
:10F51000122CC712F911E50C2408F50C5002050D48
:10F52000F582850D83E0C0E0740B122CC7D0E01289
:10F53000F755E0FAA3E0F9EAF8740C122CC712F7B9
:10F5400049503A050D8036740A122CC77402F085B2
:10F550000C82850D8312F917122CC712F74950023D
:10F56000050DF582850D83E0C0E0740B122CC7D029
:10F57000E012F755740C122CC7E4F0A3F0850C824E
:10F58000850D83E0F91238298A108B11850C82854C
:10F590000D83A385820C85830D12F768F508E43985
:10F5A000F509E50C2402F50C5002050DF582850DD8
:10F5B00083E0C0E07401122CC7D0E012F75FE0F5E1
:10F5C0000BA3E0F50AA385820C85830D7402650FF9
:10F5D000701A12F768FEE439FFEE2414F8E43FF9DC
:10F5E000E50C2402F50C5016050D8012E0FE7F009C
:10F5F000A385820C85830D240AF8E43400F9E51014
:10F6000045116011C3E894FBE99400500302F6E948
:10F6100012F784600B851882851983740202F7291A
:10F62000EE2418FAE43FFB123CF1900719EAF0A32C
:10F63000EBF012F784851882851983700574100227
:10F64000F729E4F0900719E02418FAA3E03400FB4E
:10F6500012FFABEAF0A3EBF07402122A9A880C892D
:10F660000D750E00780C122A1D7C0C7D0012FF5ABD
:10F67000123C2B7403122A3412FF9FE510F0A3E50D
:10F6800011F012FF93E508F0A3E509F012FF7EEEFA
:10F69000F0A3EFF07401122CC7E0C0E012FF8A243F
:10F6A00014F582E438F583D0E0F012FF72E50BF038
:10F6B000900719E0F8A312FF67E50A12F773740FB9
:10F6C000F09080AC1228417A087B0090071DE0F989
:10F6D000123DB77404122A34E9604F7A087B009017
:10F6E000071DE0F9123C918041780A122A25740224
:10F6F000122A9A881489157814122A21780C122A51
:10F70000218E0C8F0D780C122A217808122A21A93B
:10F710000BAC10AD11740B122AA212381774091217
:10F720002A34E9851882851983F074E05512642023
:10F73000700DAC18AD197B01AA0F79641238F574FD
:10F740000E122A347F0E0226BDE8F0A3E9F0E50C84
:10F750002402F50C2212F75F85820C85830D22F0BE
:10F76000850C82850D83A322E0FAA3E0F8E4C8F9B2
:10F77000EA2822F012FF8A12F77B222417F582E48E
:10F7800038F58322900719E0F8A3E0F9E8492274DC
:10F79000EC12242D74F2122AC8EAFEEBFF851882BF
:10F7A000851983740112F90AA3E0F50EEE2403FE15
:10F7B00050010F7C0C7D0079007402122AA2123CC9
:10F7C00037740A122CC77402F08E828F8312F917D5
:10F7D000122CC712F911EE2402FE50010F8E828FF7
:10F7E00083E0C0E0740B122CC7D0E012F90AE0F9F4
:10F7F000A3AE82AF831238298A0A8B0B8E828F8345
:10F8000012FE53EE2402FE50010F8E828F83E0C061
:10F81000E07401122CC7D0E012F90AE0F50FA3E062
:10F82000F512A3E0F513A3AE82AF8325E0FAE4332B
:10F83000FB123CF18A088B09EA4509700302F8EAD9
:10F840007C00802412F76BE439FBEC25E0F8E4330C
:10F85000F9E50828F582E50939F583EAF0A3EBF02C
:10F86000EE2402FE50010F0CECC395138E828F83A1
:10F87000E0FAA340CFAE82AF83E50A450B700A855C
:10F880001882851983740280577808122A21E5139B
:10F89000F5107810122A25E512F5107810122A2595
:10F8A0007405122A9A881089117810122A218E1054
:10F8B0008F117810122A218A107511007810122ADF
:10F8C00021780C122A21A90FAC0AAD0B740E122A52
:10F8D000A212381D740C122A34E985188285198306
:10F8E000F0AA08AB09123CF78009851882851983B4
:10F8F0007410F0AC18AD197B01AA0E79641238F5BA
:10F90000740E122A347F0C0226BDF08E828F83A3E0
:10F9100022E8F0A3E9F022E0FAA3E0F9EAF87402A1
:10F9200022C082C08374FD122AC812F975C0E07427
:10F9300001122CC7D0E012F95CC0E07402122CC78F
:10F94000D0E0F0AC18AD197B037A8079441238F519
:10F950007403122A34D083D0820229E612F961E0BE
:10F960002212F967A3A322F08A828B83A322F08854
:10F97000828983A3228A828B83A3E08518828519DA
:10F980008312F9852212F967A3E02274E912242D6B
:10F990008A108B11EA242012FC2912FE4BE50A245E
:10F9A00014F508E4350BF509751681751200751309
:10F9B00000EA12FC43E0F9EA241012FC2912FC9B35
:10F9C000124783E97017E510240E12FC29E0640346
:10F9D000600BC3E50894F1E5099400400E751682AA
:10F9E000E508240AF508E43509F509C3E50894FBA0
:10F9F000E50994004036E50A2409FAE4350BFB12C8
:10FA00003CF18A128B13EA4513700302FC24EA24AA
:10FA100009F8E43513F98A828B83A3A312F911C381
:10FA2000E508950AF508E509950BF509AA08AB095B
:10FA3000123CF18A148B15EA45157010E512451336
:10FA40006007AA12AB13123CF702FC24AE14AF15E8
:10FA5000E510240212FCAD240412FCA112FC8B74EC
:10FA6000826516705CE510240E12FC3512FC8B8842
:10FA7000828983E064037025E5102406F50CE435E3
:10FA800011F50D750E00780C122A1D7C087D00EE14
:10FA9000FAEFFB123C2B7403122A34800E12FC3155
:10FAA00012FC8512F96E12FC85A3F0EE2408FE50BC
:10FAB000010FE51012FC4312FCBD241012FCA180C2
:10FAC0000D12FC3112FC7B0E12FCB612FC4312FC30
:10FAD000BD241412FC74AE82AF83E510241512FC11
:10FAE0002912FCBD241612FC2912FCBD241912FC9B
:10FAF0002912FCBD241AFAE43511FB8A828B837823
:10FB00000C122C7012FC4D122C70E50D8E828F831E
:10FB100012FC53122C707410780C122A6912FC4DCE
:10FB2000122C707418780C122A698E828F83E50C5F
:10FB3000F0A30EAF8374826516700EE4F0A3E50A9D
:10FB4000F0A3E50BF0A30E800BE510241F12FC744C
:10FB5000E50AF0A30E0EAF83E5124513700302FB16
:10FB6000E312FE3985128285138312F9119007176B
:10FB7000E512F0A3E513F0851282F583A3A3A3A3F6
:10FB8000A3A3A3A3740FF09080AC1228417A087B42
:10FB90000090071DE0F9123DB77404122A34E960A1
:10FBA0000C7A087B0090071DE0F9123C91E51024C7
:10FBB0001A12FC29122CA4851282851383A3A3A3F5
:10FBC000A3122CB012FC5F122A1DAC0AAD0B8512D9
:10FBD00082851383A3A312FC9B123C2B7403122A6D
:10FBE00034801E12FC5F122A1DAC0AAD0BEEFAEF38
:10FBF000FB123C2B7403122A34EE250AFEEF350B60
:10FC0000FFE510242412FCAD242612FC2912FC80EE
:10FC1000AC14AD15AB08AA1679441238F5AA14AB8A
:10FC200015123CF77F0F0226BDF582E43511F583EE
:10FC300022E510240612FC3922F8E43511F98882F5
:10FC4000898322240FF582E43511F583228E828F79
:10FC500083E50CF0A30EAF838A828B83780C22E5B8
:10FC6000102422F582E43511F583E0F50CA3E0F5CC
:10FC70000D780C22F582E43511F58312FC80A32265
:10FC800012FC85F022E08E828F832212FC8F2212DA
:10FC9000FC85F0A30EAF8322900719E0FAA3E0FBE6
:10FCA0002212FC3912FC8F88828983A32212FC392C
:10FCB00012FC80A3AE82AF8388828983A312FC8F5B
:10FCC000E5102274EB12242D8A088B099007171275
:10FCD000FE4B7A01751400E5082403F5085002056F
:10FCE00009F582850983E0F50CE4F50DF50EF50FB5
:10FCF000A3E0F510E4F511F512F51374087810126D
:10FD000029C1780C7910122B92850882850983A36A
:10FD1000A3E0F510E4F511741078101229C1780CE5
:10FD20007910122B92850882850983A3A3A3E0F59D
:10FD300010E4F512741878101229C1780C79101299
:10FD40002B9280078C828D8312FE4BE50A450B6057
:10FD500059AC0AAD0B8C828D83A3A3A3A3780C129C
:10FD60002ADE70E0E5082404F50850020509F58252
:10FD700085098312FE53850882850983A3A3E0F5D4
:10FD800014704512FE39EC687002ED698C828D8327
:10FD9000700512FE42800712FE3C8C828D8312F9A0
:10FDA00011AA0AAB0B123CF77A00EA850882850992
:10FDB00083F0A3E514F0AC08AD097B027A127964F4
:10FDC0001238F57F0D0226BD2402FAE43400FB123E
:10FDD0003CF18A0E8B0FAE0EAF0FEE4F70077A100C
:10FDE00075140080C58E828F83E4F0A3E514F0853E
:10FDF0000A82850B83A3A3E0250CF508A3E0350D4B
:10FE0000F509750A007808122A1D851408AC087DCA
:10FE100000EE2402FAE43FFB123C2B7403122A3456
:10FE2000EEFCEFFD74022514FB7A1279641238F5AA
:10FE3000EEFAEFFB123CF7808A900717E0F8A3E098
:10FE4000F922E0F8A3E0F990071722E0F50AA3E011
:10FE5000F50B22E0FAA3E0F8E4C8F9EA28F50CE48F
:10FE600039F50D2274F512242D74FF122AC8851855
:10FE7000828519837401F0EA2403FA50010B8A8207
:10FE80008B83E0FCA3E0F8E4C8F9EC28FEE439FF3A
:10FE90008A828B83A3A3E0FCEA2403FA50010B12AD
:10FEA000F784700B851882851983741002FF37EC74
:10FEB000705E12FF67E0F5087808122A259007198E
:10FEC000E02414F508A3E03400F5097808122A218B
:10FED00012FFAB12284512FF7E12284512FF931223
:10FEE000284512FF72E0F912FF9FE0FCA3E0FD122B
:10FEF000FF5A1238177409122A34E98518828519B5
:10FF000083F012FC98123CF7900719E4F0A38027C5
:10FF10008A088B09750A007808122A1D7D0012FFD5
:10FF2000ABE02EFAA3E03FFB123C2B7403122A3401
:10FF3000851882851983E412FF527A117964123888
:10FF4000F57401122A347F030226BDE985188285E3
:10FF50001983F0AC18AD197B0122900719E0240237
:10FF6000FAA3E03400FB22E0C82416F582E438F559
:10FF7000832212FF8A2415F582E438F5832212FFCA
:10FF80008A2412F582E438F58322900719E0F8A359
:10FF9000E0C82212FF8A2410F582E438F583221289
:10FFA000FF8A240EF582E438F58322900719E0F8E1
:10FFB000A3E0F583888222C082C083124873801038
:10FFC000C082C0831248798007C082C0831248A9CA
:10FFD000D083D0820229E6C082C0831248AF80F06D
:10FFE000C082C08390093FE0F9D083D0820229E625
:10FFF0000229E60229E60229E60229E6FFFFFFFFC1
:020000040001F9
:10000000C082C0837900EA1282053BF583C082C0BA
:100010008390051212D406D083D082C3E09CA3E063
:100020009D500CEA240B12805212803260010902AA
:10003000A385EA75F00BA4FAA8F075F00BEBA428E1
:10004000FB900514E02AF8A3E03B8882F583E05496
:100050000F22F582E43B12B4FE2274F712242D899C
:100060000812AB97A3E0F9E875F00BA4F8ACF075B3
:10007000F00BE9A42C1283B6E8FEE9FF74016508D1
:1000800060067402650870228A828B831286E2748D
:100090000265087021EA2403FA50010B122DF1E9E0
:1000A00070148E828F83E4F0800CEA2403FCE43B1E
:1000B0001286D9122DEB8E828F83E0D2E7F0123FA9
:1000C0002502A81074F412242D12879C79008E82C8
:1000D0008F83E06075890A890B8064E50A75F00BEF
:1000E000A4FAA8F075F00BE50B12803E7049E50A02
:1000F00075F00BA4F8AAF075F00BE50B12833A8E9D
:10010000828F83E085088285098312A203128659B3
:10011000EE2403FCE43F1281F8122DEB12A9D21257
:10012000BF2F1298EAD2E7F0123F2579019005120D
:10013000E0F50AA3E0F50B050AE50A7002050B12CB
:1001400085B5E50A9AE50B9B409102AE8574F512E0
:10015000242DEAFEEBFF750A01740B122CC71290D6
:10016000A9EC4D6015EC1282053D1287AA790112A7
:100170002DBBE508450960758023E5084509604405
:1001800012820335091287AA1281F9122DF1E9644E
:1001900001701BEEFAEFFB122DC1E9F50A8508820A
:1001A0008509831286517902AA08AB09801112864B
:1001B000DA122DF1E9640170347903EEFAEFFB12E3
:1001C0002DBB80298E828F83A3E064FE7003A3E0A1
:1001D000F4700B1286DA122DF1E96401700CEEFA5C
:1001E000EFFB122DC1E9F50A8003750A00028C1499
:1001F000E50A2403FCE4350BFDE5082403FAE435A5
:1002000009FB22E50812C4352274F712242D90054B
:100210001212AAEFEA4B602FEA75F00BA4FAA8F0CD
:1002200075F00BEBA428FBEAFEEBFF123CF1900506
:100230001412AAEF90051412B4E96012EEFCEFFD5F
:100240007900123C378007900514E4F0A3F002A86F
:100250001074F612242DE4F508F5097808122A2105
:100260009005121290A475F00BA4FCA8F075F00B89
:10027000EDA428FD7A237B00123D697402122A3412
:10028000E9FE6003122DD9EEF9028B2774F61224D1
:100290002D74FF122AC87E007F00803C851882855D
:1002A0001983E4128E13122A21750801750900784A
:1002B00008122A21EEFCEFFDEC75F00BA4FCA8F06F
:1002C00075F00BEDA428FD7A237B00123D757404B4
:1002D000122A340EEE70010F1283C240BF74010265
:1002E0008B2474F612242D7E007F008039EEF8EF07
:1002F000F912832E7808122A2175080B75090078E7
:1003000008122A21EEFCEFFDEC75F00BA4FC75F051
:100310000BEDA42AFD7A237B00123D7B7404122A84
:10032000340EEE70010F1283C240C2028B27E875B3
:10033000F00BA4F8AAF075F00BE9A42AF9900514C3
:10034000E028F508A3E039F5092274F612242D7E81
:10035000007F00804AEEF8EF1283A788828983E04D
:10036000A2E75036C2E7F085820885830978081233
:100370002A2175080B7509007808122A21EEFCEF76
:10038000FDEC75F00BA4FC75F00BEDA42AFD7A23AF
:100390007B00123D757404122A340EEE70010F12A8
:1003A00083C240B1028B27F9E875F00BA4F8AAF0DC
:1003B00075F00BE9A42AF9900514E028F8A3E039B8
:1003C000F92290051212A7F7C3EE98EF9922C08286
:1003D000C083EC4D60051246ED80097C087D0079F4
:1003E00000123C3702A38574F612242D7900EA4BE3
:1003F00060177800EA28F582E412BC4660047901AF
:10040000780808E8C3940840EB028B2774F712249D
:100410002D74F3122AC8ECFEEDFF8518828519832E
:10042000E4F004122CC7EAF0A3EB12A7E9122E0F96
:100430007403122CC7AC82AD83EEFAEFFB122DEBE6
:10044000EEFAEFFB122DF102A80B74F712242D74B3
:10045000F3122AC8ECFEEDFF851882851983E4F0BB
:10046000EAFCEBFD7403122CC7AA82AB83122DEBBE
:10047000AA18AB19122E157401122CC712A2108ED5
:10048000828F8312A7DA74FE68700374FF696004B8
:1004900079018002790002A80B74F712242DEAFE7C
:1004A000EBFF122DB5E9F50874016508701112858E
:1004B00002F4FA88828983E05A4480F0123F2502D0
:1004C000985F74F712242DEAFEEBFF7508008E8208
:1004D0008F83E0602A122DB5E9F508740165087074
:1004E0001E128502FA88828983E05A70128E828FEA
:1004F00083E04480FA88828983E04AF0123F250233
:10050000985F12A9D6129A371283A78E828F83E042
:100510002274F412242D8A088B097C007D00EA12D3
:1005200081FB122DEBE50812867379008508828520
:100530000983A3E064FE7003A3E0F460757E007F8E
:10054000008066EEFAEFFB1280326058EEFAEFFBA5
:10055000EA75F00BA4FAA8F075F00BEBA428FB9059
:100560000514E02AF50AA3E03BF50B85088285090E
:1005700083A312BC21850A82850B83A3E06A7003E2
:10058000A3E06B701FE50A2403FAE4350BFB122D80
:10059000F1E9640170061281F0122DEB1286687980
:1005A0000112D23A0EEE70010F1285B5EE9AEF9B52
:1005B000409102AE8590051212B500C32274F31269
:1005C000242D8A088B098A828B83128651EA12862F
:1005D00073750C00EA1281FB122DF1E96401706A57
:1005E0007E007F00805FEEF8EFF9E875F00BA4F86D
:1005F000AAF075F00BE9A42AF990051412D2ACE028
:10060000540F603CEEF8EFF9E875F00BA4F8AAF08F
:1006100075F00BE9A42AF9900514E028F50AA3E087
:1006200039F50B1281F01246E7E964017012850A70
:1006300082850B83128659128668750C0112D23A94
:100640000EEE70010F1283C2409CA90C7F0502269A
:10065000BDA374FEF0A304F022A312A7F7850882BD
:10066000850983A3129F1522E50812867DEEF0A36B
:10067000EFF02212867D74FEF0A304F02212C4393A
:100680003509F5832274F512242DEAFEEBFF8E82E4
:100690008F831286517C007D001286DA122DEBEEDC
:1006A000FAEFFB122DB5E9F50A7401650A702712FD
:1006B000A7F012832E850882F5831286E21281F953
:1006C000122DF1E96401700EE5082403FCE43509FC
:1006D0001286D9122DEB028C14FDEE2403FAE43FAE
:1006E000FB22A312BC2B129F152274F212242D742C
:1006F000E6122AC812879C750C017508007509005E
:10070000750A00750B00851882851983E4F0EE24C4
:1007100003FCE43FFD7403122CC7AA82AB83122DA5
:10072000EBAA18AB19122E15E96401701F740B1295
:100730002CC71287AC7401122CC712BC257003A3FE
:10074000E069604AA818A91988088909740D122C53
:10075000C712A202A312A210740E122CC712A7DA9B
:10076000740D122AA2122E0FE964017009740D1281
:100770002A9A880A890B780A122A21AC08AD09EE58
:10078000FAEFFB122DC77402122A34E9F50CEEFAC7
:10079000EFFB122E09A90C741A02BB81EAFEEBFFD3
:1007A00012A9D674FEF0A304F022F583129A37F949
:1007B00012A9D6129F1522C082C0837800790080CA
:1007C0000508E87001091285B5E89AE99B5029E807
:1007D000FAE9FBEA75F00BA4FAACF075F00BEBA4A8
:1007E0002CFB900514E02AFCA3E03B8C82F583E00F
:1007F000540F70CD79008002790102A385C082C0B8
:1008000083904FE1E49375F016A4FCADF079FF7A84
:100810000D7B0E123C3702A38574F612242DEAF8E4
:100820007508007D008012ED12BC38C3994009E0C4
:10083000FAE8C39A400205080D904FE1E493FAEDFF
:10084000C39A40E3AA087B00028B2774F012242D80
:1008500074F3122AC88A0C8B0D8C088D09890AEC56
:1008600045096016AA08AB09122E5D8A0E8B0FAEE1
:100870000EAF0FEE4F600302893E7B0080010B122A
:10088000BF25500F1289E670F5740D28FE740E39DD
:10089000FF80047E007F00EE4F7003028992904F2C
:1008A000D31289B960217403650A60067404650A6D
:1008B00070157A047903122E33904FE1E493FC9083
:1008C0004FD31289BF5029904FD11289B960287433
:1008D00001650A60067402650A701C7A02790112C9
:1008E0002E33904FE1E493FC904FD11289BF400723
:1008F0007A007B000289B68518828519837401F01D
:10090000122CC7E50CF0A3E50DF0AC08AD0974039B
:10091000122CC7AA82AB83122DEBAA18AB19122E88
:1009200021740B122CC7129F0E8E828F83A3A3A358
:10093000A3A3A3E412D402AA0CAB0D1233DF7800F8
:10094000E50A6007C39405500278048E828F83E520
:100950000CF0A3E50D12C9E6E50AF0E88E828F835C
:10096000A3A3A3A3A312BF365001097A027B0012EE
:10097000224612942AA312BB61A312946EE50A6068
:100980000DC3940350081293F91289D7800312946F
:1009900010F07A047900122E338A08904FE1E49324
:1009A000FAC3E5089AEB940040059014E6E4F012CF
:1009B00032B3EEFAEFFB028D721289CFE8492212B0
:1009C00089CFECC398F8E499F9C3EA98EB9922E44B
:1009D00093F8740193F922F9EE2414F582E43FF5BB
:1009E00083E8F0A3E922EB75F016A4F8A9F01294BD
:1009F00063F42274F212242D74F3122AC88A088B2D
:100A000009ECFEEDFF750A00EEFAEFFB122E5D8A8F
:100A10000C8B0DA80CA90DE8497003028AB78882D7
:100A20008983E065087004A3E065097003028AB752
:100A300088828983A3A3A3A3E0C394055079888205
:100A4000898312C86612AC53E0603488828983A31C
:100A5000A3A3A3E0C394035026904FCFE493FA746A
:100A60000193FB12974C904FD9E493FA740193FBD6
:100A7000E82414F582E439F583EAF0A3EB800DE86D
:100A80002412128ABEF0E82414128ABEF08518825D
:100A90008519837401F0122CC712C866F0EEFCEFC2
:100AA000FD7403122CC7AA82AB83122DEBAA18ABDC
:100AB00019122E21750A01A90A740D02BB81F58253
:100AC000E439F58374FEF0A3042274F612242D1287
:100AD0002E578A088B09A808A909E849601488825A
:100AE0008983A3A3A3A3E06009C3940550047901FB
:100AF00080027900803174F612242D122E578A0854
:100B00008B09A808A909E849601488828983A3A3EE
:100B1000A3A3E06009C39403500479018002790023
:100B200080057402122A347F020226BD74F6122454
:100B30002D122E578A828B83E5824583600BA3A3F7
:100B4000A3A3E0700479018002790080DAC082C03A
:100B500083EAFCEBFD7A007B0002A382C082C083A3
:100B60007C007D0002A38274F512242D74F3122AF6
:100B7000C8EAFEEBFF8C088D09C3EC94F8ED94FFF6
:100B80004004EE4F606A750A00801974FF650870B2
:100B90000474FF6509600B12CB637004A3E0650960
:100BA000603B050A904FE1E493F8E50AC398504092
:100BB000E50A1289E760EBEE4F60D0128BFB122C36
:100BC000C712A7E5122E1BE960D87403122CC7AC1C
:100BD00082AD83EEFAEFFB1246E7E960C5E50A75E0
:100BE000F016A4F8A9F0740D28FA740E39FB8004ED
:100BF0007A007B00740D122A34801B8518828519B7
:100C0000837401F0740F28F582740E39F58312A7EE
:100C1000F7740B22A90A7F030226BD74F412242D57
:100C200074F3122AC8750800122E5D8A0A8B0BAE67
:100C30000AAF0BEE4F601F128C7E128C0E122CC767
:100C400012A7E5122E037C167D0079FFEEFAEFFB6A
:100C5000123C377508017A047900122E338A0A9003
:100C60004FE1E493FAC3E50A9AEB9400500990141B
:100C7000E67401F01232B3A908740D02AE82851831
:100C8000828519837401F08E828F83A3A32274F767
:100C900012242DE9FC74FE6A700374FF6B7D0070F2
:100CA00003802C0D128CF05026ED1289E760F412AF
:100CB000D6476A7003A3E06B70E98012ED75F016F9
:100CC000A4F8A9F012D63A6018E0640360130D127C
:100CD0008CF05015EC60E512945760F2C394055007
:100CE000ED12CDA712BC1E80047AFE7BFF02A81075
:100CF000904FE1E493F8EDC39822122E6F02A38582
:100D0000C082C083790180F274F012242D8A0A8B8C
:100D10000B7A047901122E338A0C8B0DEA450D6093
:100D200040EA2AFAEB33FB123CF18A088B09AE0841
:100D3000AF09EE4F60267AFE7BFF122E7574FE6AB5
:100D4000700374FF6B601E85088285098312AAEF09
:100D5000E5082402F50850E2050980DE750C0080E4
:100D6000047E007F00850A82850B83E50C12AA238E
:100D70008005740D122A347F080226BDE493F8EC36
:100D8000C3982274F612242DE4F508F509780812A8
:100D90002A21904FE1E493F50874037808122BDEC2
:100DA000129096123D697402122A34E9FE740A6E9A
:100DB0006024E4F508F5097808122A21904FE1E44F
:100DC0009325E0FCE433FD7A3F7B00123D69740219
:100DD000122A34EE6003122E8702828774F61224E0
:100DE0002D74FE122AC8851882851983E4F0A31297
:100DF0008E13122A217508027509007808122A211B
:100E00007C007D007A227B00123D757404122A3426
:100E1000028B22F0A818A919880889097808227479
:100E2000EE12242D74E4122AC88A0E8B0F8C088DC2
:100E300009750C007A227B00123D6F8A0A8B0B7AAF
:100E40003F7B00123D6F8A108B11AE10AF11E50A87
:100E5000450B6017E508650A7004E509650B600B32
:100E6000AC0AAD0B7A227B00123D817430122CC784
:100E7000E0F50AA3E0F50BEE4F6015E50A6E70038E
:100E8000E50B6F600BEEFCEFFD7A3F7B00123D81BE
:100E9000E4F510F5117810122A21AC08AD097A2278
:100EA0007B00123D697402122A34E9640A7003025D
:100EB000908CE4F508F5097808122A21AC0AAD0BEC
:100EC0007A3F7B00123D697402122A34E9640A7089
:100ED0000302908C7404122A9A88088909780812EF
:100EE0002A217508027509007808122A217C007DE4
:100EF000007A017B03123D7B7404122A34E96003FB
:100F000002908C851882851983E4F0A3F0FE02908C
:100F1000037406122A9A880889097808122A21750A
:100F200008087509007808122A218E0874037808C9
:100F3000122BDEE5082402FCE43509FD7A017B036F
:100F4000123D7B7404122A34E9600302908C740809
:100F5000122CC7E0F47003A3E0F470030290027453
:100F600006122A9A880889097808122A2175080821
:100F70007509007808122A217404122CC71290A94E
:100F800074037808122BDE129096123D75740412C9
:100F90002A34E9600302908C7402122A9A88088924
:100FA000097808122A217508027509007808122AA2
:100FB00021EE25E0FCE433FD7A027B03123D7B74D5
:100FC00004122A34E970387402122A9A88088909AE
:100FD0007808122A217508027509007808122A215A
:100FE0007404122CC71290A42CFCED33FD7A3F7BC5
:100FF00000123D757404122A34E9600302908C12C9
:10100000955F0E851882851983C082C083904FE159
:10101000E493F8D083D082C3E098A3E094005021F9
:10102000851882851983C082C0837404122CC7126C
:10103000A210D083D082C3E098A3E0995003028F1E
:1010400011A818A919880889097808122A21750891
:10105000027509007808122A217C007D007A227B23
:1010600000123D757404122A34E97020AC0EAD0FE5
:101070007A017B03123D81E97012742E122CC71283
:10108000D4067A027B03123D81E96003750C01A945
:101090000C741C02B14AE5082402FCE43509FD7A0F
:1010A000227B002212D40AEC22E0F508A3E0F50925
:1010B0002274EC12242D74FE122AC8750A008518B9
:1010C00082851983E4F0A3F0904FE193F510F508C1
:1010D00075090074037808122BDEE5082402F50870
:1010E00050020509E51025E0F510E433F5117A22E8
:1010F0007B00123D6F8A0C8B0DAE0CAF0D7A3F7BDF
:1011000000123D6F8A0E8B0FA818A919880C890D43
:10111000780C122A21750C02750D00780C122A2108
:101120007C007D007A227B00123D7B7404122A34FD
:101130007A017B03123D6F8A0C8B0D7A027B0312BE
:101140003D6F8A128B13A812A913E50C450D700A86
:10115000E5086E7003E5096F7025E849700CE5102D
:10116000650E7004E511650F7015E50C450D607B8B
:10117000EE4F604E85188285198312AAF560437C74
:10118000017D037A227B00123475E9F8880A705BCE
:101190007C027D037A3F7B00123475E9F8880A707F
:1011A0004AEEFCEFFD7A227B00123D81E9700EAC25
:1011B0000EAD0F7A3F7B00123D81E96011750A0187
:1011C0008029AE0CAF0DE8496004880E890F7810B5
:1011D000122A21780E122A21AC08AD09EEFAEFFB93
:1011E000122E8D7404122A34E9F50AA90A74021227
:1011F0002A347F0C0226BD74F112242D74D9122AD0
:10120000C87402122CC7E4F0A3F0122E93E9600315
:101210000293E87402122A9A880889097808122A27
:10122000217508027509007808122A217C007D00CA
:101230007A227B00123D7B7404122A34E960030297
:1012400093E8904FE1E493FA7402122CC712A210B3
:10125000C3EA98E49950030293E8750A00750B00FD
:10126000750800803E85188285198312BD0A12CD4B
:101270009A12A7DA851882851983129A371289D7AC
:10128000F07A047900122E338A0C904FE1E493FA3D
:10129000C3E50C9AEB940040059014E6E4F012329A
:1012A000B30508904FE112BB4040030293E874027B
:1012B000122CC712A210C3E50A98E50B994003024D
:1012C00093E87411122A9A880C890D780C122A213D
:1012D000750C08750D00780C122A2185080C740312
:1012E000780C122BDEE50C2402FCE4350DFD7A228D
:1012F0007B00123D7B7404122A34E970A47413122B
:101300002CC7E0F47003A3E0F46096050AE50A70C8
:1013100002050B7404122CC77401F07413122CC74D
:1013200012A210740F122CC712A7DA7404122AA288
:10133000122E1BE970030292A112D4037411122C15
:10134000C712BC211233DFE50875F016A4F8A9F026
:10135000740D28FE740E39FF7411122A9A880C89B4
:101360000D750E00780C122A1D7C087D00EEFAEF38
:10137000FB123C2B7403122A3412BF3B5001097A32
:10138000027B0012224612942A12946EA818A91900
:10139000880C890D780C122A21750C02750D0078C5
:1013A0000C122A21AC08EC2CFCE433FD7A3F7B00C4
:1013B000123D7B7404122A34E9600302928185187D
:1013C00082851983E0F47003A3E0F4600302926560
:1013D000E508129458600BC3940350061293F90267
:1013E000927D1294100292807402122CC7E0F9745C
:1013F00027122A347F070226BD904FCF1289CFEEE5
:1014000012CD9E129F15904FD9E493F87401932248
:10141000EE241212941EF0EE241412941E22F58271
:10142000E43FF58374FEF0A30422E88E828F83A349
:10143000A3A3A3A3A3A3A312944F740112944FA335
:1014400074AAF0EE2410F582E43FF583E4F0221252
:10145000CA09A3A3A3A322ED75F016A4F8A9F0125C
:10146000946322741128F582740E12D4F622A3F02C
:1014700012A9D6E4F0EE240CF582E43FF583E4F003
:10148000A3F0A3F0A3F02274F312242D74FE122A09
:10149000C8851882851983E4F0A3F0F50C02952025
:1014A000E50C75F016A4F8A9F0740D28F50A740E71
:1014B00039F50B850C82AE82780A122A217508084C
:1014C0007509007808122A218E0874037808122BF7
:1014D000DE129096123D757404122A34E50A241423
:1014E000F508E4350BF5097808122A21750802750C
:1014F00009007808122A21EE2EFEE433FFEEFCEFFD
:10150000FD7A3F7B00123D757404122A34850A82ED
:10151000850B83A3A3A3A3E0F4600312955F050CDE
:10152000904FE1E493F8E50CC39850030294A0A80F
:1015300018A919880889097808122A2175080275DE
:1015400009007808122A217C007D007A227B001293
:101550003D757404122A347402122A3402864C85B2
:101560001882851983E02401F0A3E03400F022C042
:1015700082C0837D008009EA24FF1AEB34FFFB0D53
:10158000128CF05016129457C3940550F2EA4B7027
:10159000E6740D28FA740E39FB80047A007B000291
:1015A000A38574F712242D74F3122AC87E000296C4
:1015B0003AEF75F017A4F8A9F012D61D12BD077501
:1015C000F016A4FAABF0740D2AF582740E12BF590E
:1015D0007003A3E0696040EF75F017A4F8AAF0EA81
:1015E000F912D61D39F58312A2107401122CC7E02E
:1015F000687003A3E069601FEF75F017A4F8EAF9BB
:1016000074DD28FC740F39FD7403122CC7AA82AB59
:10161000831246E7E96013EF75F017A4F8A9F07498
:10162000DB28FA740F39FB1233EB0F904FDCE49395
:10163000F8EFC39850030295B10E904FE112D18C90
:10164000501FEE12D640F47003A3E0F460EB128B4F
:10165000FB122CC712A7E5122E1BE960DC7F00806D
:10166000CA02A80B74F712242D74F3122AC890052D
:10167000E512B4E97003029710750800802BE508A5
:1016800075F016A4F8EAF9742128F582740E12D4C4
:10169000F264FE7003A3E0F4600D741F28F58274F9
:1016A0000E39F58312BB770508904FE112BB40500D
:1016B0005FE50875F016A4F8AAF0EAF912945F60E5
:1016C000E6C3940350E1741F28F582740E12B4E649
:1016D00070ACE50875F016A4F8EAF9740D28F874F2
:1016E0000E39F9E8FEE9FF1297AE1297A412261EF2
:1016F000128C7E128C0E122CC712A7E5122E1BE93B
:1017000060A57403122CC7AA82AB83122E6980973E
:1017100002A80B74F612242D122E578A088B09A8E2
:1017200008A909E849602088828983A3A3A3A3E0CC
:101730006011C39403500CE82414F582E412BC1E1B
:1017400012974C790180027900028B27E82412F568
:1017500082E439F583EAF0A3EBF02274F712242D2A
:10176000EAFEEBFF9005DF12B4E960309005E51268
:10177000B4E960289005E912B4E9602012CEE812BD
:10178000261EE9701712979F12261EE96401700C3D
:101790008E828F83A3A312CED512261E02A810120A
:1017A00097AEA3A312B5009005E512CEDF22904FAD
:1017B000D9E493FC740193FD8E828F8322C082C092
:1017C0008390051B746FF0A37431F090051D74694C
:1017D000F0A37431F09005217465F0A3742FF0022A
:1017E000A385C082C08390051F7463F0A37431F099
:1017F00002A38574F712242DEAFEEBFF900555E055
:101800006408601CE0640460178E828F83E05403D8
:101810006401704112B8D9F8129864E0640670351A
:101820008E828F83A3A3E064FE7003A3E0F460259F
:101830008E828F83A3A312C41B7003A3E069700878
:10184000EE241512C410600512322F8003123235B7
:10185000E9F50880037508C2EEFAEFFB123CF7A920
:101860000802A810A3E0F58388822274F412242DC4
:101870008A088B09129A33FAE82AFAE43400FB1238
:101880003CF18A0A8B0BAE0AAF0BEE4F6055850810
:1018900082850983E0FC7D007900123C378E828FBF
:1018A00083A312865112326B8E828F83A3A3A3A3CC
:1018B000EAF0A3EB1298EAF8EE28F8E43F1287AFBB
:1018C000850882850983A3E0C0E012BF1BD0E0F049
:1018D00012327D12BF11E9129EF1E0C0E0129EE7C4
:1018E000D0E0F0EEFAEFFB02AE85F08508828509C4
:1018F00083E02274F412242D74E8122AC88A088B1B
:10190000098C0A8D0BE9FE900555E064046005E042
:101910006408700479C2803CA37808122C61EE90B0
:10192000055C129B76123C378518828519837808EE
:10193000122C617405122CC7EEF07404122CC774BB
:1019400001F07407122CC7E4F0900555740212A739
:10195000E91247D702AE8074F412242D74E8122ADB
:10196000C8EAFEEBFF90051612B4E96003029A2E56
:101970007A077B00123CF190051612AAEF9005162B
:1019800012B4E97003029A2A8E828F83122CA490DB
:101990000516E0FCA3E0F5838C82122CB0EE240443
:1019A000F50AE43FF50B850A82F583E0C0E0900577
:1019B0001612B4BDA3A3A3D0E0F0EE2405F508E40D
:1019C0003FF509850882F583E0C0E090051612B462
:1019D000CBD0E012A7DFC0E0900516129A37C824DA
:1019E00006F582E438F583D0E0129B76123C378E00
:1019F000828F83122CA4851882851983122CB085BE
:101A00000A82850B83E0C0E07405122CC7D0E01277
:101A100098EAC0E07404122CC7D0E0F07407122CCE
:101A2000C7E412A7E91247D780067910800279012E
:101A300002AE808A828B83E0F8A3E022C082C0835A
:101A400090051612B4E9601090051612BC21123CE4
:101A5000F7900516E4F0A3F012319912338B02A32C
:101A60008574F412242D74E8122AC88A0A8B0BECB0
:101A7000FEEDFF89087428122CC7E0FC7429122C93
:101A8000C7E0FD740F6C7005740F6D6012901554F3
:101A9000E064026005ECC39D500579C1029B73743C
:101AA00024122CC7122CA4900556122CB0E50890D5
:101AB000055CF0EC90055AF0EDA3F0742A122CC7E7
:101AC000E090055DF074FF650A700474FF650B70AB
:101AD00024901568E0F47003A3E0F4700C123C4904
:101AE000900553EAF0A3EB801290156812CDC4E87C
:101AF000F0A3E9800690055312BF2FF0EE4F601758
:101B0000EEFAEFFB12343FE96401700BEEFCEFFDDF
:101B10007A677B051246ED900546E4F0A3F0900548
:101B200049F0A3F0900566F0901554E06402700847
:101B300090055A740FF0A3F09005557405129B762A
:101B4000123C377404122CC7E4F0900556122CA4F2
:101B5000851882851983122CB090055CE0C0E07472
:101B600005122CC7D0E0F07407122CC7E412A7E9C5
:101B70001247D702AE80F07C187D007900AA18AB1E
:101B8000192274F712242DE990051AF07A807B004F
:101B90009005A0E0F9123DC3122EFF790002A810B3
:101BA000C082C08390051AE07003124069122EFFB4
:101BB00002A38574F012242D90051AE09014E570AC
:101BC0000FE060057900123EE99014E5E4F0804AE8
:101BD000E06401600890051AE0F9123EE99014E50E
:101BE0007401F090051AE0F46030E0F50CE4F50DB6
:101BF000F50EF50FF09080AC7808122C70780C7907
:101C00000812233E780C122A197A807B009005A0D6
:101C1000E0F9123DB77404122A347AE57B14794155
:101C20001247BF028D7774F712242D7CFE7DFF12C0
:101C30002F0B02A81074F212242DEAFEEBFF8C0881
:101C40008D09890A900555E06408706C122E5D8B31
:101C50000DEA450D600479C5806074FE6508700466
:101C600074FF6509701C7402550AF91230378A082E
:101C70008B0974FE6508700474FF6509700479C7E8
:101C80008038E50AA2E1500CA2E350047904800EEA
:101C90007903800AA2E35004790280027901EEFC04
:101CA000EFFDAA08AB09122E398B09EA4509600439
:101CB000790080067910800279C202BB8474F41224
:101CC000242D74E8122AC88A088B098C0A8D0BE926
:101CD000FE9005557401129B76123C37851882855B
:101CE00019837808122C617405122CC7EEF0740465
:101CF000122CC77403F07407122CC7E412A7E91260
:101D000047D702AE8074F712242D7C01122F2302D4
:101D1000A81074F712242D7C0080F174F012242D89
:101D200074FC122AC8E9851882851983F0EAFEEB53
:101D3000FF8C0A12D40312318D8A088B09EA4509F7
:101D4000700579CA029EE28A828B83A3A3A3A3A310
:101D5000A3A3E064FE7003A3E0F4700579C3029EC0
:101D6000E212326B8A0C8B0DA80CA90D85088285B6
:101D70000983A3A3A3A3A3A3A3E0687003A3E069BB
:101D8000700579C2029EE290055312A21085088266
:101D9000850983E0687003A3E06960128508828585
:101DA000098312A068AA08AB0979501247BF9005B1
:101DB0005312BC211233F1850882850983A3A3A3A2
:101DC000A3A3A3A3A3A3A3E00490056612A05412A7
:101DD00046ED7402122CC77402F014122AA21232B9
:101DE000E98A0C8B0DAE0CAF0DEE4F7003029ED83E
:101DF00012AE097406F0A3A882A98390054012C010
:101E00004712B8B612326512AAE6EE241312B8B918
:101E100012BF077440F0A3E4129EF1A3A3A3A3A3EF
:101E2000129F0E129EE7E50A12AA23122ECFE9F5A1
:101E30000B6003029EDB9005557409F0E50824074A
:101E4000FEE43509FFEEFAEFFB794B1247BF8E82B5
:101E50008F8312A05E900548E0F88518828519836B
:101E6000E068600CE090054812A7E979E11247BFED
:101E700090154012A210901542E0687003A3E0692B
:101E8000602890051812A7DA90154212BC21123270
:101E900095129EFB780C122A197A017B009005A0FE
:101EA000E0F9123DB77404122A347A007B049005DD
:101EB000A0E0F9123DC3129EFB7402780C1229C1F6
:101EC000780C122A197A007B049005A0E0F9123DE3
:101ED000B77404122A348003750B1090078CE4F059
:101EE000A90B7404028D74EE2411F582E43FF5838E
:101EF00022F0850882850983A3A322901542E0F58C
:101F000008A3E085080CF50DE4F50EF50F2212BFCD
:101F100051129F1522E8F0A3E9F02274F612242D45
:101F200074E2122AC8851882851983ECF0A3EDF0BB
:101F3000EAFEEBFF8908900555E064046005E06463
:101F400008700579C202A04F7429122CC7E064FE04
:101F50007003A3E0F4700579C302A04F7C197D00E3
:101F600079007405122AA2123C37900555740312A9
:101F7000A7E979501247BF7429122AA2794B124758
:101F8000BF85188285198312A068E508900548F07E
:101F90007429122CC712A05E7428122CC7E0F50910
:101FA00090054012A0541246ED74CE55094480C0ED
:101FB000E0741D122CC7D0E0F0900912E0600464B8
:101FC00001700B742B122CC7E004900566F0741A94
:101FD000122CC77402F07429122CC712A2107412AA
:101FE000122CC7E8F0A3E912A209741B122CC71225
:101FF000A7DA7410122CC7E508F0740D122CC7E490
:10200000F090055B740FF07A5B7B0579541247BF43
:1020100090055A740FF07A5A7B0579471247BF90A2
:10202000055AE0C3940F501F7410122CC7E0C0E093
:102030007402122CC7D0E0F07404122CC77401F0A3
:1020400004122AA21247E37405122AA21247C57489
:102050001E028B24F0EEFCEFFD7A677B052212A7AF
:10206000F7900549129F152212CDC8129F152274B0
:10207000F712242DEB90055DF012317B02A810744D
:10208000F712242D74E9122AC8EAFEEBFF75080046
:102090008E828F83A3A3A3E0C0E07406122CC7D066
:1020A000E0128C86E0C0E07408122CC7D0E0F07417
:1020B00009122CC7740112A20312B4E9600D8E82BA
:1020C0008F8312BC21122DF1E970357407122CC7D1
:1020D000E4F01232657404122CC712AAEF90055571
:1020E000E06404700E1232717402122CC7EAF0A37D
:1020F000EB80557402122CC774FDF0A374FF804866
:10210000900912E060076401600302A194AC18AD6D
:10211000198E828F8312BC21122DFD8E828F83A394
:10212000A3A3A3E070307407122CC7740112A20994
:102130007402122CC712A7DA8E828F8312A2107437
:1021400004122CC7E8F0A3E9F07402122AA212329A
:10215000D1E9F508803E12A20A740A122CC712A710
:10216000DA7414122CC7128C84A3E0C0E074151228
:102170002CC7D0E0F07416122CC712A20212D4069B
:10218000740C122CC7AA82AB831246ED740A122A71
:10219000A2123F01A908741702A80D74F712242D8A
:1021A00074F8122AC8EAFEEBFF7900900555E06446
:1021B000086005E06404704585188285198374FD04
:1021C000F0A374FFF01232657402122CC712AAEF4A
:1021D0007405122CC712A202A3E0C0E07404122CF2
:1021E000C7D0E012A203E0C0E07406122CC7D0E012
:1021F000F07407122CC7E412A7E91232D174080256
:10220000A80DE4F08E828F8322F0851882851983D1
:1022100012A7F72274F112242DECFEEDFF7C008C46
:102220000BE92479602B24FC700302A2B424F36030
:102230001324FC601514603A14600302A320900577
:102240005502A33F90054302A33F1233D9EA02A3EC
:1022500040750BC11233E58A0C8B0D8B09EA4509D9
:10226000700302A345750E00780C122A1D7C17021C
:10227000A30D750BC9900912E060076401600302A9
:10228000A345784B79117A00801788828983E064AE
:10229000FE7003A3E0F460010CE82407F850010984
:1022A0000A904FF5E493FBEAC39B40DEEC8E828FED
:1022B00083F08067750BC9900912E06007640160C4
:1022C0000302A345750BC175084B75091178008091
:1022D0000C0CE5082407F5085002050908904FF595
:1022E00012C8CA5060850882850983E064FE7003C5
:1022F000A3E0F460DD8C0CEA650C4B70D485080C0F
:1023000085090D750E00780C122A1D7C077D00EEE4
:10231000FAEFFB123C2B7403122A34750B00802554
:10232000747F29C3941E4005750BC9801874322927
:10233000F8E43405F9E8247FF582E934FFF583E019
:102340008E828F83F0A90B0293F4C082C083900524
:10235000277407F0A37430F09005CD7431F0A374A6
:1023600033F090052B743DF0A37430F090052D747C
:1023700007F0A37430F090052F7443F0A37430F08D
:102380008003122E63D083D0820229E674F41224D3
:102390002D74F9122AC88A088B098C0A8D0B8518AE
:1023A000828519837808122C617404122CC7E9F015
:1023B0007405122CC7E4F07406122CC7E412A7E9C6
:1023C000122EE1740702AE8274F512242D8A088B56
:1023D000098A828B8312D23DEE4F700302A5809052
:1023E00004E412B4E960158A828B83A3A3E0F9EEBA
:1023F000FAEFFB9004E512986512261E8E828F83F9
:10240000A3A3A3A3A3A3A3A3A3E06402600302A4C2
:10241000E98E828F83A3A3A3A3A3A3E05402700336
:1024200002A50D850882850983A3A3E064E97003F2
:1024300002A50D850882850983A3A3E064CD7003FE
:1024400002A50D850882850983A3A3E064F07003CB
:1024500002A50D8E828F83A3A3A3A3A3A3A3A3A3EB
:10246000A3E07016901558E0048E828F83A3A3A377
:10247000A3A3A3A3A3A3A3F0801012A591123307D3
:10248000E970077A307B011242CD85088285098385
:10249000A3A3E0701F750A0080097A367B011242FF
:1024A000CD050A850882850983A3A3A3E0F8E50A80
:1024B000C39840E68E828F83A3A3A3A3A3A3A3A361
:1024C00012C9FDA3A3A3A37404F090155912BF4B26
:1024D000E812A583123DC9EA4B4C4D700C7A207B63
:1024E000009005A0E0F9123C918E828F83A3A3A3F4
:1024F000A3A3A3A3A3A3E0640260128E828F83A38D
:10250000A3A3A3A3A3A3A3A3E0640670738E828FE7
:1025100083A3A3A3A3A3A3E0A2E0506485088285BC
:102520000983A3A3E0F9EEFAEFFB1249698E828FCB
:1025300083A3A3A3A3A3A3E054FEF012A591123397
:1025400007E9850882850983A3A3702AE070237AAE
:102550002F7B011242CD7E00850882850983A3A3CB
:10256000A3E0F8EEC39850187A367B011242CD0EE4
:1025700080E67A318005E070077A2D7B011242CD2A
:10258000028C16F0A3E9F07A207B009005A0E0F918
:10259000228E828F8312CEDF12B5002274EC1224B9
:1025A0002D74DB122AC8EAFEEBFF8C108D11750E1C
:1025B000007405122AAA122D5B7412122CC7E07047
:1025C000087415122CC7E060207405122CC7E0A215
:1025D000E6501B8E828F83A3A3A3A3A3A3A3A3A3CD
:1025E00012BC21123307E960057A3502A6E57405AD
:1025F000122CC7E0540C64047005750D018003753E
:102600000D00E0A2E55030750E01E50DA2E0402777
:1026100012326B8A088B09A808A90912B8D9687008
:1026200003A3E06960117405122AAA12C42A124891
:10263000D9E9600302A6E37405122CC7E0A2E650B4
:10264000227406122CC7E0540370187405122CC7AC
:10265000E0540C640C600CE0540C64086005750CCC
:10266000018003750C007405122CC7E05403F87444
:102670000268700E7405122AAA12C42A122D6D0265
:10268000A7CF7401687041E50CA2E0500B740512ED
:102690002AAA12C42A122D617405122A9A740312EE
:1026A0002CC7E8F0A3E912A7EF851882851983E803
:1026B000F0A3E912A7DFC0E07402122CC7D0E01229
:1026C000A7E9124A1702A7CFE8600302A7CF900537
:1026D0003DE0640170178E828F83A3A3A3A3A3A3FD
:1026E000E0700A7A347B011242CD02A7CF74241223
:1026F0002CC7740212A7EF741C122CC712A7DAE5BC
:102700000CA2E0500B7405122AAA12C42A122D61E1
:102710007439122CC77808122C70E50DA2E0EE5027
:1027200072240F12C410C0E07417122CC7D0E0F04E
:102730009004E612B4E9700302A7CF12326B8A123A
:102740008B13A812A913741C122CC7E0687003A382
:10275000E069707B7808122A19E50EF508780812EE
:102760002A258E828F83A3A3A3A3E0F508780812FD
:102770002A257810122A21A90C740D122AAA742471
:10278000122AA29004E612BC9312261E7408122A82
:1027900034803C12C40EF50C780C122A25780812ED
:1027A0002A19E50EF5087808122A257810122A2130
:1027B000900553122845EE241212C410F974261203
:1027C0002AAA740F122AA212495D740A122A3474BA
:1027D000250291EFA3A3A3A3A3A3E8129F1622129D
:1027E000CA05A3E022E8F0A3E9F0AA18AB1922F089
:1027F00012A9D612A7F72212A7FB22E0F8A3E0F94C
:102800002274F712242D123EC58005740D122A344D
:102810007F010226BD74F712242D123ED180F1747F
:10282000F712242D123EDD80E7C082C083123ED70E
:1028300002A38574F712242D123EE380D374F7129D
:10284000242D7409122CC7E0F5087808122A2512E5
